:100000000C94F1000C946B010C946B010C946B013B
:100010000C946B010C94F2170C946E160C946B01FB
:100020000C946B010C946B010C946B010C946B01A0
:100030000C946B010C946B010C946B010C946B0C85
:100040000C946B010C946B010C94DA160C943E1713
:100050000C946B010C946B010C946B010C946B0170
:100060000C946B010C946B010C946B010C946B0160
:100070000C946B010C946B010C9497110C94091166
:100080000C946B010C946B010C946B0100780A7852
:100090001178177821782F78FD77FD77FD77FD7738
:1000A0003E784478477859785C786778FD776A7845
:1000B0007078737879787C78827885788D780A0082
:1000C00072252E32787C000A0077252E32782000A7
:1000D0000A007C0072252E327820005445524D498A
:1000E0004E414C204552524F523A2063616E6E6F22
:1000F0007420616C6C6F63206D656D6F72790A009E
:1001000025630021214C494E4520544F4F204C4F30
:100110004E4721210A0025632025630025733A20DC
:10012000636F6D6D616E64206E6F7420666F756EA7
:10013000640A000A002563202563000A20756172A5
:10014000742072656164206572723A2025640A0029
:1001500042544E5F5445524D494E414C3A2045520F
:10016000524F523A207768696C6520726561646904
:100170006E672066726F6D20756172740A00666129
:10018000696C65642120636D6473206275666665C1
:10019000722066756C6C210A0072656769737465FC
:1001A00072696E6720636D643A2573200066616929
:1001B0006C656421206E616D6520746F6F206C6FBB
:1001C0006E67210A007265676973746572696E678C
:1001D00020636D643A257320000A0009000A000AB2
:1001E000000085B7806885BFECE6F0E0808180681C
:1001F0008083BF9ABE9AC798C69880EC85BFAF9A95
:10020000A79AAE9AA69A81EE8093008380E48093A9
:10021000018385B78F7785BF80E090E09D9B05C007
:10022000019641F09D9BF8CFFBCF019619F09D9967
:10023000F3CFFBCF85B7806885BFAF98A798AE98FE
:10024000A69887E089B98093990011241FBECFEF4B
:10025000D0E1DEBFCDBF17E0A0E0B1E0EEE2FBE011
:1002600001E00BBF02C007900D92A037B107D9F78C
:100270001BE0A0E7B7E001C01D92AA34B107E1F787
:100280008FEF9FEF9EBF8DBF2AE43BE0C9018095B1
:1002900090958158914038F06FEF7EEF621B730BA1
:1002A000C9010E9408090E944209892B41F067E4B4
:1002B00073E08CEE98E00E94B9840E94290920E83E
:1002C00031E040E050E067EA73E080E593E00E94AF
:1002D000070B0C9400000C940000EF92FF920F9318
:1002E0001F93CF93DF93EC0120E030E042E953E02D
:1002F00067E070E10E9403277B018C0197FF05C036
:1003000080E091E00E94031905C040E050E0CE017A
:100310000E946F27C801B701DF91CF911F910F9104
:10032000FF90EF9008958F929F92AF92BF92CF92DD
:10033000DF92EF92FF920F931F93CF93DF93CDB78E
:10034000DEB724970FB6F894DEBF0FBECDBF80E0B6
:100350009BE4A0E0B0E089839A83AB83BC830E94D6
:10036000225381E00E94FB6301E613E040E060E07D
:1003700070E0C8010E94EC03409173045091740432
:1003800061E271E0C80102960E94781880917304BE
:10039000909174040E941818AE014F5F5F4F61E0A6
:1003A00071E00E9478190E942B6684E291E09F938D
:1003B0008F930E94E31884E591E00E9403198CE773
:1003C00091E09F938F938AE891E09F938F930E948F
:1003D000E31881EA91E09F938F930E94E31880EDE8
:1003E00091E09F938F930E94E3180E943B538EEEFF
:1003F00091E09F938F930E94E31884EF91E09F9385
:100400008F930E94E3188DED93E00E9489234C01A5
:1004100096E0A92E92E0B92EC5010E9403198CE046
:1004200092E09F938F930E94E31860E074E0C40110
:100430000E941A24C5010E94031986E292E09F934C
:100440008F930E94E31844E050E060E170E0C40143
:100450000E9481276C01C5010E94031983E492E088
:100460009F938F930E94E318B601C4010E949F28B6
:10047000C5010E94031981E692E09F938F930E9429
:10048000E31885EAE82E83E0F82E012D112D24EFE4
:100490003FE143E050E1B601C4010E94495AC50161
:1004A0000E9403198DE792E09F938F930E94E318B7
:1004B0000AEE13E526E030E045E050E1B601C40164
:1004C0000E94EB6AC5010E94031967E070E1C60152
:1004D0000E946D0168EA72E0809173049091740447
:1004E0000E943E7189EB92E09F938F930E94E318E4
:1004F00064E273E080EE92E00E94267266EA72E0A7
:1005000086EE92E00E94267260E070E081E00E9438
:10051000B7758DB79EB74A960FB6F8949EBF0FBEBB
:100520008DBF80E090E024960FB6F894DEBF0FBE3A
:10053000CDBFDF91CF911F910F91FF90EF90DF9092
:10054000CF90BF90AF909F908F900895EF920F93B0
:100550001F93CF93DF93CDB7DEB762970FB6F894B2
:10056000DEBF0FBECDBF8E01095F1F4F1F930F93DC
:100570009E01275F3F4F3F932F939E01255F3F4F83
:100580003F932F939E01235F3F4F3F932F939E01F5
:10059000215F3F4F3F932F939E012F5E3F4F3F932D
:1005A0002F932CEE32E03F932F939F938F930E94D3
:1005B0001A192DB73EB7205F3F4F0FB6F8943EBFD4
:1005C0000FBE2DBF069761F5F801DE0111969E0161
:1005D0002D5E3F4F80818D933296E217F307D1F75E
:1005E000EE2401E027E030E1AE014F5F5F4F60E0B5
:1005F00070E080E090E00E94F06D9F938F937F9376
:100600006F9384E093E09F938F930E94E46F8DB784
:100610009EB706960FB6F8949EBF0FBE8DBF08C05A
:100620008AE193E09F938F930E94E46F0F900F9065
:1006300062960FB6F894DEBF0FBECDBFDF91CF91AB
:100640001F910F91EF900895EF920F931F93CF9307
:10065000DF93CDB7DEB762970FB6F894DEBF0FBE5B
:10066000CDBF8E01095F1F4F1F930F939E01275F20
:100670003F4F3F932F939E01255F3F4F3F932F9313
:100680009E01235F3F4F3F932F939E01215F3F4F7A
:100690003F932F939E012F5E3F4F3F932F932CEE5E
:1006A00032E03F932F939F938F930E941A192DB797
:1006B0003EB7205F3F4F0FB6F8943EBF0FBE2DBF31
:1006C0000697E1F4F801DE0111969E012D5E3F4F81
:1006D00080818D933296E217F307D1F7EE2400E084
:1006E00027E030E1AE014F5F5F4F60E070E080E0F7
:1006F00090E00E94F06D85E393E002C08AE193E010
:100700009F938F930E94E46F0F900F9062960FB6A5
:10071000F894DEBF0FBECDBFDF91CF911F910F9137
:10072000EF9008950F931F938C01FC0180819181BC
:100730000E94696B25E043E06FE082E00E944F6316
:10074000C8011F910F91089580935A0308950E9444
:10075000AD0420E033E040E050E063E971E085E57E
:1007600093E00E94070B8EEF0E948C070E941008F6
:100770000E94570720915A032F3FC1F395B785B7C1
:10078000837E822B85BF85B7806285BF889585B7BC
:100790008F7D85BF85B7837E9C71892B85BFE6CF12
:1007A0000F931F93CF93DF938C01C0917107D0916A
:1007B00072070AC0B801CE0102960E94AF84892B4D
:1007C00029F00990D881C02D2097A1F7CE01DF91A3
:1007D000CF911F910F910895CF93DF93EC01892B57
:1007E00011F16115710511F07D876C8741114E87FC
:1007F000CE0102960E94D003892BA9F4EB89FC89D3
:10080000309721F0CE010995892B69F48091710709
:100810009091720799838883D0937207C093710770
:1008200080E090E002C08FEF9FEFDF91CF910895BD
:100830008091DB089091DC08A091DD08B091DE0882
:100840000196A11DB11D8093DB089093DC08A09355
:10085000DD08B093DE080895CF93DF93EC011B828F
:100860001A82E091D908F091DA081AC028853985F2
:100870004A855B8580859185A285B38528173907D0
:100880004A075B0780F0281B390B4A0B5B0B288754
:1008900039874A875B87FB83EA830190F081E02DEB
:1008A000309721F718C0821B930BA40BB50B8087E0
:1008B0009187A287B387F983E883D383C283EA81D0
:1008C000FB81309719F0D183C08308C0D093DA0838
:1008D000C093D90803C019821882F1CFDF91CF915C
:1008E00008950FB6F8940F926091DB087091DC08C0
:1008F0008091DD089091DE080F900FBE0895CF9390
:10090000DF93EC01EA81FB8188819981309719F0AE
:100910009183808304C09093DA088093D908E8819A
:10092000F9813097A1F08A819B81938382838085AE
:100930009185A285B385288539854A855B85820F97
:10094000931FA41FB51F80879187A287B387CE010D
:100950000E949B08DF91CF91089588E194E00E9466
:10096000C10B87B7826087BF0895EF92FF920F9304
:100970001F93CF93DF930FB6F8940F922091DB086B
:100980003091DC084091DD085091DE080F900FBED9
:100990008091730790917407A0917507B0917607C5
:1009A00079018A01E81AF90A0A0B1B0B20937307D5
:1009B0003093740740937507509376074FC088852E
:1009C0009985AA85BB85E816F9060A071B07A0F4D6
:1009D0008E199F09A00BB10B88879987AA87BB87BF
:1009E0000097A105B10521F0EE24FF24870136C050
:1009F000EE24FF24870108C0E81AF90A0A0B1B0B32
:100A0000188619861A861B86EC85FD85309721F09D
:100A10006E857F85CE0109958C819D81AE81BF81D8
:100A200088879987AA87BB870097A105B10521F41C
:100A3000CE010E947F0412C0E091D908F091DA083B
:100A40000190F081E02DF093DA08E093D908309717
:100A500011F013821282CE010E942C04C091D90899
:100A6000D091DA08209731F0E114F1040105110565
:100A700009F0A5CFDF91CF911F910F91FF90EF90DB
:100A800008952F923F924F925F926F927F928F9232
:100A90009F92AF92BF92CF92DF92EF92FF920F930D
:100AA0001F93CF93DF93CDB7DEB724970FB6F8949B
:100AB000DEBF0FBECDBF0FB6F8940F92A090DB083B
:100AC000B090DC08C090DD08D090DE080F900FBE1B
:100AD0000E94BC0B9B01AC01C601B5010E941B85A5
:100AE00039014A010E94BC0B1B012C010E94BC0B66
:100AF00069837A838B839C83C401B30128EE33E03E
:100B000040E050E00E94DD847B018C01C401B30110
:100B1000A20191010E94DD84A61AB70AC80AD90A67
:100B2000C601B50128EE33E040E050E00E94DD84CC
:100B300029813A814B815C810E941B85E20EF31E64
:100B4000041F151FC801B70124960FB6F894DEBF25
:100B50000FBECDBFDF91CF911F910F91FF90EF900E
:100B6000DF90CF90BF90AF909F908F907F906F90CD
:100B70005F904F903F902F900895EF92FF920F93C8
:100B80001F930FB6F8940F92E090DB08F090DC080A
:100B90000091DD081091DE080F900FBE0E94BC0B83
:100BA0009B01AC01C801B7010E941B85CA01B901B4
:100BB0001F910F91FF90EF900895AF92BF92CF9247
:100BC000DF92EF92FF920F93CF93DF936B017C0143
:100BD000EA01590180E190E00E942808FC01892B7C
:100BE00081F10FB6F8940F928091DB089091DC08A8
:100BF000A091DD08B091DE080F900FBE8C0D9D1DF9
:100C0000AE1DBF1D20917307309174074091750789
:100C100050917607821B930BA40BB50B80879187AD
:100C2000A287B38700FF05C014821582168217823F
:100C300004C0C482D582E682F782D587C487B7868E
:100C4000A686CF01DF91CF910F91FF90EF90DF90BB
:100C5000CF90BF90AF9008950F93CF93DF930E94F2
:100C6000DD05EC01009711F00E942C04CE01DF910C
:100C7000CF910F910895CF92DF92EF92FF920F9351
:100C80006A0179010E94110C9701A6010E942C06AD
:100C90000F91FF90EF90DF90CF900895AF92BF92A9
:100CA000CF92DF92EF92FF920F93CF93DF935B018E
:100CB0006C016115710581059105D1F1C1EED8E096
:100CC000BE018091E3089091E4080E94F206E09151
:100CD000E308F091E40883E08787E090E308F09070
:100CE000E40801E097014DE257E0C601B5010E941A
:100CF0003B06F701968B858B892B19F00E94CB0759
:100D000019C0E091E308F091E408D08FC78B80917F
:100D1000E1089091E2089383828381E08787809144
:100D2000E3089091E4089093E2088093E10802C000
:100D30000E941008DF91CF910F91FF90EF90DF900C
:100D4000CF90BF90AF900895CF93DF93DC019B01CC
:100D5000EC01788F6F8B1D821C820FB6F8940F9276
:100D6000EB01E881F9818FEFEF3FF80749F4ED01DE
:100D70008C819D8101969D838C83E0E0F0E015C01D
:100D8000309799F00F900FBEED019A8908C09F012E
:100D90002E5F3F4F0280F381E02D309719F082895A
:100DA0009817A8F70FB6F8940F92ED01FB83EA832A
:100DB000F901B183A083EA81FB81309771F08481CE
:100DC0009581892B51F08C819D8124813581820F01
:100DD000931F9D838C83158214820F900FBEDF9129
:100DE000CF910895CF93DF939C01DB010FB6F89468
:100DF0000F92ED91FC9111970F900FBE8FEFEF3F87
:100E0000F80731F527C082819381E217F307E9F4EF
:100E10000FB6F8940F9211969C938E9384819581CE
:100E2000892B59F0A281B381109729F08481958193
:100E3000ED019D838C83158214820F900FBEF90102
:100E400013821282108E178A05C0DF011296FC01F0
:100E50003097C9F6DF91CF910895FB01168A158A64
:100E600082E0878761EE78E0CF010E94A4060895B2
:100E70000F931F93CF93DF938C01C091DF08D09124
:100E8000E0080CC0B801CE0106960E94AF84892B01
:100E900011F4CE0107C00990D881C02D209791F799
:100EA00080E090E0DF91CF911F910F910895E09144
:100EB000E508F091E608309741F0838994890E9413
:100EC0009B081092E6081092E5080895CF93DF93EF
:100ED000C091DF08D091E0080E9457072091E308F5
:100EE0003091E408EFEDF8E00AC088819981C217DB
:100EF000D30719F49183808304C0FE01EC0120978D
:100F0000A1F78091E3089091E4089093E60880931C
:100F1000E508DF91CF9108950F931F93182FE0916B
:100F2000E308F091E408028961EE78E0CF010E94C5
:100F3000F206E091E308F091E408128B1F3F49F0BC
:100F400061EE78E08091E3089091E4080E94A406A5
:100F500002C00E946607E091E308F091E4088091E6
:100F6000E1089091E208E817F90719F481E0878712
:100F700009C082E087870FB6F8940F920E94C80AD2
:100F80000F900FBE802F99271F910F9108958FEF1B
:100F90000E948C070895CF93DF93C091DF08D09112
:100FA000E00820C00FB6F8940F928C819D810F90BD
:100FB0000FBE892BA1F0EF89F88D0FB6F8940F9230
:100FC0008C819D8101979D838C830F900FBE8081C2
:100FD00091818F5F9F4F19F0CF010E945E090990A8
:100FE000D881C02D2097F1F60E94B504E091E30866
:100FF000F091E4088091E1089091E208E817F90780
:1010000061F08785813011F482E087870FB6F8940C
:101010000F920E94C80A0F900FBEDF91CF910895E2
:10102000E091E308F091E40882819381892B69F0D3
:1010300061EE78E0CF010E94F20661EE78E08091E7
:10104000E3089091E4080E94A4060E94CB0708954B
:101050000F931F93CF93DF93009177071091780739
:101060008017910730F080E090E060C0EF01DB0175
:101070002FC0AC014A5F5F4F4430510510F444E08B
:1010800050E0E091E708F091E80867EE78E0C0E012
:10109000D0E0A0E0B0E017C02081318124173507EF
:1010A00060F02417350711F3209729F08881998182
:1010B0002817390710F4EF01DB01BF016E5F7F4F86
:1010C0000280F381E02D309739F7CE01209771F13E
:1010D00028813981CA010A966A817B818217930728
:1010E00070F4FE01E40FF51F241B350B31832083C0
:1010F0007383628359834883ED93FC9302C06D939D
:101100007C93E881F9810E1B1F0B109378070093E5
:101110007707EC0FFD1F34978FEE9EEBADEABEED27
:1011200080839183A283B383CE010296DF91CF9116
:101130001F910F910895CF93DF93DC0112976D916A
:101140007C911197E091E708F091E808C7EED8E0AC
:101150003AC040815181CF01840F951F8A179B07A8
:10116000C1F49A01260F371F318320838281938136
:10117000DF01A20FB31FA817B90791F58D919C91BC
:101180001197280F391F31832083ED018A819B81BC
:1011900025C0AE17BF0778F4B983A8832D913C9181
:1011A0001197CD01820F931F8E179F0779F0ED01E4
:1011B000FB83EA8315C0A817B90728F1EF0122962F
:1011C0000280F381E02D309721F617C0240F351FE0
:1011D00011963C932E9382819381FD0193838283A8
:1011E0008091770790917807860F971F90937807E3
:1011F0008093770780E090E008C0FD01138212829F
:10120000B983A883EDCF8FEF9FEFDF91CF91089542
:10121000FC0161937193CF010E949B080895809116
:1012200077079091780708950F931F93CF93DF93DB
:101230008C010E942808EC01009729F0A80160E0C9
:1012400070E00E94A584CE01DF91CF911F910F9194
:10125000089583E18093E9088FE48093EA0883E5A9
:101260008093EB0843E150E069EE78E080E090E0A5
:101270000E94BA0A892B19F08FEF9FEF089580E042
:1012800090E0089543E150E069EE78E080E090E07E
:101290000E94BD0A892B79F48091E908833159F4C1
:1012A0008091EA088F3439F48091EB08833519F482
:1012B00080E090E008958FEF9FEF0895CF93DF9344
:1012C000DC010FB6F8940F92CD91DC9111970F903D
:1012D0000FBE8FEFCF3FD80709F43AC0209771F1C6
:1012E0000FB6F8940F92EA81FB811196FC93EE936E
:1012F0008C819D81892B71F0309729F08C819D81A3
:101300009583848305C08FEF9FEF11969C938E93F6
:101310001D821C820F900FBE8D899E89009721F03F
:101320000E947F041E8A1D8A82E08F8761EE78E02A
:10133000CE010E94A40681E090E00CC00FB6F894A4
:101340000F928FEF9FEF11969C938E930F900FBE8D
:1013500080E090E0DF91CF9108950F931F93CF939A
:10136000DF93EC010FB6F8940F92888199810F906A
:101370000FBE2FEF8F3F920741F40FB6F8940F92F4
:10138000198218820F900FBE02C0892B19F400E059
:1013900010E012C000E010E0CE010E945E09080FCC
:1013A000191F0FB6F8940F92888199810F900FBE84
:1013B00001978E5F9F4F80F3C801DF91CF911F91FE
:1013C0000F9108950F931F930E94AD098C010E9405
:1013D0001008C8011F910F9108950F931F930E9449
:1013E0005E098C010E941008C8011F910F91089599
:1013F000CF93DF93AC01DB010FB6F8940F92CD9140
:10140000DC9111970F900FBE8FEFCF3FD80799F562
:1014100034C08D899E892A813B818417950741F5C7
:101420000FB6F8940F9211963C932E938C819D8168
:10143000892B81F0EA81FB81309729F08C819D8195
:101440009583848305C08FEF9FEF11969C938E93B5
:101450001D821C820F900FBE82E08F8761EE78E0C4
:10146000CE010E94A4068FEF9FEF9E8B8D8B05C04F
:10147000DE011296E901209761F6DF91CF91089580
:10148000AF92BF92CF92DF92EF92FF920F93CF93E2
:10149000DF93EC015A016B010FB6F8940F9288812B
:1014A00099810F900FBE8F5F9F4F51F40FB6F89444
:1014B0000F92198218820F900FBE0E94100838C038
:1014C00061EE78E08091E3089091E4080E94F206D2
:1014D000BE018091E3089091E4080E94A406E09187
:1014E000E308F091E40883E08787E090E308F09058
:1014F000E408A114B104C104D10461F001E09E012B
:1015000048EF59E0C601B5010E943B06F701968BF2
:10151000858B03C0F701168A158A0E94CB07E091DC
:10152000E308F091E408858996898F5F9F4F19F051
:1015300080E090E004C0168A158A8FEF9FEFDF915C
:10154000CF910F91FF90EF90DF90CF90BF90AF9031
:101550000895FC010FB6F8940F92808191818F5FFE
:101560009F4F11F4118210820F900FBECF010E9485
:10157000400A08950E94B31508950E94D315089556
:101580009F918F910F900BBE0F900FBE1F901895DB
:101590002F923F924F925F926F927F928F929F9283
:1015A000AF92BF92CF92DF92EF92FF920F931F9371
:1015B000CF93DF938DB79EB7E091E308F091E408F5
:1015C000918B808BE091E108F091E208F093E408C0
:1015D000E093E30881E08787E091E308F091E40875
:1015E000808991898DBF9EBFDF91CF911F910F910F
:1015F000FF90EF90DF90CF90BF90AF909F908F9033
:101600007F906F905F904F903F902F900895CF9272
:10161000DF92EF92FF920F931F93CF93DF938C0192
:101620007B016A01E901C90149960E942808FC0171
:10163000009719F480E090E075C0C80FD91F9E0193
:1016400027503040AE014B515040CE01069668E025
:10165000D8010D908D01DC010D92CD016150C1F7D3
:101660001E8641505040598B488B4F5F5F4FFC8B1B
:10167000EB8B8FEE9EEBADEABEED80839183A28370
:10168000B38384839583A683B78380879187A2875A
:10169000B38784879587A687B78780E48A8B8F2D49
:1016A0009927F9018583E68280E883831282148278
:1016B000C1828D2D9927808320EC3AE0832F9927D2
:1016C000FA01828B238B8091DF089091E008998347
:1016D0008883D093E008C093DF0812E01F871E8A3A
:1016E0001D8A188E1F8A61EE78E0CE010E94A40642
:1016F000E091E308F091E408309721F40FB6F894F4
:101700000F9260CF8091E1089091E208E817F90705
:1017100041F017870FB6F8940F920E94C80A0F90F5
:101720000FBECE01DF91CF911F910F91FF90EF90EF
:10173000DF90CF9008951F93182F609179077091D3
:101740007A0780917B0790917C0720EA3FE040E098
:1017500050E00E941B85822F932F0197F1F71A9575
:10176000D1F71F9108956091790770917A07809160
:101770007B0790917C07089560E074E080E090E042
:101780000895BC0187B78D7F87BF80B7886080BF11
:1017900012BE82E083BF80B7992787709070892B33
:1017A000D1F781E086BF0FB6F8940F9281E090E008
:1017B000A0E0B0E0B6B7B170E9F3B6BF0894811D00
:1017C000911DA11DB6B7B170C9F3BB270F900FBE15
:1017D00027E0880F991FAA1FBB1F2A95D1F7809376
:1017E000790790937A07A0937B07B0937C0787B71C
:1017F0008D7F87BF80B7886080BF12BE89E083BFBE
:101800008FE181BF80B7992787709070892BD1F7BE
:1018100082E086BF40E050E08BE593E00E94347B9D
:10182000089528EE33E040E050E00E94DD843AE085
:1018300096958795779567953A95D1F708959C0188
:10184000FB0187B7482F55274270507087B78D7FAF
:1018500087BF20313105D9F0213131053CF4211504
:10186000310581F02130310551F40EC022313105AE
:1018700071F122313105E4F020323105E1F02FEF32
:101880003FEF1FC040E050E082E086BF18C006B6C0
:1018900001FE05C081E090E09183808302C0118247
:1018A0001082452BA1F08081918180689183808393
:1018B00020E030E008C08EE090E09183808320E05B
:1018C00030E0452B31F087B7826087BF02C020E04F
:1018D00030E0C90108951F920F920FB60F921124A4
:1018E0002F933F934F935F936F937F938F939F9328
:1018F000AF93BF93EF93FF938BE593E00E94267B1A
:10190000FF91EF91BF91AF919F918F917F916F91D7
:101910005F914F913F912F910F900FBE0F901F90AD
:101920001895559A89B78F7E89BF0895CF93DF9315
:10193000DC01EC01EA81FB8120917E07422F5527D3
:10194000CA0180739070892B89F044FF04C083E141
:101950008CB9206403C081E18CB92F7B20937E0772
:1019600080917E078F7C80937E0755C027FF02C041
:10197000559851C0ED018A859B85892BB1F18091E5
:101980008107882339F00C9B05C0559889B7806181
:1019900089BF41C0ED018A859B8501979B878A8716
:1019A00080917F07882311F0509A01C0509881914F
:1019B0008CB99F01FD01868197812817390711F4A1
:1019C00024813581ED013B832A832A853B858C85E3
:1019D0009D8528173907F9F4E889F989309769F066
:1019E0008FEFEF3FF807B9F011C05598ED011B8656
:1019F0001A86E889F989309729F48FEF9FEF998B40
:101A0000888B09C08FEFEF3FF80729F0848195811B
:101A1000019695838483DF91CF910895CF93DF93CF
:101A2000DC013BB180917D07382B30937D076CB191
:101A300020917E07222361F0633119F455982068C4
:101A400004C0613129F4559A2F7720937E075DC039
:101A5000ED014A855B85888599854817590720F0EF
:101A6000386030937D0751C04F5F5F4F4130510563
:101A7000A1F4ED01E889F989309729F48FEF9FEF00
:101A8000998B888B2AC08FEFEF3FF80731F1848163
:101A9000958101969583848320C0222399F0ED01DE
:101AA0008E859F8548175907C0F026FD16C05D9B9F
:101AB00005C083E18CB920642F7D01C02062209392
:101AC0007E070BC080918007882339F0FD01868551
:101AD00097854817590708F01A9AED91FC911197CC
:101AE00061931196FC93EE932D913C911197ED012A
:101AF0008E819F812817390729F48C819D81119649
:101B00009C938E93FD0153874287DF91CF91089577
:101B1000529B03C089E090E008958091950082FF78
:101B20000AC08091950081FF03C088E090E008958D
:101B300087E090E008958091950081FF03C086E0E2
:101B400090E0089585E090E008958091950085FDEE
:101B500003C080E090E008958091950084FF03C069
:101B600081E090E0089582E090E0089580919500F2
:101B700083FF03C082E090E0089581E090E0089543
:101B8000EF92FF920F931F9380917D07682F772725
:101B9000CB0174E0969587957A95E1F79C014427EF
:101BA0005527217030704070507063FD226062FDD7
:101BB000246080917E07882321F086FD426087FDA6
:101BC00048601A9B14C0E12C62E0F62E012D112D05
:101BD000E22AF32A042B152B80918007882381F0B9
:101BE000E12C92E0F92E92E0092F112D05C0E12C95
:101BF00081E0F82E012D112DE22AF32A042B152B5A
:101C00000C9B0CC0A8019701386080918107882344
:101C100041F0A80197013860426003C0A801970114
:101C2000346041FF416043FF446080917F07882317
:101C300021F0CA01B901806403C0CA01B9018068FA
:101C4000589B02C0806101C080621F910F91FF907C
:101C5000EF900895EF92FF920F931F937B018C01F9
:101C600080917E078823D9F00FB6F8940F9200FF79
:101C700002C08F7B03C001FF03C0806480937E0796
:101C800002FF04C080917E078F7705C003FF05C067
:101C900080917E07806880937E070F900FBE8091B1
:101CA0008007882321F001FD1A9A00FD1A98F1FCA3
:101CB0001A9AF0FC1A9806FF03C081E080937F0710
:101CC00007FF02C010927F0704FD589A05FD58983F
:101CD000E0FE05C080917D078F7E80937D07E1FE49
:101CE00005C080917D07877F80937D07E2FE05C058
:101CF00080917D078B7F80937D070E94C00D687F58
:101D00006E157F058007910719F08FEF9FEF02C0D6
:101D100080E090E01F910F91FF90EF9008958091E7
:101D2000950086FF0BC0129B02C093E001C091E0BA
:101D30008091950080FF07C0946005C0599B02C048
:101D400090E201C090E0892F9927089580917E0745
:101D5000882329F020E230E040E050E004C020E099
:101D600030E040E050E080918007882311F021604E
:101D700001C02E7F80918107882321F0CA01B9011B
:101D800062600895CA01B9016D7F0895559A08955A
:101D900090917E079923A9F096FF13C00FB6F8948F
:101DA0000F925D9B04C081E18CB99F7E01C0906160
:101DB00090937E0780917E078F7980937E070F90A6
:101DC0000FBE8091800781111A9808950FB6F8947C
:101DD0000F925798569855980F900FBE8AE00E9420
:101DE0009B0B5498539808951F93182F0E94E60E4A
:101DF0005298809195008D7F8093950080919500F9
:101E00008B7F809395001730A1F0183018F41630AE
:101E1000A9F405C0183041F0193081F404C0809154
:101E20009500826009C0529A8091950082608093EB
:101E30009500809195008460809395000FB6F8948A
:101E40000F9288EB8AB90F900FBE0E94880D811700
:101E500019F08FEF9FEF02C080E090E01F9108958E
:101E60008F929F92AF92BF92CF92DF92EF92FF92AA
:101E70000F931F9389B0909090008091950086FFFA
:101E800006C0B2E0AB2EB12CC12CD12C0DC0599B99
:101E900006C0A8E0AA2EB12CC12CD12C05C0F0E1BF
:101EA000AF2EB12CC12CD12C0E94B30B7B018C0125
:101EB000282D3327892D9927982F8827282B392BD0
:101EC000442755272F5F3F4F4F4F5F4FC601B50146
:101ED0000E94DD849B01AC01C801B7010E941B85F3
:101EE000CA01B9011F910F91FF90EF90DF90CF9041
:101EF000BF90AF909F908F90089540E050E060E0D9
:101F000070E08FE594E00E94347B40E050E060E0B8
:101F100070E085E694E00E94347B809181078823FD
:101F200059F010928107149840E050E060E070E0B2
:101F30008BE694E00E94347B80918007882319F01F
:101F400010928007129880E090E0089546EA53E0EE
:101F50006EE07DE08FE594E00E94347B892B19F0E0
:101F60008FEF9FEF089544E953E066E97CE085E652
:101F700094E00E94347B892B19F480E090E008956E
:101F800040E050E060E070E08FE594E00E94347B38
:101F90008FEF9FEF0895EF92FF920F931F937B01B6
:101FA0008C0165FF0BC080917E07882371F40FB60A
:101FB000F8940F9281E480937E0705C00FB6F894E1
:101FC0000F9210927E070F900FBEE0FE06C01A9A85
:101FD000129A81E08093800707C080918007882350
:101FE00019F0109280071298E1FE10C040E050E016
:101FF00061E97CE08BE694E00E94347B892BF9F464
:102000001C9A149881E0809381070FC0809181070A
:10201000882359F01092810740E050E060E070E0C2
:102020008BE694E00E94347B14980E94A60E6E15F5
:102030007F058007910719F480E090E002C08FEFE0
:102040009FEF1F910F91FF90EF900895EF92FF92F5
:102050000F931F937B018C010E94E60E80919500E7
:1020600086FD11C0599B08C092E0EE0CFF1C001FBA
:10207000111F9A95D1F707C083E0EE0CFF1C001FDB
:10208000111F8A95D1F70E94B30BA80197010E94F6
:102090001B852F5F3F4F4F4F5F4F569547953795A5
:1020A00027952150304029B9232F332720939000C2
:1020B0000FB6F8940F9288EB8AB90F900FBE80E0AC
:1020C00090E01F910F91FF90EF9008951F93182FAC
:1020D0000E94E60E812F992780FF13C081FF02C066
:1020E000129A01C0129882FF04C08091950081600D
:1020F00003C0809195008E7F8093950059985E9AD9
:102100000FC085FF02C0599A01C05998809195006F
:102110008E7F80939500809195008F7B80939500B2
:102120000FB6F8940F9288EB8AB90F900FBE0E94F9
:102130008F0E811719F08FEF9FEF02C080E090E0C3
:102140001F9108951F93182F0E94E60E113071F011
:10215000113018F01230C1F40DC0809195008F7EBF
:1021600080939500809195008F7D0CC080919500A3
:10217000806103C0809195008F7E8093950080914F
:1021800095008062809395000FB6F8940F9288EBCB
:102190008AB90F900FBE0E94A50D811719F08FEF1D
:1021A0009FEF02C080E090E01F9108951F93182FC9
:1021B0000E94E60E113021F480919500877F05C0C2
:1021C000123029F4809195008860809395000FB6B5
:1021D000F8940F9288EB8AB90F900FBE809195000A
:1021E00083FF03C082E090E002C081E090E0181716
:1021F00019F08FEF9FEF02C080E090E01F910895EB
:10220000EAE9F0E080818062808389B78F7D89BFB1
:1022100008951F920F920FB60F9211242F933F93A0
:102220008F939F93EF93FF93E0911204F091130427
:1022300080911A0490911B04892B09F44EC080915F
:102240008607882359F00D9B09C080919A008F7DE5
:1022500080939A0089B7806289BF5EC080911A041A
:1022600090911B04019790931B0480931A04809112
:102270008407882321F080919A00816003C08091B7
:102280009A008E7F80939A00819180939C009F0199
:102290008091160490911704E817F90721F4209112
:1022A00014043091150430931304209312042091E8
:1022B0001A0430911B0480911C0490911D0428176E
:1022C000390751F5E0912004F09121043097A1F0F5
:1022D0008FEFEF3FF80701F11AC080919A008F7DD0
:1022E00080939A0010921B0410921A04E09120042B
:1022F000F0912104309739F48FEF9FEF90932104F0
:102300008093200409C08FEFEF3FF80729F0848104
:102310009581019695838483FF91EF919F918F9191
:102320003F912F910F900FBE0F901F9018951F9205
:102330000F920FB60F9211242F933F934F935F93F9
:102340006F937F938F939F93AF93BF93EF93FF937D
:1023500060918207A0918507B0E080919B00682B77
:1023600070919C0020912C0430912D0480912A04BE
:1023700090912B042817390708F047C0A9014F5F37
:102380005F4F4130510511F4B1E00AC0AA2341F07A
:1023900080913004909131044817590708F0949ABD
:1023A000E0912204F09123047193F0932304E093CD
:1023B00022042091220430912304809128049091DA
:1023C00029042817390741F48091260490912704A5
:1023D000909323048093220450932D0440932C0463
:1023E00080919B0087FDB9CF60938207BB23D1F01A
:1023F000E0913204F0913304309759F48FEF9FEF5E
:1024000090933304809332040DC068606093820718
:1024100009C08FEFEF3FF80729F08481958101967D
:1024200095838483FF91EF91BF91AF919F918F919D
:102430007F916F915F914F913F912F910F900FBEC0
:102440000F901F90189580919A0082FF03C089E039
:1024500090E0089580919D0082FF0AC080919D00C8
:1024600081FF03C088E090E0089587E090E0089540
:1024700080919D0081FF03C086E090E0089585E093
:1024800090E0089580919D0085FD03C080E090E07C
:10249000089580919D0084FF03C081E090E008953D
:1024A00082E090E0089580919D0083FF03C082E068
:1024B00090E0089581E090E00895EF92FF920F93ED
:1024C0001F9380918207682F7727CB0174E0969540
:1024D00087957A95E1F79C01442755272170307044
:1024E0004070507063FD226062FD2460809183071C
:1024F000882321F086FD426087FD4860949B14C0CC
:10250000E12C62E0F62E012D112DE22AF32A042B94
:10251000152B80918507882381F0E12C92E0F92E1C
:1025200092E0092F112D05C0E12C81E0F82E012D3C
:10253000112DE22AF32A042B152B0D9B0CC0A801A8
:102540009701386080918607882341F0A8019701A0
:102550003860426003C0A8019701346041FF4160C8
:1025600043FF446080918407882311F0406401C0D8
:10257000406880919B0080FF04C0CA01B90180615E
:1025800003C0CA01B90180621F910F91FF90EF90C3
:102590000895EF92FF920F931F937B018C0180911E
:1025A00083078823D9F00FB6F8940F9200FF02C07A
:1025B0008F7B03C001FF03C080648093830702FF09
:1025C00004C0809183078F7705C003FF05C0809109
:1025D00083078068809383070F900FBE80918507E3
:1025E000882321F001FD949A00FD9498F1FC949ABF
:1025F000F0FC949806FF03C081E08093840707FFF6
:1026000002C01092840704FF05C080919B00816086
:1026100080939B0005FF05C080919B008E7F809377
:102620009B00E0FE05C0809182078F7E8093820729
:10263000E1FE05C080918207877F80938207E2FEDA
:1026400005C0809182078B7F809382070E945D1274
:10265000687F6E157F058007910719F08FEF9FEF58
:1026600002C080E090E01F910F91FF90EF900895DD
:1026700080919D0086FF0BC0129B02C093E001C0B9
:1026800091E080919D0080FF09C0946007C0809117
:102690009B0081FF02C090E201C090E0892F992742
:1026A000089580918307882329F020E230E040E0FC
:1026B00050E004C020E030E040E050E08091850729
:1026C000882311F0216001C02E7F80918607882326
:1026D00021F0CA01B90162600895CA01B9016D7F94
:1026E0000895EAE9F0E08081806280830895909106
:1026F00083079923C1F096FF16C00FB6F8940F9286
:1027000080919B0085FF05C081E180939C009F7EA6
:1027100001C0906190938307809183078F798093A4
:1027200083070F900FBE80918507811194980895BB
:1027300080E090E008950F931F930FB6F8940F92E6
:102740000AE910E0F80180818F77808380818F7B98
:10275000808380818F7D80830F900FBE8AE00E94EE
:102760009B0BF80180818F7E80838081877F8083AF
:102770001F910F9108951F93182F0E949B13809112
:102780009A008B7F80939A0080919D008D7F80932B
:102790009D0080919D008B7F80939D001730C1F03C
:1027A000183018F41630C9F405C0183061F019302B
:1027B000A1F404C080919D0082600DC080919A00B8
:1027C000846080939A0080919D00826080939D0038
:1027D00080919D00846080939D000FB6F8940F92C5
:1027E00088EB80939A000F900FBE0E9423128117EE
:1027F00019F08FEF9FEF02C080E090E01F910895E5
:102800008F929F92AF92BF92CF92DF92EF92FF9200
:102810000F931F93809099009090980080919D0055
:1028200086FF06C0B2E0AB2EB12CC12CD12C0FC05C
:1028300080919B0081FF06C0A8E0AA2EB12CC12C7C
:10284000D12C05C0F0E1AF2EB12CC12CD12C0E94AF
:10285000B30B7B018C01282D3327892D9927982FC5
:102860008827282B392B442755272F5F3F4F4F4F61
:102870005F4FC601B5010E94DD849B01AC01C80118
:10288000B7010E941B85CA01B9011F910F91FF90EA
:10289000EF90DF90CF90BF90AF909F908F90089572
:1028A00080918607882359F010928607159840E09A
:1028B00050E060E070E089E594E00E94347B809114
:1028C0008507882319F0109285078C9880E090E0A6
:1028D0000895EF92FF920F931F937B018C0165FF88
:1028E0000BC080918307882371F40FB6F8940F9280
:1028F00081E48093830705C00FB6F8940F9210927D
:1029000083070F900FBEE0FE06C0949A8C9A81E078
:102910008093850707C080918507882319F010925E
:1029200085078C98E1FE10C040E050E060E071E166
:1029300089E594E00E94347B892BF9F41D9A15985F
:1029400081E0809386070FC080918607882359F025
:102950001092860740E050E060E070E089E594E086
:102960000E94347B15980E9451136E157F058007D5
:10297000910719F480E090E002C08FEF9FEF1F9164
:102980000F91FF90EF900895EF92FF920F931F9396
:102990007B018C010E949B1380919D0086FD13C0DA
:1029A00080919B0081FF08C092E0EE0CFF1C001F8D
:1029B000111F9A95D1F707C083E0EE0CFF1C001F92
:1029C000111F8A95D1F70E94B30BA80197010E94AD
:1029D0001B852F5F3F4F4F4F5F4F5695479537955C
:1029E00027952150304020939900232F332720939F
:1029F00098000FB6F8940F9288EB80939A000F908E
:102A00000FBE80E090E01F910F91FF90EF9008952E
:102A10001F93182F0E949B13812F992780FF1BC0A3
:102A200081FF02C0129A01C0129882FF04C08091F7
:102A30009D00816003C080919D008E7F80939D00EA
:102A400080919B008D7F80939B0080919B00806490
:102A500080939B0015C085FF04C080919B0082601D
:102A600003C080919B008D7F80939B0080919D008F
:102A70008E7F80939D0080919D008F7B80939D0031
:102A80000FB6F8940F9288EB80939A000F900FBEC8
:102A90000E943813811719F08FEF9FEF02C080E07A
:102AA00090E01F9108951F93182F0E949B131130DF
:102AB00071F0113018F01230C1F40DC080919D00FA
:102AC0008F7E80939D0080919D008F7D0CC08091B2
:102AD0009D00806103C080919D008F7E80939D004A
:102AE00080919D00806280939D000FB6F8940F92B4
:102AF00088EB80939A000F900FBE0E9442128117BC
:102B000019F08FEF9FEF02C080E090E01F910895D1
:102B10001F93182F0E949B13113021F480919D0068
:102B2000877F05C0123029F480919D0088608093D2
:102B30009D000FB6F8940F9288EB80939A000F9047
:102B40000FBE80919D0083FF03C082E090E002C031
:102B500081E090E0181719F08FEF9FEF02C080E03E
:102B600090E01F910895CF93DF93EA019C0140E02C
:102B700050E0FB0110C0D9010E947085802D90812A
:102B8000981721F0D901092E0E9478854F5F5F4F79
:102B900031962F5F3F4F4C175D0769F780E090E05B
:102BA000DF91CF910895CF93DF93EA01DC01FB0120
:102BB000219724F00E9470850192FACF80E090E086
:102BC000DF91CF9108959C01FB0189B7482F5527CC
:102BD0004072507089B78F7D89BF21313105D1F1A5
:102BE000223131054CF421303105F9F02031310525
:102BF000F9F0232BA1F066C02831310571F129319C
:102C000031052CF42231310509F05CC063C0293153
:102C10003105B9F12032310509F054C023C08AB71B
:102C20008B7F8ABF8AB7877F8ABF80E288BF1EC03A
:102C300008B605FE05C081E090E09183808302C064
:102C400011821082452B09F445C0808191818068F2
:102C50009183808320E030E039C08AB7982F987044
:102C600083FF07C085E090E09183808320E030E01F
:102C70002BC0943019F487E090E0F6CF81E090E02B
:102C8000F3CF608171816130710519F48AB78B7F50
:102C900005C06730710531F48AB784608ABF8AB78E
:102CA000877F0EC06530710519F48AB78B7F05C028
:102CB0006630710539F48AB784608ABF8AB7886044
:102CC0008ABFD4CF2FEF3FEF452B31F089B7806219
:102CD00089BF02C020E030E0C90108951F920F9221
:102CE0000FB60F9211242F933F934F935F936F93DF
:102CF0007F938F939F93AF93BF93EF93FF9389E558
:102D000094E00E94267BFF91EF91BF91AF919F913C
:102D10008F917F916F915F914F913F912F910F9084
:102D20000FBE0F901F9018959C01FB018AB1482F90
:102D3000552740785070579820313105D9F021310E
:102D400031053CF42115310581F02130310551F474
:102D50000EC02231310559F122313105DCF020322B
:102D60003105D9F08FEF9FEF1EC040E050E08CB1ED
:102D70008CB117C05F9B05C081E090E09183808398
:102D800002C011821082452B91F080819181806870
:102D90009183808380E090E008C080E190E091839F
:102DA000808380E090E0452B21F0579A089580E0E1
:102DB00090E008951F920F920FB60F9211242F9357
:102DC0003F934F935F936F937F938F939F93AF93B3
:102DD000BF93EF93FF938FE594E00E94267BFF91D2
:102DE000EF91BF91AF919F918F917F916F915F9183
:102DF0004F913F912F910F900FBE0F901F901895FC
:102E00009C01FB018AB1482F55274072507055989C
:102E10002131310519F1223131053CF421153105FB
:102E200051F12031310539F409C02231310519F150
:102E300020323105B1F08FEF9FEF19C05D9B05C0C7
:102E400081E090E09183808302C011821082452B43
:102E500091F08081918180689183808380E090E00F
:102E600008C080E190E09183808380E090E0452B72
:102E700021F0559A089580E090E008951F920F92F6
:102E80000FB60F9211242F933F934F935F936F933D
:102E90007F938F939F93AF93BF93EF93FF9385E6B9
:102EA00094E00E94267BFF91EF91BF91AF919F919B
:102EB0008F917F916F915F914F913F912F910F90E3
:102EC0000FBE0F901F9018959C01FB0189B7482FEA
:102ED00055274071507089B78F7E89BF21313105E8
:102EE000D1F1223131054CF421303105F9F0203196
:102EF0003105F9F0232BA1F069C02831310571F1BA
:102F0000293131052CF42231310509F05FC066C04A
:102F100029313105B9F12032310509F057C053C0CC
:102F20008AB78E7F8ABF8AB78D7F8ABF80E188BFCC
:102F30001EC008B604FE05C081E090E09183808346
:102F400002C011821082452B09F448C08081918112
:102F500080689183808320E030E03CC08AB7982F5E
:102F6000927081FF07C085E090E09183808320E02C
:102F700030E02EC0913019F487E090E0F6CF81E088
:102F800090E0F3CF608171816130710519F48AB7E7
:102F90008E7F05C06730710531F48AB781608ABFC2
:102FA0008AB78D7F0EC06530710519F48AB78E7FA0
:102FB00005C06630710551F48AB781608ABF8AB74F
:102FC00082608ABFD4CF84E090E0CFCF2FEF3FEF75
:102FD000452B31F089B7806189BF02C020E030E025
:102FE000C90108951F920F920FB60F9211242F93CB
:102FF0003F934F935F936F937F938F939F93AF9381
:10300000BF93EF93FF938BE694E00E94267BFF91A2
:10301000EF91BF91AF919F918F917F916F915F9150
:103020004F913F912F910F900FBE0F901F901895C9
:10303000FC01808191810895CF92DF92EF92FF92FF
:103040000F931F93CF93DF936C01CB010E94771FE7
:103050007C018F5F9F4F71F440C00F5F1F4F32960E
:103060000830110559F487E190E09093490B809363
:10307000480B33C003E010E0E7E7F4E08081918182
:10308000892B59F787E090E00E94F819EC01000FB6
:10309000111F0F581B4FD801CD93DC932097E9F0F7
:1030A000B701C6010E948A1999838883D801ED91DE
:1030B000FC918F5F9F4F39F4CF010E94F519F80101
:1030C000118210820AC0F382E2821482D801ED914B
:1030D000FC9116821582CF0102C080E090E0DF9162
:1030E000CF911F910F91FF90EF90DF90CF900895B7
:1030F0009F92AF92BF92CF92DF92EF92FF920F9387
:103100001F93CF93DF935C01CB01EA010E94771FED
:103110006C018F5F9F4F71F448C00F5F1F4F329655
:103120000830110559F489E090E09093490B8093A1
:10313000480B3BC000E010E0E1E7F4E080819181C2
:103140008C179D0751F787E090E00E94F8197C01E9
:10315000E801CC0FDD1FCF58DB4FF982E882E11484
:10316000F10419F1B601C5010E948A19F701918392
:103170008083E881F9818F5F9F4F71F4CF010E94B6
:10318000F51982E0801728F00F5F1F4F198308831D
:103190000CC01982188209C0D382C2821482E881CD
:1031A000F98116821582CF0102C080E090E0DF91A4
:1031B000CF911F910F91FF90EF90DF90CF90BF9034
:1031C000AF909F900895CF93DF93CDB7DEB722974E
:1031D0000FB6F894DEBF0FBECDBFFE0137966191EA
:1031E0007191FA83E983AF01809173049091740423
:1031F0000E94381922960FB6F894DEBF0FBECDBFDD
:10320000DF91CF91089560917304709174040E94CE
:10321000CB1F8F5F9F4F19F48FEF9FEF0895609141
:103220007304709174048AE090E00E94A31F80E010
:1032300090E00895CF93DF93CDB7DEB722970FB616
:10324000F894DEBF0FBECDBFAE01455F5F4F5A831E
:10325000498369857A858F8198850E945A192296BB
:103260000FB6F894DEBF0FBECDBFDF91CF910895AA
:10327000FC01CB019A0160817181AC0182EE99E180
:103280000E942D1A0895CF93DF93EC0180E090E027
:10329000DB0105C02D933196F983E88301968417ED
:1032A000950729F0E881F9812081222399F7DF91A0
:1032B000CF910895CF93DF93CDB7DEB722970FB6A6
:1032C000F894DEBF0FBECDBF9A019A838983AB010C
:1032D000BE016F5F7F4F83E499E10E946F1D2296CC
:1032E0000FB6F894DEBF0FBECDBFDF91CF9108952A
:1032F000CF93DF93EC01AA81BB81109719F4EB8582
:10330000FC8504C0ED01ED89FE89CD010995DF91B1
:10331000CF910895EF92FF920F931F93CF93DF9376
:10332000CDB7DEB729970FB6F894DEBF0FBECDBF7D
:103330007B018C01FE013196AE01475F5F4F03C0F8
:1033400021930F5F1F4F302F381BD8012C91222360
:1033500029F02A3319F0E417F50791F7CE01019609
:10336000FC01E30FF11D10820E94D003DC01892BC8
:1033700049F482E090E09093490B8093480B8FEFE3
:103380009FEF13C0F80180818A3319F060E070E08C
:1033900003C0B8016F5F7F4FFD01058D168D20E0E2
:1033A00030E0A701CD01F801099529960FB6F894F0
:1033B000DEBF0FBECDBFDF91CF911F910F91FF9068
:1033C000EF900895CF93DF93DC01EC01EA81FB815C
:1033D000309719F4EF81F88503C0018CF28DE02D50
:1033E000CD010995DF91CF9108950E949B08089522
:1033F0000E9428089C01892B31F48CE090E0909386
:10340000490B8093480BC9010895CF92DF92EF9248
:10341000FF920F931F93CF93DF936C017B018A017F
:10342000E90107C040E150E0B801C701F601099584
:103430006097C131D105B4F71C161D062CF4AE01FE
:10344000B801C701F6010995DF91CF911F910F9146
:10345000FF90EF90DF90CF9008952F923F924F9280
:103460005F926F927F928F929F92AF92BF92CF9214
:10347000DF92EF92FF920F931F93CF93DF93CDB71D
:10348000DEB76B970FB6F894DEBF0FBECDBF998F36
:10349000888F7B8F6A8F1A0159011D8A1C8AB1019E
:1034A00003C00894211C311CD101FC90FF2019F0AD
:1034B000B5E2FB16B1F78101061B170B61F0A801FD
:1034C0008A8D9B8DE88DF98D09952C893D89200F7A
:1034D000311F3D8B2C8BFF2009F4E6C2F1013196A0
:1034E000198266241B8A1A8A4FEF442E542E02C07A
:1034F0005C01F101DF019D901D01B0E29B1621F4FA
:1035000089818823B1F703C02BE2921611F49982C6
:10351000F0CF3DE2931619F444E0642AEACF53E277
:10352000951619F461E0662AE4CF70E3971619F452
:1035300080E1682ADECF9CE6991619F4A8E06A2A91
:10354000D8CFBAE79B16A9F22AE2921691F4C501E8
:103550000296D501AD90BC90BB8AAA8AB7FEC8CFAF
:10356000B4E06B2AF501F095E195FF4FFB8BEA8BF8
:10357000BFCF2EE2921691F581818A3219F0442450
:1035800055241FC00894211C311CD5014D905C901E
:10359000E2E0F0E0AE0EBF1E1BC08AE090E0A201A8
:1035A000489F2001499F500C589F500C1124822F96
:1035B000992787FD9095480E591E60ED7FEF460EC6
:1035C000571E21813196822F80538A3030F31F019C
:1035D00057FE8FCF3FEF432E532E8BCF892D815334
:1035E000893010F5892D9927C0979B8B8A8B2AE00B
:1035F00030E012C04A895B89429FD001439FB00DE1
:10360000529FB00D1124892F992787FD9095A80FFF
:10361000B91FD097BB8BAA8B91813196892F80538C
:103620008A3040F31F0165CFF501792C57E6591513
:10363000E8F065E6961608F09FC170E59716D1F19F
:10364000791548F085E4981609F496C197E499161F
:1036500009F096C191C1A3E69A1621F1A91508F4C3
:1036600072C0B8E59B1609F08BC128C120E79216FD
:1036700009F424C1291548F039E6931609F463C00A
:103680004FE6941609F07CC1CDC055E7951609F4B4
:1036900059C068E7961609F411C173E7971609F047
:1036A0006FC124C082E090E0A80EB91E80818A8399
:1036B00019826CC1A2E0B0E0AA0EBB1EE080F180CE
:1036C000E114F10439F421E8C22E24E0D22E93E76C
:1036D000792E19C0C7010E94828401960E94F819B0
:1036E0008C01B7010E947B84680106C022E030E0B3
:1036F000A20EB31EC080D180C114D10421F481E890
:10370000C82E84E0D82E57FC12C0A20160E070E001
:10371000C6010E948B84009711F4820111C08C199C
:103720009D098201841595055CF48C0109C0D601C0
:103730000D900020E9F78D01015010400C191D0972
:103740001982AAC1198263FE0CC024E030E0A20EE7
:10375000B31EE080F1800281138135E79316B1F446
:1037600021C0D5011296F50100811181F5E79F1660
:1037700031F45D01980179010027112713C05D0123
:10378000A8017A010027F7FC0095102F17FF0AC047
:1037900010950095F094E094E11CF11C011D111DA1
:1037A0008DE2898357FC02C05FEE6522E114F104CB
:1037B0000105110539F44114510451F402E1C02E00
:1037C000D12C0CC06AE0E616F1040105110548F49D
:1037D0008E2D805D898B11E1C12ED12CCC0EDD1E8A
:1037E000C4C0B2E1CB2ED12CCC0EDD1EC801B70176
:1037F0002AE030E040E050E00E941B85605DD60189
:103800006E936D01C801B7012AE030E040E050E05E
:103810000E941B8579018A01211531054105510559
:1038200029F7A3C063FE09C024E030E0A20EB31E56
:10383000008111812281338109C042E050E0A40E51
:10384000B51E808191818C0122273327198257FC74
:1038500002C05FEE6522011511052105310549F40D
:103860004114510431F4A2E1CA2ED12CCC0EDD1E3C
:103870001FC0F2E1CF2ED12CCC0EDD1E802F877021
:10388000805DD6018E936D01E3E0369527951795FF
:103890000795EA95D1F7011511052105310571F755
:1038A00060FE06C0803321F080E3FD0182936F014A
:1038B0008E010C191D090E5E1F4F70C020E7921675
:1038C00071F442E050E0A40EB51E808191818C011C
:1038D0002227332751E0652A78E7972E14C063FE2C
:1038E00009C064E070E0A60EB71E0081118122813C
:1038F000338109C082E090E0A80EB91E80819181D9
:103900008C012227332757FC02C09FEE6922A8E5CD
:103910009A1619F048E854E002C049E954E01982C7
:1039200062E1C62ED12CCC0EDD1EF801EF70F070D6
:10393000E40FF51F8081F60182936F0194E03695C4
:103940002795179507959A95D1F70115110521052A
:10395000310559F760FE09C0319790826F010894D4
:10396000C108D10880E3D6018C938E010C191D0982
:103970000E5E1F4F792C12C0E4E0F0E0AE0EBF1EC9
:10398000992009F491C09A821982792C82E0C82E7C
:10399000D12CCC0EDD1E01E010E07EC078010415B4
:1039A00015050CF472018981882319F00894E11C33
:1039B000F11C4201262D33273F8B2E8B290134E148
:1039C000432255244114510461F42A893B892E195C
:1039D0003F094AEA54E06A8D7B8D888D998D0E945B
:1039E000051A8981882359F041E050E0BE016F5FDC
:1039F0007F4F8A8D9B8DA88DB98DFD010995B0E112
:103A00004B16510461F42A893B892E193F094AEB70
:103A100054E06A8D7B8D888D998D0E94051A801ADD
:103A2000910A94014AEB54E06A8D7B8D888D998DC3
:103A30000E94051A0115110539F0A801B6018A8DF9
:103A40009B8DE88DF98D0995F0E57F1619F4C60177
:103A50000E94F5192E8922FF0CC02A893B892E1954
:103A60003F094AEA54E06A8D7B8D888D998D0E94CA
:103A7000051A4A895B894E155F053CF06C897D8982
:103A8000640F751F7D8B6C8B0ACD8C899D898E0D83
:103A90009F1D9D8B8C8B03CD780117FF02C0EE24F8
:103AA000FF248824992486CF8C899D896B960FB634
:103AB000F894DEBF0FBECDBFDF91CF911F910F9164
:103AC000FF90EF90DF90CF90BF90AF909F908F903E
:103AD0007F906F905F904F903F902F9008952F921E
:103AE0003F924F925F926F927F928F929F92AF928E
:103AF000BF92CF92DF92EF92FF920F931F93CF93DB
:103B0000DF93CDB7DEB763970FB6F894DEBF0FBE75
:103B1000CDBF3C014B012A01590122243324FF244B
:103B2000D2011C91112309F494C10894411C511C29
:103B3000812F99270E945B85892B99F041E050E005
:103B4000BE016F5F7F4FC401F3010995019741F7F3
:103B5000898199270E945B85892B81F7A1E0FA2E44
:103B6000DFCF153289F0FF2059F441E050E0BE016B
:103B70006F5F7F4FC401F3010995019709F0A5C05C
:103B80008981811761F265C1F20181912F0185322E
:103B900091F4FF2059F441E050E0BE016F5F7F4F88
:103BA000C401F3010995019709F08FC0898185321D
:103BB00009F4B5CF4EC1982FCC24DD2400E02AE0D3
:103BC00030E09A3211F4026016C09C3611F40160A4
:103BD00012C0892F80538A3090F4A601429F600161
:103BE000439FD00C529FD00C1124C90ED11C80EDE4
:103BF0009FEFC80ED91ED2019D912D01E2CF9F36B5
:103C000009F450C1903748F4933609F44FC19936FE
:103C100061F0992309F443C149C0933721F09837E3
:103C200009F044C005C012E042C013E0EE2441C0D8
:103C3000006113E0F0E1EF2E3CC001FD12C024C092
:103C4000FF2059F440E150E0BE016E5F7F4FC40198
:103C5000F301099518161906C4F5E0EFFFEFCE0E33
:103C6000DF1EF1E1CF16D10458F7FF2009F07EC026
:103C7000A601BE016E5F7F4FC401F30109951816BE
:103C800019060CF473C021C0FF2009F06EC0D501E5
:103C90006D917C91A601C401F301099518161906CE
:103CA000A4F4E2E0F0E0AE0EBF1E5FC013E0EAE075
:103CB000EE2EFF2071F441E050E0BE016F5F7F4FB8
:103CC000C401F3010995019721F0222009F4E7C00E
:103CD000C0C0F9808F2D99270E945B85892B59F7E9
:103CE000123009F048C0C114D10419F47FEFC72E77
:103CF000D72E01FF17C00894C108D108C114D10400
:103D0000A9F141E050E0BE016F5F7F4FC401F301B4
:103D10000995019759F5898199270E945B85892B1F
:103D200029F5E9CFD5010D911C91F801F1928F0190
:103D30000894C108D108C114D10489F041E050E0D1
:103D4000BE016F5F7F4FC401F3010995019739F4FC
:103D5000F9808F2D99270E945B85892B31F342E0F2
:103D600050E0A40EB51ED8011C9233942394D7CEF4
:103D700061E0F62E6AC0133009F0D1CEC60101977A
:103D80000F9718F05FE0C52ED12C102F1C62FE019A
:103D90003296FB8BEA8B54C09981903349F4EE2024
:103DA00019F4106148E0E42E15FF20C0137D32C0E5
:103DB000892F8153873018F4EE20C1F406C0892F73
:103DC0008853823048F4EE2019F43AE0E32E0EC016
:103DD000F8E0FE15C8F50AC0892F8154863018F026
:103DE0008052863028F44AE04E1570F5137E12C0DA
:103DF0009D3211F09B3221F412FF26C01B7F0AC0B6
:103E0000983719F0983509F0B3CF14FF1DC01F7E05
:103E100020E1E22EAA89BB899D93BB8BAA8BB2E0DD
:103E2000CB16D10450F041E050E0BE016F5F7F4FF0
:103E3000C401F3010995019739F40894C108D10828
:103E4000C114D10409F0A8CFFF24012F112703FFCB
:103E500003C0832D992732C001FD1FC0EA89FB8969
:103E600010824E2D552760E070E0CE0102960E9430
:103E7000418395012E5F3F4F00FF08C0D501ED91B2
:103E8000FC91608371838283938305C0D501ED919A
:103E9000FC917183608359013394239441CE8FEF59
:103EA0009FEF0CC013E098E0E92E03CFC114D104BA
:103EB00009F0C3CE81E0C82ED12CBFCE63960FB6D9
:103EC000F894DEBF0FBECDBFDF91CF911F910F9150
:103ED000FF90EF90DF90CF90BF90AF909F908F902A
:103EE0007F906F905F904F903F902F900895FC01CE
:103EF0008081823759F0873719F08136B1F403C0D9
:103F000081E093E41BC088E091E418C080E090E475
:103F100015C02B3219F0223641F404C08E7F826026
:103F200093600CC09F7B906809C086E190E09093FD
:103F3000490B8093480B8FEF9FEF089531962081B6
:103F4000222339F708950F931F93CF93DF93CDB7B3
:103F5000DEB721970FB6F894DEBF0FBECDBF8C0140
:103F6000FB01898341E050E0BE016F5F7F4F80819C
:103F700091810E94E219019711F00FEF1FEFC80124
:103F800021960FB6F894DEBF0FBECDBFDF91CF9163
:103F90001F910F910895FC01CB01DF010D900020CE
:103FA000E9F71197AE1BBF0BAD01BF01FC0180818A
:103FB00091810E94E2190895CB0108950895089512
:103FC000FC01E95DFD4F6193719331832083769706
:103FD000518340830895FC01ED5BFD4F7183608345
:103FE0003C97518340830895FC01EB58FD4F61934A
:103FF0007193518340830895FC01EE59FC4F619306
:104000007193518340830895AF92BF92CF92DF9214
:10401000EF92FF920F931F93CF93DF936C01A42E27
:10402000B22EFC01E758FD4F20E080819181861778
:10403000970731F02F5F77962A3009F44BC0F5CF00
:10404000822F992727E130E0829FE001839FD00DE6
:10405000929FD00D1124CC0DDD1DC657DD4F8881F8
:10406000CA58D2408530B1F5C601815E9D4F0E948D
:10407000BA51FE01E257FD4F80818F5F808382E05D
:10408000F7018083FE01E558FD4F8081E7018983B8
:1040900021818A2D99278370907034E0880F991FB1
:1040A0003A95E1F7282BBB0CBB0CBB0CBB0CBB0C33
:1040B000BB0C2B292A830B83812F99278C83B70173
:1040C000C6010E94FA2AFC01BF01882777FD80956E
:1040D000982F04C06DEF7EEF8FEF9FEFDF91CF91B0
:1040E0001F910F91FF90EF90DF90CF90BF90AF9016
:1040F0000895CF92DF92EF92FF920F931F93CF9389
:10410000DF93EC015CE6C52E53E0D52EC80ED91E18
:1041100060E070E00E940441F601A085B18510972F
:1041200051F0FD01E480F580068117812D913D91CC
:104130004D915C910CC04FEFE42E4FEFF42E4FEBFE
:10414000042F4FEF142F2FEF3FE140E050E060E0ED
:1041500070E0CE010E944F41F60146815781411522
:10416000510531F060E070E0CE010E948B4326C023
:104170001F921F9281E08F931F921F92DF93CF9324
:104180000E94D64382E090E09F938F931F921F92EC
:1041900082E08F931F921F92DF93CF930E94D643AA
:1041A000CE59DC4F19821882C256D3408DB79EB7C4
:1041B00040960FB6F8949EBF0FBE8DBFF601A28148
:1041C000B381109719F04D915C9102C040E45FE11A
:1041D00060E070E0CE010E94773FF601A689B789C2
:1041E000109719F04D915C9102C040E050E260E000
:1041F00070E0CE010E94D63EF601A28DB38D1097DD
:1042000011F04C9101C043E060E070E0CE010E94EB
:104210003E3EF601A285B385109711F04C9101C086
:1042200040E060E070E0CE010E94343DF601A685DA
:10423000B785109711F04C9101C041E060E070E04B
:10424000CE010E94173CF601A089B189109711F0A8
:104250004C9101C041E060E070E0CE010E947E3BE5
:10426000F601A481B581109739F04D915C9160E021
:1042700070E0CE010E94AB4EF601A485B585109783
:1042800069F0FD01E580F680038114814D915C9118
:10429000228160E070E0CE010E94AF3CF601A2896D
:1042A000B389109749F02D913D914D915C9160E05B
:1042B00070E0CE010E94903DF60144895589411578
:1042C000510529F060E070E0CE010E94FD42F60148
:1042D000A08DB18D109731F04C9160E070E0CE016F
:1042E0000E946C40D601ED91FC91309711F06081F5
:1042F00001C063E0CE010E94674F60E070E0CE0134
:104300000E94EE44DF91CF911F910F91FF90EF90AB
:10431000DF90CF9008958F929F92AF92BF92DF92DD
:10432000EF92FF920F931F93CF93DF93EC01FC0169
:10433000EA5BFD4F80819181892B09F096C08091C5
:10434000E3089091E40891838083EDE0AE2EB12CD8
:10435000AC0EBD1EC5010E94BA517DE6E72E72E08B
:10436000F72EEC0EFD1EC7010E94BA518E01085BAC
:104370001D4FC8010E94BA51C7010E94AC51C8012B
:104380000E94AC51FE01EE59FC4F808091808FED70
:104390009FE1918380838A819B810E94181840E06D
:1043A00052EC61E070E00E945C2D81E088870E9401
:1043B0003B53CF58DD4F19921882C257D24069E75C
:1043C000E62E62E0F62EEC0EFD1EDD24F70181895B
:1043D0008823A1F18FEF9FEF938382838081918166
:1043E0008F5F9F4F49F1D7014D915C9100E01FEF26
:1043F0002FEF3FEF6FEF7FEFCE010E94B9308C01BE
:104400008F5F9F4F81F7F7018189853091F4FE011D
:10441000EB58FD4FC958DD4F28813981C757D2402D
:10442000D7014D915C910190F081E02D68E083E02F
:104430000995F70111830083F701118AD39487E16D
:1044400090E0E80EF91E9AE0D91609F0BFCFCE0130
:104450000E947920CE59DC4F99828882C5010E9442
:10446000AC51CC51D14019821882DF91CF911F916C
:104470000F91FF90EF90DF90BF90AF909F908F9043
:104480000895CF93DF93CDB7DEB72C970FB6F8948E
:10449000DEBF0FBECDBF4C01AE014D5F5F4FBE0111
:1044A0006F5F7F4FC4010E94562C3C01009709F4B6
:1044B00076C0DC018C91833009F448C0843021F04F
:1044C000823009F06CC005C0B301C4010E943B35C5
:1044D00066C0F3010281602F77276F707070762FAE
:1044E000662781819927682B792BC4010E94582F58
:1044F000F3018183492F55272281207F242B22839A
:10450000F401E95DFD4FAB80BC80CD80DE80E980A9
:10451000FA8002950F70202F237049E252E0840E3A
:10452000951E0190F081E02D06950695AC01B30132
:10453000D4018D919C910995EAEEFFEF8E0E9F1E9E
:10454000D4018D939C93EDEEFDEF27C0F3016281C2
:1045500077276F707070762F662781819927682B77
:10456000792BC4010E94582F23E432E0820E931E5F
:10457000D401ED91FC912DEB3DEF820E931E29812C
:10458000AC01B301C401099547E352E0840E951EC6
:10459000D4018D939C93E9ECFDEF8E0E9F1E21E7D5
:1045A00032E0820E931ED4018C91EFE8FDEF8E0E67
:1045B0009F1E882309F440C0840106571D4FAA247A
:1045C000BB248DE7C82E82E0D82EC80CD91CB9E8D0
:1045D000EB2EB2E0FB2EE80CF91CF40187859089E4
:1045E00018161906D4F48385948518161906ACF4A8
:1045F000D8018C91823089F484E08C93F70140815A
:1046000042954F704370B601C4010E943749F401CE
:10461000EF58FD4F8081815080830894A11CB11C0C
:1046200027E130E0E20EF31EC20ED31E095E1F4FDB
:104630003AE0A316B10489F642E752E0840E951ED3
:10464000D4018C91EEE8FDEF8E0E9F1E882309F4B5
:1046500051C0A9E7EA2EA2E0FA2EE80CF91CAA2420
:10466000BB24FDE7CF2EF2E0DF2EC80CD91CF401ED
:1046700087859089181619067CF583859485181608
:10468000190654F5F7018689882331F584E090E016
:104690009A838983DE011796F60186E001900D92D8
:1046A0008150E1F7D7016D917C910AEC14E02981EA
:1046B000AE01495F5F4FC4010E940B48611571054F
:1046C0008105910549F483E0F701868BF401EE58EA
:1046D000FD4F8081815080830894A11CB11C27E18B
:1046E00030E0C20ED31EE20EF31E3AE0A316B10470
:1046F00009F0BDCF0E941008CFCE0F931F938B01FE
:10470000BA0141E050E00E949C42C8011F910F9104
:1047100008950F931F93CF93DF938C0188E893E064
:104720000E941409009719F4C0E0D0E053C0EC01D6
:104730001983088360E070E0815E9D4F0E94D15133
:1047400060E070E0CE01825C9D4F0E94D15161E03B
:1047500070E0CE01885B9D4F0E94D151CE010E9436
:10476000902D81E090E09093FD088093FC08CE01AD
:104770000E940431C95DDD4F8DE793E289939993DF
:1047800019821882669719821882E0968CED9FE153
:10479000998388832C9719821882EE968EED9FE17B
:1047A0008993999319821882C757D24020E034E048
:1047B000AE0161E472E28FEC94E00E94070BCE013F
:1047C0000E947920AE014A595C4F60E070E0CE0152
:1047D0000E94A844CE01DF91CF911F910F910895BF
:1047E000FC01828199278F709070982F88272181F2
:1047F0003327822B932B0895FC01818182958F7042
:104800009927837090700895FC0181818295869527
:10481000869583709927089505960895FC01E95EB1
:10482000FD4F808191810895FC01EB5DFD4F8081FA
:1048300091810895EF92FF920F931F93CF93DF938F
:10484000EC0164FF04C0AAE1EA2EF12C03C0F0E100
:10485000EF2EF12C72FF03C0E9E7EE2EF12C73FF6F
:1048600003C057EBE52EF12C76FF03C040EEE42E9B
:10487000F12C77FF04C033E5E32E31E0F32EC95E5F
:10488000DD4F79836883C751D2408E010B5D1D4F88
:10489000F801F182E08261E070E0CE01855D9D4F1C
:1048A0000E94D151C15DDD4F8FEF9FEF89939993A6
:1048B0001992199219821882F801808191810796C4
:1048C0000E9414096E9799838883C701DF91CF9165
:1048D0001F910F91FF90EF900895EF92FF920F9329
:1048E0001F93CF93DF93EC017A018C01015D1D4F83
:1048F000F80140815181FFEF4F3F5F0729F464EFDA
:104900007EEF8FEF9FEF43C0CD5CDD4FE881F981F3
:104910009F012E0D3F1D9A918A91C153D24082175B
:10492000930750F48FEF9FEFF8019183808365EF39
:104930007EEF8FEF9FEF2BC0452B81F0A701CE01BB
:104940000E94F42A892BB1F08FEF9FEFF801918339
:1049500080836FEF7EEF8FEF9FEF19C0CB5EDD4F4F
:1049600088819981C551D2400596A7018E0F9F1F5E
:104970000E949884FE01ED5CFD4F808191818E0D37
:104980009F1D9183808360E070E080E090E0DF9184
:10499000CF911F910F91FF90EF9008955F926F92CA
:1049A0007F928F929F92AF92BF92CF92DF92EF92BF
:1049B000FF920F931F93CF93DF93CDB7DEB7259769
:1049C0000FB6F894DEBF0FBECDBF7C013B01C42EF5
:1049D000D22E48018BE2A82E82E0B82EAE0CBF1C6E
:1049E000C5010E94BA514FE252E0E40EF51E8FEF6E
:1049F0009FEFD7018D939C93E4E0F0E0EE0EFF1E55
:104A0000D7011D921C92F701129212927F014FEC76
:104A10005DEFE40EF51E6114710421F420E030E036
:104A200055242AC0F701E758FD4F55248189853068
:104A300029F4808191818615970569F053947796C2
:104A40005AE0551699F7C5010E94AC516DEF7EEF03
:104A50008FEF9FEF9BC0252D332787E190E0289FA4
:104A6000F001299FF00D389FF00D1124EE0DFF1D70
:104A7000E558FD4F2081318185E292E0E80EF91E74
:104A8000D7018D919C91EBEDFDEFEE0EFF1E881589
:104A9000990540F4C5010E94AC5165EF7EEF8FEFA0
:104AA0009FEF74C082E089832A83232F3327DD0C94
:104AB000DD0CDD0CDD0CDD0CDD0C8C2D99278370FD
:104AC000907014E0880F991F1A95E1F7D82AD22A1E
:104AD000DB828C82892D99278D836E010894C11CFD
:104AE000D11C6114710489F18701015E1D4FC80159
:104AF0000E94BA51252D332787E190E0289FF001CD
:104B0000299FF00D389FF00D1124EE0DFF1DE25787
:104B1000FD4F80818F5F8083C7010E94682A45E036
:104B200050E0B601C7010E94F42A97FF1FC0C701D9
:104B30000E94642AC8010E94AC51C5010E94AC5178
:104B40006FEF7EEF8FEF9FEF21C045E152E0E40E63
:104B5000F51ED701ED91FC914BEE5DEFE40EF51ED5
:104B6000D60185E00D9001928150E1F78FE292E04D
:104B7000E80EF91ED7016D927D92FD01819291920E
:104B80001182108260E070E080E090E025960FB620
:104B9000F894DEBF0FBECDBFDF91CF911F910F9173
:104BA000FF90EF90DF90CF90BF90AF909F908F904D
:104BB0007F906F905F9008952F923F924F925F92F7
:104BC0006F927F928F929F92AF92BF92CF92DF921D
:104BD000EF92FF920F931F93CF93DF93CDB7DEB782
:104BE00024970FB6F894DEBF0FBECDBF9C838B8396
:104BF0003FE2E32E32E0F32EE80EF91EF70180814A
:104C00009181892B91F08B819C810E94642AF7010C
:104C1000808191818F5F9F4F09F04DC08B819C8176
:104C2000815E9D4F0E94AC5146C00E9441055B01D0
:104C30006C0125E1222E22E0322E2B813C81220EB6
:104C4000331EF10160807180F301818097E2492E6B
:104C500092E0592E420E531E2D5C3D4FF901E0802B
:104C6000F180E353F240FC83EB83082D0295069517
:104C700006950370112786948694869486949924C9
:104C8000F3E08F229924C3010E94F0232B813C8101
:104C9000275D3D4F3A832983F201A081B181282D00
:104CA000AC01B301E981FA8180819181FD0109950F
:104CB000F101918380838B819C81855D9D4F0E9452
:104CC000AC5124960FB6F894DEBF0FBECDBFDF9176
:104CD000CF911F910F91FF90EF90DF90CF90BF90F9
:104CE000AF909F908F907F906F905F904F903F908C
:104CF0002F900895AF92BF92CF92DF92EF92FF92E2
:104D00000F931F93CF93DF93EC0158016701870145
:104D10000E94CE247B018C016115710581059105EE
:104D200051F4A601B501CE010E946D247B018C01D6
:104D3000CE010E94DC25C801B701DF91CF911F9100
:104D40000F91FF90EF90DF90CF90BF90AF900895BC
:104D5000FC01248135810280F381E02D60E070E068
:104D60000AC0808191813A96892B19F48827992766
:104D700008956F5F7F4F6217730799F76DEF7FEFAD
:104D80008FEF9FEF0895FC01AB01248135810280F4
:104D9000F381E02D60E070E00BC0808191813A9654
:104DA0008417950719F48827992708956F5F7F4F17
:104DB0006217730791F76AEF7FEF8FEF9FEF089508
:104DC000CF93DF93EC018C819D818617970788F044
:104DD0008AE090E0689FF001699FF00D789FF00DE8
:104DE00011248A819B81E80FF91F80819181892B91
:104DF00011F4E0E0F0E0CF01DF91CF910895FC01E4
:104E0000808591850895CF92DF92EF92FF920F9364
:104E10001F93CF93DF93EC018B017A0169010E940C
:104E2000C3266A5F7F4F8F4F9F4F29F04EEF5FEF92
:104E30006FEF7FEF24C0CE010E94A826AB01BC011A
:104E400077FF05C04DEF5FEF6FEF7FEF18C08AE08F
:104E500090E0489FF001499FF00D589FF00D1124FC
:104E60008A819B81E80FF91FF582E482D782C6828E
:104E700011830083538342832696D187C087CB0159
:104E8000BA01DF91CF911F910F91FF90EF90DF90CA
:104E9000CF900895CF93DF93DC01EC018C819D814D
:104EA0008617970718F48BEF9FEF16C08AE090E003
:104EB000689FF001699FF00D789FF00D1124ED01BE
:104EC0008A819B81E80FF91F11821082158214825A
:104ED0001782168280E090E0DF91CF910895CF9302
:104EE000DF93EA010E94E026FC01892B19F48BEF85
:104EF0009FEF04C0D187C08780E090E0DF91CF9121
:104F00000895AF92BF92CF92DF92EF92FF920F93EC
:104F10001F936C017B015A018AE090E09C01629F23
:104F2000C001639F900D729F900D11240E960E94F8
:104F300014098C01FC01F582E4820E96938382832E
:104F4000D182C082B501C6010E94A452F8019783A4
:104F50008683B186A0860E947D52F801938782875E
:104F600020E038E0A8016BE378E287ED94E00E944E
:104F7000070BC8011F910F91FF90EF90DF90CF902A
:104F8000BF90AF9008956F927F928F929F92AF9251
:104F9000BF92CF92DF92EF92FF920F931F93CF9326
:104FA000DF935C016B013A014901B8010E94C326FD
:104FB0009B01AC0197FF03C08AEF9FEF4DC08AE0D1
:104FC00090E0289FD001299FB00D389FB00D11248B
:104FD000E5018A819B81A80FB91FFD01C085D1859C
:104FE000209749F188819981009731F4E701D982AE
:104FF000C88289EF9FEF30C0F70191838083FC0165
:105000008281938199838883E701E881F981138202
:105010001282F6017782668291868086B787A6879C
:10502000B601E5018A859B850E943152C5010C9627
:105030000E945E090FC0FD01068117812281338124
:105040000480F581E02DA401B301C6010995E701B3
:105050009983888380E090E0DF91CF911F910F9139
:10506000FF90EF90DF90CF90BF90AF909F908F9088
:105070007F906F900895EC018A859B850E94FE5178
:10508000009711F1FC01E684F784F701068117818E
:1050900022813381FC014085518566817781F7014A
:1050A000C480D580F6010995DC01F70120853185A2
:1050B000F90180819181FD0193838283F901B1839C
:1050C000A0830E941008D8CF40E050E060E070E07C
:1050D000CE010C960E94400ACFCFFC0162857385F9
:1050E00084859585089560911009709111098091CA
:1050F000120990911309089560910C0970910D099E
:1051000080910E0990910F09089560911409709192
:10511000150980911609909117090895709309094E
:105120006093080950930B0940930A0908958091F0
:10513000FE089091FF080E94142406970895AF92EC
:10514000BF92CF92DF92EF92FF920F931F935C0179
:105150008B019093FF088093FE0870930109609380
:1051600000090E948952FC0190930309809302096F
:105170004081518120E030E068EA79E2C5010E9477
:10518000E01F109209091092080910920B09109261
:105190000A09C5010E9414246C0110920C09109296
:1051A0000D0910920E0910920F0910921009109219
:1051B00011091092120910921309109214091092F9
:1051C00015091092160910921709109204091092ED
:1051D00005091092060910920709C8010E94FF26CE
:1051E00025E030E0C20ED31EEE24FF248C0120E027
:1051F000A60160E070E0C5010E94AF3C1F910F91D5
:10520000FF90EF90DF90CF90BF90AF9008950E94F5
:105210000C2406960895AB01BC018091FE08909184
:10522000FF080E946D240895809110099091110942
:10523000A0911209B09113090196A11DB11D80938F
:10524000100990931109A0931209B093130980914A
:10525000FE089091FF080E94DC250895EF92FF92CE
:105260000F931F93CF93DF93CDB7DEB726970FB67B
:10527000F894DEBF0FBECDBF242F2E5F29834E5F73
:105280005F4F252F33272A8322E02B831C826D83D7
:10529000672F77276E834C5F5F4F8A0120E042E0E3
:1052A000BC018091FE089091FF080E94CE247B01F2
:1052B0008C0197FD15C046E050E0BE016F5F7F4F47
:1052C0008091FE089091FF080E946D247B018C0163
:1052D00097FF06C08091FE089091FF080E94DC2590
:1052E000C801B70126960FB6F894DEBF0FBECDBF3A
:1052F000DF91CF911F910F91FF90EF900895CF9282
:10530000DF92EF92FF920F931F93CF93DF936C0185
:10531000EB01CA01AB01B9010E942E297B018C016E
:10532000611571058105910541F4BE01C6010E9418
:105330000B297B018C010E941429C801B701DF9160
:10534000CF911F910F91FF90EF90DF90CF90089534
:105350002F923F924F925F926F927F928F929F9285
:10536000AF92BF92CF92DF92EF92FF920F931F9373
:10537000CF93DF93CDB7DEB722970FB6F894DEBF99
:105380000FBECDBF1C014B01622F2501360180915C
:105390000C0990910D09A0910E09B0910F09019689
:1053A000A11DB11D80930C0990930D09A0930E09C6
:1053B000B0930F09E5E0CE2ED12CC80CD91CF60114
:1053C0002281332783819927982F8827282B392BEF
:1053D0002230310571F0E0910809F0910909309708
:1053E00041F063015201262FB401C10109954C011E
:1053F00051C0C4010E94F0238F5F9F4F79F1F601E5
:105400000481112785819927982F8827082B192B2C
:105410002081332781819927982F8827282B392BA2
:10542000E0910209F09103094286538664867586ED
:10543000918280822250304086E090E0C80ED91ED2
:105440007E010894E11CF11CA601BF0180910009B6
:10545000909101090E94C327892BA1F08091140922
:1054600090911509A0911609B09117090196A11DF7
:10547000B11D8093140990931509A0931609B09358
:10548000170908C0E981FA81F0930309E093020942
:1054900080809180C40122960FB6F894DEBF0FBEC3
:1054A000CDBFDF91CF911F910F91FF90EF90DF90D3
:1054B000CF90BF90AF909F908F907F906F905F90B4
:1054C0004F903F902F90089504960E94AC510895FC
:1054D00004960E94BA510895AF92BF92CF92DF9284
:1054E000EF92FF920F931F93CF93DF93CDB7DEB769
:1054F00063970FB6F894DEBF0FBECDBF5C017B0192
:105500006A01DE011196EDEDF4E083E101900D9268
:105510008150E1F780918D07882341F080ED90E084
:105520009F938F930E94177C0F900F9000E010E0E4
:1055300011C0C5010E941818A601401B510BB701EC
:10554000600F711F0E94E2192FEF8F3F920781F1C8
:10555000080F191F0C151D0560F380918D07882316
:1055600001F100E010E012C0F70181917F0199275D
:105570009F938F9389EC90E09F938F930E94177C69
:105580000F5F1F4F0F900F900F900F900C151D0580
:1055900059F787EC90E09F938F930E94177C0F90B0
:1055A0000F90C5010E94EC7B8F5F9F4F51F406C0A6
:1055B000BE016F5F7F4F8BE00E94E5708FEF9FEF22
:1055C00002C080E090E063960FB6F894DEBF0FBE95
:1055D000CDBFDF91CF911F910F91FF90EF90DF90A2
:1055E000CF90BF90AF900895FC01828193810E947B
:1055F0006C2A0895EF92FF920F931F93CF93DF933E
:105600007C018B01FB014081423029F1433020F4C1
:10561000413009F04BC006C0433041F1443009F03D
:1056200045C02AC0FB018381C82FDD2723969281C4
:10563000892F86958695833021F5892F9927982F74
:10564000882721813327822B932B93700397C9F4EA
:10565000F701408716C0FB0184819927D82FCC27FA
:1056600083819927C82BD92B24960BC0FB018381FA
:10567000C82FDD27239605C0FB018281C82FDD27B7
:105680002296C7010E94682A2196AE01B801C7017F
:105690000E94F42A8C01C7010E94642A8FEFF7014F
:1056A000818B17FD03C080E090E002C08FEF9FEF79
:1056B000DF91CF911F910F91FF90EF9008954F923E
:1056C0005F926F927F928F929F92AF92BF92CF9292
:1056D000DF92EF92FF920F931F93CF93DF93CDB79B
:1056E000DEB7C954D0400FB6F894DEBF0FBECDBFB1
:1056F0003C012B015A01FC01E280F380DE0192960D
:10570000E0EFF4E082E101900D928150E1F7DE01DB
:105710005396E2E0F5E08FE001900D928150E1F7C1
:10572000DE01D496E1E1F5E086E101900D92815031
:10573000E1F7DE011596E7E2F5E08EE001900D92CB
:105740008150E1F7CC24DD2462C0C7010E94181803
:10575000A5014C195D09B2016C0D7D1D0E94047CF0
:105760004C018F5F9F4F09F45DC0C7010E9418185C
:105770008E010F5F1F4FA8016AE071E00E94781947
:10578000F3018085882369F087E090E0A0E0B0E035
:1057900089839A83AB83BC83C7010E941818A80130
:1057A00030C029813A814B815C81DA01C90187705F
:1057B0009070A070B0700097A105B10531F120FF85
:1057C00004C0BE016D5E7F4F0BC021FF04C0BE014F
:1057D0006C5C7F4F05C022FF06C0BE016B5F7F4F30
:1057E0008BE00E94E57087E090E0A0E0B0E0898364
:1057F0009A83AB83BC83C7010E941818AE014F5F28
:105800005F4F69E071E00E947819C80CD91CCA1476
:10581000DB0408F49ACF80918D07882361F480E03F
:1058200090E02CC0BE016E5D7F4F8BE00E94E57062
:105830008FEF9FEF23C000E010E0720112C0F7016C
:1058400081917F0199279F938F9384ED90E09F939F
:105850008F930E94177C0F5F1F4F0F900F900F9038
:105860000F900A151B0559F782ED90E09F938F93D7
:105870000E94177C80E090E00F900F90C75BDF4F95
:105880000FB6F894DEBF0FBECDBFDF91CF911F9151
:105890000F91FF90EF90DF90CF90BF90AF909F90CF
:1058A0008F907F906F905F904F900895CF92DF928E
:1058B000EF92FF920F931F93CF93DF93CDB7DEB795
:1058C000A1970FB6F894DEBF0FBECDBF7C016B0170
:1058D0008A01FC0182819381DE011296E5E3F5E005
:1058E00020E201900D922150E1F70E94181841E04A
:1058F00050E0BE016F5F7F4F0E94047C019709F06A
:10590000C9C080918D07882371F0898199279F9361
:105910008F9380EC90E09F938F930E94177C0F9061
:105920000F900F900F9089818330C1F1843009F47A
:105930005FC0823009F096C00E944105F801608383
:1059400071838283938323E132E0E20EF31EF70139
:10595000008111812DEE3DEFE20EF31E8981F801E9
:10596000819344E050E0BF01C7010E945F2B892B67
:1059700009F090C0F80184819927582F442783812A
:105980009927482B592BF601518340834115510526
:1059900009F473C0B8016B5F7F4F23C027E332E087
:1059A000E20EF31EF7010081118129EC3DEFE20EBA
:1059B000F31EF801819343E050E0BF01C7010E944C
:1059C0005F2B892B09F066C0F8018381482F55278A
:1059D000F60151834083882309F44FC0B8016C5FFE
:1059E0007F4FC7010E945F2B892B09F446C052C02C
:1059F00087010F5E1E4FF801819342E050E0BF0126
:105A0000C7010E945F2B892B09F044C0F8018281F5
:105A1000482F5527F60151834083882341F0B80170
:105A20006D5F7F4FC7010E945F2B892B99F5F701AE
:105A30008085882311F1F80181818E30F1F4958100
:105A4000892F86958695C9F4892F9927982F8827BD
:105A500024813327822B932B9370892B71F4F701C8
:105A600010860BC0F70180858823A1F4BE016E5F0C
:105A70007F4F8CE00E94E5700DC080918D078823D8
:105A800059F08EEB90E09F938F930E94177C0F90BC
:105A90000F9002C000E010E0C801A1960FB6F89484
:105AA000DEBF0FBECDBFDF91CF911F910F91FF9051
:105AB000EF90DF90CF9008950F931F93CF93DF93D4
:105AC000CDB7DEB724970FB6F894DEBF0FBECDBFBB
:105AD0008C0149835A836B837C8340E050E060E013
:105AE00070E00E94E21984E60E949B0BAE014F5FBA
:105AF0005F4F61E071E0C8010E947819892B19F0AD
:105B00008FEF9FEF02C080E090E024960FB6F894EC
:105B1000DEBF0FBECDBFDF91CF911F910F910895D2
:105B20002F923F924F925F926F927F928F929F92AD
:105B3000AF92BF92CF92DF92EF92FF920F931F939B
:105B4000CF93DF93CDB7DEB724970FB6F894DEBFBF
:105B50000FBECDBF2C0161E070E004960E94D151D0
:105B600040E060E070E0F201808191810E94EC03EE
:105B7000892B09F01BC1F2018081918165E575E0F7
:105B800002960E941C18F201938382830E941818C7
:105B9000181619060CF00AC1F201828193810E9445
:105BA000181840E052EC61E070E00E945C2D892BF7
:105BB00009F0FCC019821A821B821C82F2018281C8
:105BC00093810E9418181E010894211C311CA10108
:105BD00065E071E00E947819892B09F0E7C088E040
:105BE00090E0A0E0B0E089839A83AB83BC83F201AC
:105BF000828193810E941818A10163E071E00E94E4
:105C00007819892B09F0D2C081E090E0A0E0B0E0E3
:105C100089839A83AB83BC83F201828193810E9442
:105C20001818A10167E071E00E947819892B09F02A
:105C3000BDC019821A821B821C82F201828193816B
:105C40000E941818A10163E171E00E947819892B64
:105C500009F0ACC083E090E0A0E0B0E089839A83D3
:105C6000AB83BC83F201828193810E941818A10149
:105C700061E171E00E947819892B09F097C0F20167
:105C80001086828193810E94181840E050E060E005
:105C900070E00E94047C80E092E0A0E0B0E08983A4
:105CA0009A83AB83BC83F201828193810E9418188E
:105CB000A1016BE171E00E9478193C01882477FC16
:105CC0008094982CF201828193810E941818A1017E
:105CD0006DE171E00E947819AA2797FDA095BA2F6F
:105CE000680E791E8A1E9B1E84EF91E0A0E0B0E052
:105CF00089839A83AB83BC83F201828193810E9462
:105D00001818A10162E271E00E9478197C01F20189
:105D1000828193810E941818A10166E271E00E94BD
:105D200078195C01CC24B7FCC094DC2C0027F7FC6C
:105D30000095102FAE0CBF1CC01ED11E82EC91E04E
:105D4000A0E0B0E089839A83AB83BC83F2018281B7
:105D500093810E941818A10160E271E00E947819F5
:105D6000AA2797FDA095BA2F680E791E8A1E9B1E42
:105D7000F201828193810E941818A10164E271E00E
:105D80000E947819AA2797FDA095BA2FA80EB91ED0
:105D9000CA1EDB1E6A0C7B1C8C1C9D1C61147104CA
:105DA0008104910419F480E090E002C08FEF9EEF2F
:105DB00024960FB6F894DEBF0FBECDBFDF91CF9112
:105DC0001F910F91FF90EF90DF90CF90BF90AF9019
:105DD0009F908F907F906F905F904F903F902F900B
:105DE00008950895CF93DF93FC01E45BFD4F20E01D
:105DF00030E0EC01C459DD4FDF01808191810097D3
:105E000031F46D937C93288380E090E00FC0861777
:105E1000970719F48EEF9FEF09C02F5F3F4F12963F
:105E200032962031310549F78FEF9FEFDF91CF9107
:105E30000895DC01A45BBD4F20E0ED91FC9111972A
:105E4000309751F0808191818617970729F48281DC
:105E500093818417950731F02F5F1296203169F7EF
:105E6000E0E0F0E0CF010895DC01A657BD4F20E04F
:105E700030E04FEF5FEFFC01E758FD4F8C91882336
:105E800061F481E0818B8089806F808B51834083B6
:105E900053834283158A168A09C02F5F3F4F779636
:105EA00057962A30310551F72FEF3FEFC90108957A
:105EB0002FEF6F3F7207D1F0FC01E558FD4F20E056
:105EC00030E0DC01A758BD4F8785853041F48081E3
:105ED00091818617970719F48D919C9108952F5FF2
:105EE0003F4F579677962A30310571F78FEF9FEF26
:105EF0000895FC01E758FD4F20E030E0DC01A55893
:105F0000BD4F8189853041F4808191818617970743
:105F100019F48D919C9108952F5F3F4F5796779676
:105F20002A30310571F78FEF9FEF08958F929F927E
:105F3000AF92BF92CF92DF92EF92FF920F93CF93E7
:105F4000DF93EC014B015A016901CA5BDD4F2881E7
:105F50003981C654D2402115310539F08091E308CA
:105F60009091E4082817390721F0CE010D960E9480
:105F7000BA51033021F485E3E816F10421F0CE0193
:105F800009960E94BA5181E0F6018083000F000F4C
:105F90000283E182A114B10409F04501C401DF913B
:105FA000CF910F91FF90EF90DF90CF90BF90AF9087
:105FB0009F908F9008959C01FC01E459FD4F8081D2
:105FC0008F3F39F08FEF8083C90183599D4F0E9425
:105FD000AC5108958F929F92AF92BF92CF92DF9271
:105FE000EF92FF920F931F93CF93DF93EC017B010E
:105FF0004A016901672B99F18DE6A82E82E0B82E3F
:10600000AC0EBD1EC5010E94BA51F701D182C082FB
:106010001383028313861286B701CE010E94F22EEB
:106020000097E9F0FFEF8F3F9F0739F468EE73E0C8
:1060300080E090E00E944E06EFCF8E5F9F4F61F7A9
:10604000CE010E94F12EC5010E94AC51CE010D96E9
:106050000E94AC5160E07FEF8FEF9FEF3BC0BE012D
:106060006F5E7F4FCE010E94FA2A8C01CA5BDD4F22
:1060700028813981C654D2402115310539F08091EB
:10608000E3089091E4082817390721F0CE010D9616
:106090000E94AC510115110531F0B801882777FD38
:1060A0008095982F17C0E114F10481F0892871F4CC
:1060B00040E050E060E070E0C7010A960E94400AAC
:1060C000F701648175818681978104C060E070E08A
:1060D00080E090E0DF91CF911F910F91FF90EF90C2
:1060E000DF90CF90BF90AF909F908F900895FF92D8
:1060F0000F931F93CF93DF93EC01F62E062F1127FA
:10610000000F111F0C0F1D1F045B1D4FD801ED91D7
:10611000FC912483358346835783CF010A960E94DE
:10612000AD09D801ED91FC9111978FEF9FEF938707
:1061300082871D921C92C459DD4F8881CC56D24073
:106140008F1519F4CE010E94DB2FDF91CF911F91A3
:106150000F91FF900895FC019A01AB01E459FD4FA6
:106160006081EC56F2406F3F19F0CF010E9477300A
:1061700008956F927F928F929F92AF92BF92CF922B
:10618000DF92EF92FF920F931F93CF93DF934C0117
:106190005B013A0168017901EC01C45BDD4F2FEF2F
:1061A0003FEF00E010E0E881F9813097B9F082819B
:1061B00093818615970591F48FEFA8168FEFB80697
:1061C00029F0808191818A159B0541F4A7019601F0
:1061D000602FC4010E94773020E030E00F5F1F4F36
:1061E000229600311105F9F6C901DF91CF911F9177
:1061F0000F91FF90EF90DF90CF90BF90AF909F9066
:106200008F907F906F9008951F93CF93DF93EC0151
:106210001FEF198B61E070E009960E94D151CF5EAB
:10622000DE4F1883C151D140FE01E45BFD4F80E099
:10623000119211928F5F8031D9F7DE01A758BD4FBF
:1062400020E030E04FEF5FEFBE0167577D4FFD016B
:10625000118A11965C934E9353834283FB01808194
:106260008F7C80832F5F3F4F695E7F4F57962A3028
:10627000310569F7CF58DD4F1882C157D24061E030
:1062800070E0CE010D960E94D15160E070E0CE0129
:1062900083599D4F0E94D151CE010E94DB2FFE01F8
:1062A000ED5EFD4FC75EDD4FD183C083C951D24043
:1062B000CE01875C9D4FC95CDD4F99838883DF9158
:1062C000CF911F9108950F931F93CF93DF93EC010C
:1062D0008B01FB014381442319F40E94DB2F0AC088
:1062E0005527509541955F4F662757FD6095762F4E
:1062F0000E94AB30F80164817727CE0109960E9495
:106300009F51DF91CF911F910F9108953F924F922E
:106310005F926F927F928F929F92AF92BF92CF9235
:10632000DF92EF92FF920F931F93CF93DF93CDB73E
:10633000DEB726970FB6F894DEBF0FBECDBF5C0167
:106340007B01FB0133968281382E3694369499274F
:10635000D82ECC2481819927C82AD92A8FEF93E09F
:10636000C822D92293E0391609F4CCC0931538F02D
:10637000A1E03A1681F0A31508F455C021C3B5E099
:106380003B1609F463C23B1608F4AAC1EFE33E16BC
:1063900009F0FDC2E5C2FCE0CF16D10409F43FC00C
:1063A0003DE0C316D10439F182E0C816D10409F0EA
:1063B000EEC218E4812E12E0912E8A0C9B1CC401BF
:1063C0000E9456514FEF5FEF64E071E0C5010E94FB
:1063D000192FFC01892B59F0048115812681378101
:1063E0004FEF5FEF64E071E0C5010E94B930C40176
:1063F0000E94AC51CCC24FEF5FEF64E07DE0C5017D
:106400000E94192F20E030E0DE011196F701379647
:1064100081918D932F5F3F4F26303105C9F7C5011C
:106420000E94DB2FB4C29DE0C916D10409F440C01C
:10643000AEE0CA16D10450F4B9E0CB16D10481F015
:10644000ECE0CE16D10409F0A2C219C0FEE0CF16CE
:10645000D104E9F13FE0C316D10409F098C24BC062
:10646000FB0180859927582E442487819927482A43
:10647000592A8185682E7724882499249FC2FB019C
:1064800080859927582E442487819927482A592A9C
:106490008681882309F0CAC282859927982F882788
:1064A00021853327822B932B3C0188249924C2C257
:1064B000FB0180859927582E442487819927482AF3
:1064C000592A86819927909581959F4FAEC0FB01EF
:1064D0008681882309F0A7C280859927982F88276D
:1064E00027813327822B932B3C01882499244FEF5B
:1064F000442E542E9FC2FB01868199279095819549
:106500009F4F72C0F7E1CF16D10409F464C038E19F
:10651000C316D104D0F489E0C816D10409F48BC0A5
:106520009AE0C916D10430F4A3E0CA16D10409F0E8
:106530002EC229C0B4E1CB16D10409F483C0E5E131
:10654000CE16D10409F023C246C0F6E3CF16D1041B
:1065500009F45AC037E3C316D10458F489E1C816C8
:10656000D10409F468C093E2C916D10409F00FC23E
:1065700015C0A7E3CA16D104E9F1B4E4CB16D104DF
:1065800009F005C228C0E5E4F2E0AE0EBF1ED50159
:106590001C92EBEBFDEFAE0EBF1EF9C1FB01808537
:1065A0009927AA27BB276624782E892E9A2E8185C3
:1065B0009927AA27BB27DC0199278827278133271A
:1065C00044275527822B932BA42BB52B682A792A95
:1065D0008A2A9B2ADFC1F70180859927982F88276F
:1065E00027813327822B932B3C01882477FC8094CE
:1065F000982CD0C1FB0180859927582E442487818F
:106600009927482A592AD7C1FB0180859927582EF6
:10661000442487819927482A592A82859927982FC7
:10662000882721853327822B932B3C01882477FCF4
:106630008094982CC3C1F7018781682E7724882421
:106640009924A8C14FEF5FEF6CE074E1C5010E948F
:10665000192F9C01FC010085118584819581A681FB
:10666000B781893F9105A105B10544F088EF90E01D
:10667000A0E0B0E084839583A683B7836624772463
:1066800010C0492C5524D201AE0DBF1DFD018781DC
:10669000400E511ED2018C930894611C711C8823FA
:1066A00079F0962C462D552766277727F9018481A6
:1066B0009581A681B781481759076A077B070CF3B4
:1066C000F90184819581A681B781481759076A0726
:1066D0007B0709F49A94090D111DD8011C9257C12A
:1066E000B3E0CB16D10409F44AC0E4E0CE16D104DD
:1066F00030F4F1E0CF16D10409F049C10BC035E008
:10670000C316D10409F452C089E0C816D10409F0B7
:106710003EC185C04FEF5FEF60E171E0C5010E94AF
:10672000192FFC01A085B185F70187818C93208505
:10673000332781859927982F8827282B392BFD010E
:1067400032832183F7018285FD018383F70123854D
:10675000332784859927982F8827282B392BFD01EB
:1067600035832483F7012585332786859927982F3C
:106770008827282B392BFD013783268308C14FEF4B
:106780005FEF60E173E0C5010E94192FFC014085B5
:106790005185D70114969A01285F3F4F8D91FA01D8
:1067A0008193AF01E217F307C9F7F1C083E292E0EA
:1067B000A80EB91EFB0180859927982F882727816D
:1067C0003327822B932BD5018D939C93EFE1F0E03F
:1067D000AE0EBF1EF7018185D5018C93EEEBFDEF68
:1067E000AE0EBF1EF70163857727762F6627828559
:1067F0009927682B792BC501815E9D4F0E949F517F
:10680000F70165857727762F662784859927682B7A
:10681000792BC501825C9D4F0E949F51B8C04FEFFC
:106820005FEF60E179E0C5010E94192FFC0140850E
:106830005185D70117969A012A5F3F4F8D91FA0132
:106840008193AF01E217F307C9F7A1C0F5E0CF16B6
:10685000D10419F137E0C316D10409F440C083E034
:10686000C816D10409F0ACC0FB0180859927582EC9
:10687000442487819927482A592AB201C5010E94D8
:10688000582FAC0164E173E0C5010E94192FFC018F
:10689000A085B185F70181858DC0FB018085992791
:1068A000582E442487819927482A592AB201C501C4
:1068B0000E94582FAC0164E175E0C5010E94192FB8
:1068C000FC01A085B185F70182859927982F88273B
:1068D00021853327822B932B8D939C936CC04FEF94
:1068E0005FEF64E177E0C5010E94192FFC01A085EC
:1068F000B185109729F0F701858599278D939C9391
:10690000F70182859927AA27BB276624782E892E2E
:106910009A2E2485332744275527522F442733277F
:10692000222783859927AA27BB27DC019927882757
:10693000282B392B4A2B5B2B81859927AA27BB272C
:10694000282B392B4A2B5B2B622A732A842A952AFF
:1069500062E0660C771C881C991C6A95D1F71AC0F6
:10696000F2E1CF16D10499F4F501E45BFD4F20E08C
:10697000008111810115110531F0D8018D919C9193
:106980008C5F924159F02F5F3296203189F766244F
:10699000772443015FEF452E552E10C0F801628128
:1069A0007381C5010E94792F2C01F801A085B18562
:1069B000F70187818C9366247724430111E007C097
:1069C0006624772443014FEF442E542E10E0F70144
:1069D0008681882349F09927909581959F4F3C01A6
:1069E000882477FC8094982CFFEF4F16FFEF5F060A
:1069F00019F44FEF5FEF05C0B201C5010E94582F97
:106A0000AC011123C9F07C2D6627832D9927880FAF
:106A1000991F880F991F682B792B94018301C50159
:106A20000E94B93009C08FEF482E582EF701868199
:106A300011E0D1CF11E0D8CFF70163817727C501ED
:106A400009960E949F5126960FB6F894DEBF0FBE9E
:106A5000CDBFDF91CF911F910F91FF90EF90DF900D
:106A6000CF90BF90AF909F908F907F906F905F90EE
:106A70004F903F9008952F923F924F925F926F9266
:106A80007F928F929F92AF92BF92CF92DF92EF92BE
:106A9000FF920F931F93CF93DF93CDB7DEB72A9763
:106AA0000FB6F894DEBF0FBECDBF6C014B01FB01EA
:106AB0008181833109F459C0843128F5853009F486
:106AC00027C3863078F4823009F489C0833020F4FB
:106AD000813009F040C057C0833009F4AEC1843022
:106AE000D1F57EC28F3009F4FBC3803130F487309A
:106AF00009F48AC38E3079F5EFC3803109F4DEC51D
:106B0000823149F536C08B3109F4D8C58C3170F427
:106B1000863109F41CC5873118F48431E1F41FC0B3
:106B2000873109F424C58831B1F4C8C5823209F42B
:106B300056C0833230F48C3109F429C58D3159F4B3
:106B40004CC58F3E19F08F3F31F419C08B0181E0A5
:106B5000E82EF12C8BC58401EE24FF2498C5D601C4
:106B6000A558BD4F60E070E086C48B01EE24FF2481
:106B70007BC4D601A358BD4F20E030E0B5C38B01E4
:106B8000EE24FF2462C5FB010381002379F0112765
:106B9000109501951F4F222717FD2095322F4FEF9B
:106BA0005FEF64E071E0C6010E94B9304FEF5FEF24
:106BB00064E071E0C6010E94192FFC010481158177
:106BC000268137814FEF5FEF64E071E0C6010E94DC
:106BD000B930C601885B9D4F0E94AC516FC54FEF25
:106BE0005FEF64E071E0C6010E94192F8C01FC0187
:106BF000E084F184B401AA24BB2418861F82B1E189
:106C00002B2E312C280C391C02C1F801848195816E
:106C10008A0D9B1D2FE030E0829FD001839FB00D35
:106C2000929FB00D1124EF81F885E80DF91DAE0D8E
:106C3000BF1D349686E001900D928150E1F7F80176
:106C4000848195818A0D9B1DAFE06A2E712C869DF3
:106C5000D001879DB00D969DB00D1124AE0DBF1DC6
:106C6000FB0192859F70FD018681807F892B868341
:106C7000F801848195818A0D9B1D869DD001879D99
:106C8000B00D969DB00D1124AE0DBF1DFB01938577
:106C90009295907FFD0186818F70892B8683F40108
:106CA0008181F80144815581FB01958556848232AA
:106CB00009F052C04A0D5B1D469D9001479D300D65
:106CC000569D300D11242E0D3F1D3A8729872485AE
:106CD000332744275527892F9927AA27BB27BA2F5F
:106CE000A92F982F8827282B392B4A2B5B2B852DF2
:106CF0009927AA27BB27DC0199278827282B392B1E
:106D00004A2B5B2BE985FA85278330874187528799
:106D1000F801848195818A0D9B1D869DD001879DF8
:106D2000B00D969DB00D1124AE0DBF1DFB01208945
:106D30003327322F2227878599279068282B392BD4
:106D4000FD0134872387F1018081992787FD909584
:106D5000FD01968785874CC04A0D5B1D469D9001BD
:106D6000479D300D569D300D11242E0D3F1D3A8745
:106D70002987292F332744275527852D9927AA2787
:106D8000BB27BA2FA92F982F8827282B392B4A2BBE
:106D90005B2BFB0187859927AA27BB27DC01992755
:106DA0008827282B392B4A2B5B2BE985FA852783EB
:106DB000308741875287F801848195818A0D9B1D18
:106DC000869DD001879DB00D969DB00D1124AE0D0E
:106DD000BF1DFB0121893327322F22278089992764
:106DE0009068282B392BFD0134872387168615865A
:106DF0000894A11CB11C2F813885225F3F4F388732
:106E00002F838EE090E0280E391E625F7F4FF401E1
:106E10002381822F9927A816B9060CF4F6CEF80123
:106E200084819581A681B781820F911DA11DB11D1D
:106E300084839583A683B78341C48B010A5F1F4F68
:106E4000DE011196F80186E001900D928150E1F784
:106E5000A9817A816B815C814D819E81F601E35825
:106E6000FD4F20E030E08585882391F080818A17EE
:106E700079F48181871761F48281861749F48381CF
:106E8000851731F48481841719F48581891739F0C5
:106E90002F5F3F4F77962A30310529F701C487E1EC
:106EA00090E0289FD001299FB00D389FB00D11248C
:106EB000A758BD4FAC0DBD1DED90FC90119734C08F
:106EC000C6010E94342F9C0197FDF8C387E190E032
:106ED000289FD001299FB00D389FB00D1124A758CD
:106EE000BD4FAC0DBD1DCD010496A80126E0FA01F1
:106EF0000190AF01FC010192CF012150C1F784E064
:106F0000FD01818B8091FC089091FD0811969C9366
:106F10008E9301969093FD088093FC080197208939
:106F20002F7C2061208B7C01FD017189872F83508C
:106F3000F4019381823008F045C0992361F0FD018E
:106F4000118A8FEF9FEF8D939C9393838283F4013B
:106F50008381992739C085E0FD01818BF40124816B
:106F6000332785819927982F8827282B392BFD01D6
:106F700033832283F40194859F70FD018089807F93
:106F8000892B808B128A86010B581D4F27E732E030
:106F9000C20ED31EF6012081318189E89DEFC80E13
:106FA000D91E4D915C9160E0733009F461E081E09D
:106FB0006827D801ED91FC9182E00995870122278D
:106FC00033270AC0892F9927909581959F4F8C016F
:106FD000222717FD2095322FA70164E075E004C138
:106FE000E2E6F3E0CE0EDF1ED6018D919C91EEE934
:106FF000FCEFCE0EDF1E892B09F460C38B010D5F01
:107000001F4FDE011196F80186E001900D9281502C
:10701000E1F7F401E184F284B384C6010E94342FC5
:10702000AC018F5F9F4F09F449C387E190E0489F0F
:10703000D001499FB00D589FB00D1124A358BD4FEA
:10704000AC0DBD1DC80126E0FC010190CF010D92E1
:107050002150D1F787E190E0489F3001499F700CA3
:10706000589F700C11246C0C7D1C25E832E0620ED8
:10707000731E2E2D3327442755278F2D9927AA2796
:10708000BB27BA2FA92F982F8827282B392B4A2BBB
:107090005B2B8B2D9927AA27BB27DC0199278827F3
:1070A000282B392B4A2B5B2BD3012D933D934D93EA
:1070B0005C931397EBE7FDEF6E0E7F1ED301A7578E
:1070C000BD4FF40194859F708C91807F892B8C93A8
:1070D0008091FC089091FD0829E732E0620E731E52
:1070E000F3019183808301969093FD088093FC08BF
:1070F00021E130E0620E731E82E0F30181938C91F6
:107100008F7C80618C931082F601EF58FD4F2BC26B
:10711000FB0185819927582F442784819927482B83
:10712000592BD601A558BD4F60E070E0E9E7AE2EBF
:10713000E2E0BE2EAC0CBD1C9501FD0187858823C5
:1071400071F08D919C9111978417950741F4D901A5
:10715000ED90FC90F4010381002371F049C06F5F52
:107160007F4F87E190E0A80EB91E295E3F4F5796EA
:107170006A30710511F7A2C2F501118A8FEF9FEFF6
:10718000938382839183808380898F7C808BF601B7
:10719000EB58FD4F27E732E0C20ED31ED6012D91EA
:1071A0003C9189E89DEFC80ED91EA081B181A7014D
:1071B000F401668183E0FD010995F4010381112743
:1071C000109501951F4F222717FD2095322FA701FB
:1071D00064E076E0C6010E94B93006EF1EEF2FEFA3
:1071E0003FEFA7016FEF7FEFC6010E94B93066C283
:1071F0001127109501951F4F222717FD2095322F3B
:10720000A70164E076E0F0CF4FEF5FEF64E079E153
:10721000C6010E94192F7C01FC01408451848481A5
:107220009581A681B781893F9105A105B10544F0FB
:1072300088EF90E0A0E0B0E084839583A683B783D5
:10724000540100E010E020E030E011C0F50182853B
:10725000F201E40FF51F80838A019B010F5F1F4F2E
:107260002F4F3F4F0894A11CB11C882369F03801AF
:10727000B901A801F70184819581A681B7814817DA
:1072800059076A077B0714F3F70184819581A6816A
:10729000B781481759076A077B0719F408946108F2
:1072A0007108460C571CD2011C92F4010381002383
:1072B00049F01127109501951F4F222717FD2095A2
:1072C000322F05C08301222717FD2095322F4FEF63
:1072D0005FEF64E079E188CFC6010E948631EEC19C
:1072E000C6010E946331EAC1A4014D5F5F4F9C91CA
:1072F000FA0181819817F1F4FD019181FA018281EF
:107300009817C1F4FD019281FA018381981791F4D5
:10731000FD019381FA018481981761F4FD01948144
:10732000FA018581981731F4FD019581FA01868172
:10733000981739F02F5F3F4F57962A303105A1F645
:10734000BDC187E190E0289F7001299FF00C389F14
:10735000F00C1124EC0CFD1C29E732E0E20EF31EC8
:10736000D701AD90BC90E7E8FDEFEE0EFF1EF401F3
:107370000381002351F01127109501951F4F2227FB
:1073800017FD2095322FA501ABC0D701A757BD4FE0
:10739000F401928593709295907F8C918F7C892BCC
:1073A0008C930285112722273327A50168E07BE013
:1073B000C6010E94B9302AE832E0E20EF31ED7017E
:1073C0008C91853009F07AC1F601EB58FD4F27E723
:1073D00032E0C20ED31ED6012D913C9189E89DEF7B
:1073E000C80ED91EA081B181A50160E0F40182859B
:1073F000FD01099563C1F80167817727762F66271C
:1074000086819927682B792BC601815E9D4F0E944A
:107410009051F80185819927382F22278481992757
:10742000282B392BD601A558BD4F40E050E0B601BE
:1074300062577D4F8D919C9111978217930739F474
:10744000F8019681DB018C91891B8C9308C04F5FFA
:107450005F4F695E7F4F57964A30510559F7089440
:10746000E11CF11C0C5F1F4FF40183819927E81682
:10747000F9060CF223C18D919C9111975796F40156
:1074800025813327322F222744815527242B352B62
:107490003F708217930731F06F5F7F4F6A3071053D
:1074A00051F70CC187E190E0689FD001699FB00D52
:1074B000789FB00D1124AC0DBD1DA758BD4F4D9147
:1074C0005C911197A957B240F4010381002359F050
:1074D0001127109501951F4F222717FD2095322F58
:1074E00068E07BE081CEA557BD4FF40186818D9386
:1074F0008681882359F080859927982F88272781AE
:107500003327822B932B8D939C9302C01D921C9248
:1075100087E190E0689FF001699FF00D789FF00D82
:107520001124EC0DFD1DE457FD4F00811181222730
:107530003327322F212F102F0027F401868199271E
:10754000AA27BB27082B192B2A2B3B2B4BCEDE015E
:107550001196FB01339686E001900D928150E1F780
:10756000F601EE58FD4F80818F5F8083A7C0DE015A
:107570001196FB01339686E001900D928150E1F760
:10758000BE016F5F7F4FC6010E947E4897C0FB011E
:1075900065817727762F662784819927682B792B39
:1075A000C6010E94582FAC01F4010381002329F089
:1075B0001127109501951F4F09C0F401078111276C
:1075C000102F002786819927082B192B222717FDBA
:1075D0002095322F64E07FE107CEFB01658177279C
:1075E000762F662784819927682B792BC6010E9404
:1075F000582FAC01F4010381002329F011271095C5
:1076000001951F4F09C0F40107811127102F002792
:1076100086819927082B192B222717FD2095322FB9
:1076200064E07FE0E1CDF801828199279F938F93F9
:1076300088E595E09F938F930E94E3180894E11CDE
:10764000F11C0F900F900F900F900F5F1F4FF401E0
:1076500082819927E816F90634F330C0F801838156
:1076600099270E94FD7B0894E11CF11C0F5F1F4FBE
:10767000F40182819927E816F90684F31FC0F80106
:10768000828199270E94FD7B0894E11CF11C0F5F09
:107690001F4FF40182819927E816F90684F30EC082
:1076A000E2E6F3E0CE0EDF1ED6018D919C91EEE96D
:1076B000FCEFCE0EDF1E892B09F402CC21E131E074
:1076C000C20ED31E8FEFD6018C932A960FB6F89474
:1076D000DEBF0FBECDBFDF91CF911F910F91FF9005
:1076E000EF90DF90CF90BF90AF909F908F907F9062
:1076F0006F905F904F903F902F9008958F929F9240
:10770000AF92BF92CF92DF92EF92FF920F931F93AF
:10771000CF93DF93CDB7DEB72C970FB6F894DEBFCB
:107720000FBECDBF6C014B01142F9CE6A92E93E038
:10773000B92EAC0CBD1C96012F5E3F4F83E4E82EA2
:10774000F12C03E0AB01BE016F5F7F4FC6010E94C9
:10775000962F7C01F50180899189892B39F481E08C
:1077600090E00E942808F501918B808BF501A0899B
:10777000B1891C9381E0F601848B158B0FEF1FEF0D
:107780002CE033E4A401B701C6010E94EA2F2C9635
:107790000FB6F894DEBF0FBECDBFDF91CF911F9122
:1077A0000F91FF90EF90DF90CF90BF90AF909F90A0
:1077B0008F900895AF92BF92CF92DF92EF92FF9297
:1077C0000F931F93CF93DF93CDB7DEB72C970FB6F0
:1077D000F894DEBF0FBECDBF6C015B019C012F5E34
:1077E0003F4F42E4E42EF12C03E0AB01BE016F5F9A
:1077F0007F4F0E94962FF601148A0FEF1FEF2CE0A7
:1078000032E4A501BC01C6010E94EA2F2C960FB6F6
:10781000F894DEBF0FBECDBFDF91CF911F910F91C6
:10782000FF90EF90DF90CF90BF90AF9008958F9230
:107830009F92AF92BF92CF92DF92EF92FF920F93FF
:107840001F93CF93DF93CDB7DEB72C970FB6F89485
:10785000DEBF0FBECDBF6C014B01142F6CE6A62E10
:1078600063E0B62EA80EB91E9C012F5E3F4F55E473
:10787000E52EF12C03E0A401BE016F5F7F4F0E9453
:10788000962F7C01F50186859785892B39F481E057
:1078900090E00E942808F50197878687F501A68564
:1078A000B7851C9381E0F601848B158B0FEF1FEFDA
:1078B0002CE035E4A401B701C6010E94EA2F2C9602
:1078C0000FB6F894DEBF0FBECDBFDF91CF911F91F1
:1078D0000F91FF90EF90DF90CF90BF90AF909F906F
:1078E0008F900895AF92BF92CF92DF92EF92FF9266
:1078F0000F931F93CF93DF93CDB7DEB72C970FB6BF
:10790000F894DEBF0FBECDBF6C015B019C012F5E02
:107910003F4F74E4E72EF12C03E0A501BE016F5F39
:107920007F4F0E94962FF601148A0FEF1FEF2CE075
:1079300034E4A501BC01C6010E94EA2F2C960FB6C3
:10794000F894DEBF0FBECDBFDF91CF911F910F9195
:10795000FF90EF90DF90CF90BF90AF9008952F925F
:107960003F924F925F926F927F928F929F92AF92CF
:10797000BF92CF92DF92EF92FF920F931F93CF931C
:10798000DF93CDB7DEB72D970FB6F894DEBF0FBEED
:10799000CDBF6C011B014A012D87380127018CE600
:1079A000A82E83E0B82EAC0CBD1C96012F5E3F4F75
:1079B00003E3E02EF12C03E0AB01BE016F5F7F4FCC
:1079C000C6010E94962F7C01F50184859585892B3F
:1079D00039F487E090E00E942808F50195878487B4
:1079E000F501A485B58511969C928E928D85FD0139
:1079F0008283F501A485B585FD0174826382568278
:107A0000458287E0F601848B858A892D9927868BAC
:107A10008D85878B608E872D9927818F428E852D4E
:107A20009927838F0FEF1FEF2CE033E3A101B701FC
:107A3000C6010E94EA2F2D960FB6F894DEBF0FBE46
:107A4000CDBFDF91CF911F910F91FF90EF90DF900D
:107A5000CF90BF90AF909F908F907F906F905F90EE
:107A60004F903F902F9008958F929F92AF92BF9228
:107A7000CF92DF92EF92FF920F931F93CF93DF93FA
:107A8000CDB7DEB72C970FB6F894DEBF0FBECDBFD3
:107A90006C014B01142F2CE6A22E23E0B22EA80E6F
:107AA000B91E9C012F5E3F4F91E3E92EF12C03E0BC
:107AB000AB01BE016F5F7F4FC6010E94962F7C0114
:107AC000F50182859385892B39F481E090E00E944D
:107AD0002808F50193878287F501A285B3851C9359
:107AE00081E0F601848B158B0FEF1FEF2CE031E363
:107AF000A401B701C6010E94EA2F2C960FB6F89494
:107B0000DEBF0FBECDBFDF91CF911F910F91FF90D0
:107B1000EF90DF90CF90BF90AF909F908F9008959F
:107B20004F925F926F927F928F929F92AF92BF928D
:107B3000CF92DF92EF92FF920F931F93CF93DF9339
:107B4000CDB7DEB72C970FB6F894DEBF0FBECDBF12
:107B50006C012B0149015A016CE6662E63E0762E1A
:107B6000680E791E9C012F5E3F4F54E2E52EF12CEA
:107B700003E0A201BE016F5F7F4F0E94962F7C0140
:107B8000F30182899389892B39F484E090E00E9483
:107B90002808F301938B828BF301A289B3898D921C
:107BA0009D92AD92BC92139783E0F601848B858AF7
:107BB000BB27AB2D9A2D892D868BC501AA27BB2704
:107BC000878B0FEF1FEF2CE034E2A201B701C60153
:107BD0000E94EA2F2C960FB6F894DEBF0FBECDBFE1
:107BE000DF91CF911F910F91FF90EF90DF90CF9099
:107BF000BF90AF909F908F907F906F905F904F90CD
:107C00000895AF92BF92CF92DF92EF92FF920F93BF
:107C10001F93CF93DF93CDB7DEB72C970FB6F894B1
:107C2000DEBF0FBECDBF6C015B019C012F5E3F4FDD
:107C300073E2E72EF12C03E0A501BE016F5F7F4FD9
:107C40000E94962FF601148A0FEF1FEF2CE033E20B
:107C5000A501BC01C6010E94EA2F2C960FB6F8942C
:107C6000DEBF0FBECDBFDF91CF911F910F91FF906F
:107C7000EF90DF90CF90BF90AF9008958F929F923A
:107C8000AF92BF92CF92DF92EF92FF920F931F932A
:107C9000CF93DF93CDB7DEB72C970FB6F894DEBF46
:107CA0000FBECDBF6C014B01142FFCE6AF2EF3E0ED
:107CB000BF2EA80EB91E9C012F5E3F4FEAE1EE2EAB
:107CC000F12C03E0AB01BE016F5F7F4F0E94962F46
:107CD0007C01F501828D938D892B39F481E090E050
:107CE0000E942808F501938F828FF501A28DB38D34
:107CF0001C9381E0F601848B158B0FEF1FEF2CE0B6
:107D00003AE1A401B701C6010E94EA2F2C960FB6F2
:107D1000F894DEBF0FBECDBFDF91CF911F910F91C1
:107D2000FF90EF90DF90CF90BF90AF909F908F909B
:107D30000895AF92BF92CF92DF92EF92FF920F938E
:107D40001F93CF93DF93CDB7DEB72C970FB6F89480
:107D5000DEBF0FBECDBF6C015B019C012F5E3F4FAC
:107D6000A9E1EA2EF12C03E0AB01BE016F5F7F4F6A
:107D70000E94962FF601148A0FEF1FEF2CE039E1D5
:107D8000A501BC01C6010E94EA2F2C960FB6F894FB
:107D9000DEBF0FBECDBFDF91CF911F910F91FF903E
:107DA000EF90DF90CF90BF90AF9008956F927F9249
:107DB0008F929F92AF92BF92CF92DF92EF92FF92FB
:107DC0000F931F93CF93DF93CDB7DEB72C970FB6EA
:107DD000F894DEBF0FBECDBF6C013B014A010CE63B
:107DE000A02E03E0B02EA80EB91E9C012F5E3F4FBF
:107DF00018E1E12EF12C03E0AB01BE016F5F7F4F74
:107E00000E94962F7C01F50186899789892B39F488
:107E100082E090E00E942808F501978B868BF5019F
:107E2000A689B7898D929C9282E0F601848B858A1F
:107E3000892D9927868B0FEF1FEF2CE038E1A301E6
:107E4000B701C6010E94EA2F2C960FB6F894DEBF48
:107E50000FBECDBFDF91CF911F910F91FF90EF909B
:107E6000DF90CF90BF90AF909F908F907F906F905A
:107E70000895AF92BF92CF92DF92EF92FF920F934D
:107E80001F93CF93DF93CDB7DEB72C970FB6F8943F
:107E9000DEBF0FBECDBF6C015B019C012F5E3F4F6B
:107EA00087E1E82EF12C03E0AB01BE016F5F7F4F4D
:107EB000C6010E94962FF601148A0FEF1FEF2CE0E7
:107EC00037E1A501BC01C6010E94EA2F2C960FB62E
:107ED000F894DEBF0FBECDBFDF91CF911F910F9100
:107EE000FF90EF90DF90CF90BF90AF9008956F928A
:107EF0007F928F929F92AF92BF92CF92DF92EF923A
:107F0000FF920F931F93CF93DF93CDB7DEB72C97DC
:107F10000FB6F894DEBF0FBECDBF6C013B014A0126
:107F20005CE6A52E53E0B52EA80EB91E9C012F5E6F
:107F30003F4F46E1E42EF12C03E0AB01BE016F5F41
:107F40007F4F0E94962F7C01F50182819381892BBE
:107F500039F482E090E00E942808F501938382833F
:107F6000F501A281B3818D929C9282E0F601848B0F
:107F7000858A892D9927868B0FEF1FEF2CE036E13C
:107F8000A301B701C6010E94EA2F2C960FB6F89400
:107F9000DEBF0FBECDBFDF91CF911F910F91FF903C
:107FA000EF90DF90CF90BF90AF909F908F907F9099
:107FB0006F900895AF92BF92CF92DF92EF92FF92AF
:107FC0000F931F93CF93DF93CDB7DEB72C970FB6E8
:107FD000F894DEBF0FBECDBF6C015B019C012F5E2C
:107FE0003F4F65E1E62EF12C03E0A501BE016F5F76
:107FF0007F4F0E94962FF601148A0FEF1FEF2CE09F
:1080000035E1A501BC01C6010E94EA2F2C960FB6EE
:10801000F894DEBF0FBECDBFDF91CF911F910F91BE
:10802000FF90EF90DF90CF90BF90AF9008954F9268
:108030005F926F927F928F929F92AF92BF92CF92F8
:10804000DF92EF92FF920F931F93CF93DF93CDB701
:10805000DEB72C970FB6F894DEBF0FBECDBF4C0134
:108060002B013A01A22E9C012F5E3F4F74E1E72EB7
:10807000F12C03E0A201BE016F5F7F4F0E94962F9B
:10808000FC0171866086BB24CC24DD24A482B582E9
:10809000C682D782F401148A0FEF1FEF2CE034E17F
:1080A000A201BC01C4010E94EA2F2C960FB6F894DD
:1080B000DEBF0FBECDBFDF91CF911F910F91FF901B
:1080C000EF90DF90CF90BF90AF909F908F907F9078
:1080D0006F905F904F9008958F929F92AF92BF9252
:1080E000CF92DF92EF92FF920F931F93CF93DF9384
:1080F000CDB7DEB72C970FB6F894DEBF0FBECDBF5D
:108100006C014B01142FFCE6AF2EF3E0BF2EA80E3E
:10811000B91E9C012F5E3F4FEAE0EE2EF12C03E0EA
:10812000AB01BE016F5F7F4F0E94962F7C01F5016E
:10813000808D918D892B39F481E090E00E94280890
:10814000F501918F808FF501A08DB18D1C9381E099
:10815000F601848B158B0FEF1FEF2CE03AE0A401A2
:10816000B701C6010E94EA2F2C960FB6F894DEBF25
:108170000FBECDBFDF91CF911F910F91FF90EF9078
:10818000DF90CF90BF90AF909F908F900895AF9267
:10819000BF92CF92DF92EF92FF920F931F93CF93F4
:1081A000DF93CDB7DEB72C970FB6F894DEBF0FBEC6
:1081B000CDBF6C015B019C012F5E3F4FA9E0EA2E11
:1081C000F12C03E0AB01BE016F5F7F4F0E94962F41
:1081D000F601148A0FEF1FEF2CE039E0A501BC0176
:1081E000C6010E94EA2F2C960FB6F894DEBF0FBE90
:1081F000CDBFDF91CF911F910F91FF90EF90DF9056
:10820000CF90BF90AF900895AF92BF92CF92DF9280
:10821000EF92FF920F931F93CF93DF93CDB7DEB70B
:108220002C970FB6F894DEBF0FBECDBF6C015B017B
:10823000FC01EB5BFD4F8081882329F06BEF7EEF23
:108240008FEF9FEF1BC081E0808396012F5E3F4F31
:10825000B3E0EB2EF12C03E0AB01BE016F5F7F4F6B
:10826000C6010E94962FF601148A0FEF1FEF2CE033
:1082700033E0A501BC01C6010E94EA2F2C960FB67F
:10828000F894DEBF0FBECDBFDF91CF911F910F914C
:10829000FF90EF90DF90CF90BF90AF9008952F9216
:1082A0003F924F925F926F927F928F929F92AF9286
:1082B000BF92CF92DF92EF92FF920F931F93CF93D3
:1082C000DF93CDB7DEB72E970FB6F894DEBF0FBEA3
:1082D000CDBF6C017E876D8729013A0147015801A6
:1082E0005CE6252E53E0352E280E391E9C012F5EAC
:1082F0003F4F41E0E42EF12C03E0AB01BE016F5F84
:108300007F4F0E94962F7C01F10180859185892BFA
:1083100039F488E090E00E942808F1019187808775
:10832000F101A085B1854D925D926D927C9213977B
:10833000FD0184829582A682B78288E0F601848B53
:10834000858ABB27AB2D9A2D892D868BC501AA273F
:10835000BB27878B8B2D9927AA27BB27808F418E20
:10836000BB27A72D962D852D828FC301AA27BB275A
:10837000838F872D9927AA27BB27848F0FEF1FEFA5
:108380002CE031E04D855E85B701C6010E94EA2FE1
:108390002E960FB6F894DEBF0FBECDBFDF91CF9102
:1083A0001F910F91FF90EF90DF90CF90BF90AF9013
:1083B0009F908F907F906F905F904F903F902F9005
:1083C00008954F925F926F927F928F929F92AF9299
:1083D000BF92CF92DF92EF92FF920F931F93CF93B2
:1083E000DF93CDB7DEB72C970FB6F894DEBF0FBE84
:1083F000CDBF6C012B013A014901BA010E94792FCE
:108400005C018FEFA8168FEFB80629F46DEF7EEFB1
:108410008FEF9FEF21C096012F5E3F4FE7E3EE2ED7
:10842000F12C03E0A201BE016F5F7F4FC6010E94E5
:10843000962F24E0F601248BA58A2B2D3327268B3B
:10844000878A292D3327208F83012CE037E3A2016F
:10845000BC01C6010E94EA2F2C960FB6F894DEBF2D
:108460000FBECDBFDF91CF911F910F91FF90EF9085
:10847000DF90CF90BF90AF909F908F907F906F9044
:108480005F904F9008956F927F928F929F92AF92DC
:10849000BF92CF92DF92EF92FF920F931F93CF93F1
:1084A000DF93CDB7DEB72C970FB6F894DEBF0FBEC3
:1084B000CDBF6C013B014A01BA010E94792F5C01DA
:1084C0008FEFA8168FEFB80629F46DEF7EEF8FEFD0
:1084D0009FEF1DC096012F5E3F4FB6E3EB2EF12CB0
:1084E00003E0A301BE016F5F7F4FC6010E94962F7C
:1084F00022E0F601248BA58A2B2D3327268B8401BD
:108500002CE036E3A301BC01C6010E94EA2F2C96A1
:108510000FB6F894DEBF0FBECDBFDF91CF911F9194
:108520000F91FF90EF90DF90CF90BF90AF909F9012
:108530008F907F906F9008956F927F928F929F920D
:10854000AF92BF92CF92DF92EF92FF920F931F9361
:10855000CF93DF93CDB7DEB72C970FB6F894DEBF7D
:108560000FBECDBF6C013B014A010E94792F5C0117
:108570008FEFA8168FEFB80629F46DEF7EEF8FEF1F
:108580009FEF26C096012F5E3F4F85E3E82EF12C2A
:1085900003E040E050E0BE016F5F7F4FC6010E94E4
:1085A000962F85E0F601848B81E0858BA68A8B2D42
:1085B0009927878B808E892D9927818F83012CE0C5
:1085C00035E340E050E060E070E0C6010E94EA2F31
:1085D0002C960FB6F894DEBF0FBECDBFDF91CF91C2
:1085E0001F910F91FF90EF90DF90CF90BF90AF90D1
:1085F0009F908F907F906F9008956F927F928F924F
:108600009F92AF92BF92CF92DF92EF92FF920F9321
:108610001F93CF93DF93CDB7DEB72C970FB6F894A7
:10862000DEBF0FBECDBF6C013B015A012CE6822E8E
:1086300023E0922E880E991E9C012F5E3F4F93E1FE
:10864000E92EF12C03E0AB01BE016F5F7F4FC60145
:108650000E94962F7C01F40184899589892B59F415
:1086600089EF90E00E942808DC01F401958B848B4F
:10867000A850BF4F1C92F50101900020E9F73197F7
:10868000EA19FB09E83FF10518F049EF50E003C093
:10869000AF014F5F5F4FB501F401848995890E9456
:1086A000988488EFF601848BF50120E030E0D60154
:1086B0005596922F80818D938081882351F09F5F02
:1086C0002F5F3F4F3196283F310599F7983F09F4C6
:1086D00097EFF601E90FF11D158A0FEF1FEF2CE060
:1086E00033E1A301B701C6010E94EA2F2C960FB611
:1086F000F894DEBF0FBECDBFDF91CF911F910F91D8
:10870000FF90EF90DF90CF90BF90AF909F908F90B1
:108710007F906F9008958F929F92AF92BF92CF9269
:10872000DF92EF92FF920F931F93CF93DF93CDB71A
:10873000DEB72C970FB6F894DEBF0FBECDBF6C012D
:108740004B015A019C012F5E3F4F45E0E42EF12C76
:1087500003E0AB01BE016F5F7F4F0E94962F7C014B
:10876000F501408155274F5F5F4FB501C601449623
:108770000E9498840FEF1FEF2CE035E0A401B701B1
:10878000C6010E94EA2F2C960FB6F894DEBF0FBEEA
:10879000CDBFDF91CF911F910F91FF90EF90DF90B0
:1087A000CF90BF90AF909F908F900895AF92BF925F
:1087B000DF92EF92FF920F931F93CF93DF93CDB78A
:1087C000DEB722970FB6F894DEBF0FBECDBFAE84E2
:1087D000BF84DA88BCE6EB2EB3E0FB2EEA0CFB1C70
:1087E000CE0143969A838983F70186819781892BED
:1087F00039F48CE090E00E942808F7019783868383
:10880000F70186819781DC011196FC01D182BD01BF
:108810006F5F7F4FF7012681378181E0F901808307
:108820008D2D8150823008F069C0E981FA8132963D
:10883000FA83E98332978081FD0181836F5F7F4FE7
:10884000813079F0813040F0823009F443C06EEE1F
:108850007FEF8FEF9FEF6CC0F701A681B78182E0B9
:108860004CC0E981FA813496FA83E98352914291AE
:1088700032912291FB0121938F01BB27A52F942FC9
:10888000832FFB018183B8016F5F7F4F9A014427DB
:108890005527F80121838B010F5F1F4FE981FA8172
:1088A0003496FA83E983B291A29192918291FB016D
:1088B0008183B8016F5F7F4F292F3A2F4B2F5527A8
:1088C000F8012183CD01AA27BB27FB0181836E5FBD
:1088D0007F4F0FC0E981FA813296FA83E983CB0199
:1088E000B291A29126E00D90FC010192CF0121509E
:1088F000D1F7F701A681B78188E08C93F2E0DF160B
:1089000079F4E981FA813296FA83E983329780819A
:10891000FB018083F701A681B7818C918F5F8C93D7
:10892000F7014681578168897989C5010E948B4387
:1089300022960FB6F894DEBF0FBECDBFDF91CF9168
:108940001F910F91FF90EF90DF90BF90AF9008952F
:108950008F929F92AF92BF92CF92DF92EF92FF924F
:108960000F931F93CF93DF93CDB7DEB72C970FB63E
:10897000F894DEBF0FBECDBF6C015B014A019C01C4
:108980002F5E3F4F89E0E82EF12C04E0AB01BE01E1
:108990006F5F7F4FC6010E94962FFC0191868086F3
:1089A000F601148A0FEF1FEF20E139E0A501BC01A9
:1089B000C6010E94EA2F2C960FB6F894DEBF0FBEB8
:1089C000CDBFDF91CF911F910F91FF90EF90DF907E
:1089D000CF90BF90AF909F908F900895AF92BF922D
:1089E000CF92DF92EF92FF920F931F93CF93DF937B
:1089F000CDB7DEB72C970FB6F894DEBF0FBECDBF54
:108A00006C015B019C012F5E3F4F95E0E92EF12C3C
:108A100004E0AB01BE016F5F7F4FC6010E94962F3D
:108A2000F601148A0FEF1FEF20E135E0A501BC012C
:108A3000C6010E94EA2F2C960FB6F894DEBF0FBE37
:108A4000CDBFDF91CF911F910F91FF90EF90DF90FD
:108A5000CF90BF90AF900895AF92BF92CF92DF9228
:108A6000EF92FF920F931F93CF93DF93CDB7DEB7B3
:108A70002C970FB6F894DEBF0FBECDBF6C015B0123
:108A80009C012F5E3F4F44E0E42EF12C04E0AB014B
:108A9000BE016F5F7F4F0E94962FF601148A0FEF81
:108AA0001FEF20E134E0A501BC01C6010E94EA2FBE
:108AB0002C960FB6F894DEBF0FBECDBFDF91CF91DD
:108AC0001F910F91FF90EF90DF90CF90BF90AF90EC
:108AD00008958F929F92AF92BF92CF92DF92EF92C2
:108AE000FF920F931F93CF93DF93CDB7DEB72C97F1
:108AF0000FB6F894DEBF0FBECDBF6C015B014A011B
:108B00009C012F5E3F4F53E0E52EF12C04E0AB01BA
:108B1000BE016F5F7F4F0E94962FFC019186808679
:108B2000F601148A0FEF1FEF20E133E0A501BC012D
:108B3000C6010E94EA2F2C960FB6F894DEBF0FBE36
:108B4000CDBFDF91CF911F910F91FF90EF90DF90FC
:108B5000CF90BF90AF909F908F900895AF92BF92AB
:108B6000CF92DF92EF92FF920F931F93CF93DF93F9
:108B7000CDB7DEB72C970FB6F894DEBF0FBECDBFD2
:108B80006C015B019C012F5E3F4F62E0E62EF12CF1
:108B900004E0A501BE016F5F7F4F0E94962FF60192
:108BA000148A0FEF1FEF20E132E0A501BC01C601DE
:108BB0000E94EA2F2C960FB6F894DEBF0FBECDBFF1
:108BC000DF91CF911F910F91FF90EF90DF90CF90A9
:108BD000BF90AF9008958F929F92AF92BF92CF9225
:108BE000DF92EF92FF920F931F93CF93DF93CDB756
:108BF000DEB72C970FB6F894DEBF0FBECDBF6C0169
:108C00004B015A019C012F5E3F4F71E0E72EF12C82
:108C100004E0A401BE016F5F7F4F0E94962FFC010C
:108C2000B186A0861482158216821782F601148AF4
:108C30000FEF1FEF20E131E0A401BC01C6010E944B
:108C4000EA2F2C960FB6F894DEBF0FBECDBFDF9192
:108C5000CF911F910F91FF90EF90DF90CF90BF9039
:108C6000AF909F908F9008956F927F928F929F9276
:108C7000AF92BF92CF92DF92EF92FF920F931F932A
:108C8000CF93DF93CDB7DEB72C970FB6F894DEBF46
:108C90000FBECDBF6C014B013A01BA010E94792F82
:108CA0005C018FEFA8168FEFB80629F46DEF7EEF09
:108CB0008FEF9FEF1EC096012F5E3F4F4FE1E42ED6
:108CC000F12C01E0A401BE016F5F7F4FC6010E943D
:108CD000962F22E0F601248BA58A2B2D3327268B95
:108CE000830124E03FE140E050E0BC01C6010E9466
:108CF000EA2F2C960FB6F894DEBF0FBECDBFDF91E2
:108D0000CF911F910F91FF90EF90DF90CF90BF9088
:108D1000AF909F908F907F906F9008950F931F93C7
:108D20008B0124E031E140E050E060E070E00E941F
:108D3000EA2F1F910F9108954F925F926F927F9249
:108D40008F929F92AF92BF92CF92DF92EF92FF925B
:108D50000F931F93CF93DF93CDB7DEB72C970FB64A
:108D6000F894DEBF0FBECDBF6C014B012A01390163
:108D7000BA010E94792F5C018FEFA8168FEFB80619
:108D800029F46DEF7EEF8FEF9FEF22C096012F5EEB
:108D90003F4F7FE0E72EF12C01E0A401BE016F5FA1
:108DA0007F4FC6010E94962F24E0F601248BA58AEE
:108DB0002B2D3327268B678A272D3327208F82017F
:108DC00024E03FE040E050E0BC01C6010E94EA2FF1
:108DD0002C960FB6F894DEBF0FBECDBFDF91CF91BA
:108DE0001F910F91FF90EF90DF90CF90BF90AF90C9
:108DF0009F908F907F906F905F904F9008956F92AB
:108E00007F928F929F92AF92BF92CF92DF92EF921A
:108E1000FF920F931F93CF93DF93CDB7DEB72C97BD
:108E20000FB6F894DEBF0FBECDBF6C013B014A0107
:108E3000122FBA010E94792F5C018FEFA8168FEFD5
:108E4000B80629F46DEF7EEF8FEF9FEF1EC09601FD
:108E50002F5E3F4FB6E0EB2EF12C01E0A301BE01E7
:108E60006F5F7F4FC6010E94962F23E0F601248B8F
:108E7000A58A2B2D3327268B178B840124E036E01F
:108E8000A301BC01C6010E94EA2F2C960FB6F894EC
:108E9000DEBF0FBECDBFDF91CF911F910F91FF902D
:108EA000EF90DF90CF90BF90AF909F908F907F908A
:108EB0006F900895AF92BF92CF92DF92EF92FF92A0
:108EC0000F931F93CF93DF93CDB7DEB72C970FB6D9
:108ED000F894DEBF0FBECDBF6C015B019C012F5E1D
:108EE0003F4F12E0E12EF12C01E0AB01BE016F5FBC
:108EF0007F4F0E94962FF601148A0FEF1FEF24E098
:108F000032E0A501BC01C6010E94EA2F2C960FB6E3
:108F1000F894DEBF0FBECDBFDF91CF911F910F91AF
:108F2000FF90EF90DF90CF90BF90AF9008952F9279
:108F30003F924F925F926F927F928F929F92AF92E9
:108F4000BF92CF92DF92EF92FF920F931F93CF9336
:108F5000DF93CDB7DEB72D970FB6F894DEBF0FBE07
:108F6000CDBF2C013B011A012D874801AE2C9C017D
:108F70002F5E3F4F89E1E82EF12C01E040E050E008
:108F8000BE016F5F7F4FC2010E94962FDC01FC0182
:108F900091868086BB24CC24DD24A482B582C6823F
:108FA000D7828AE0F201848BC2014596A30126E0B4
:108FB000FA010190AF01FC010192CF012150C1F7EC
:108FC0008D85F201838F148E258E832D9927868FB0
:108FD0000FEF1FEF24E039E140E050E0BD01C20196
:108FE0000E94EA2F2D960FB6F894DEBF0FBECDBFBC
:108FF000DF91CF911F910F91FF90EF90DF90CF9075
:10900000BF90AF909F908F907F906F905F904F90A8
:109010003F902F9008954F925F927F928F929F92F0
:10902000AF92BF92CF92DF92EF92FF920F931F9376
:10903000CF93DF93CDB7DEB72C970FB6F894DEBF92
:109040000FBECDBF6C012B014A01722E58019C014D
:109050002F5E3F4F9DE0E92EF12C01E040E050E013
:10906000BE016F5F7F4FC6010E94962F8C0187E182
:10907000F601848BD6015596F40186E001900D929D
:109080008150E1F7F601738EA501D60160E070E032
:10909000272D33270DC07A01FA018191AF01FD011F
:1090A000848F1196F7018081882329F06F5F7F4FAD
:1090B0006217730781F7F80191868086820124E0A8
:1090C0003DE040E050E060E070E0C6010E94EA2F21
:1090D0002C960FB6F894DEBF0FBECDBFDF91CF91B7
:1090E0001F910F91FF90EF90DF90CF90BF90AF90C6
:1090F0009F908F907F905F904F900895AF92BF9216
:10910000CF92DF92EF92FF920F931F93CF93DF9353
:10911000CDB7DEB72C970FB6F894DEBF0FBECDBF2C
:109120005C016B019C012F5E3F4F4CE0E42EF12C63
:1091300001E040E050E0BE016F5F7F4F0E94962F3C
:1091400086E0F501848BD5015596F60101900D92CC
:109150008150E1F70FEF1FEF24E03CE040E050E0EA
:1091600060E070E0C5010E94EA2F2C960FB6F894DB
:10917000DEBF0FBECDBFDF91CF911F910F91FF904A
:10918000EF90DF90CF90BF90AF9008956F927F9255
:109190008F929F92AF92BF92CF92DF92EF92FF9207
:1091A0000F931F93CF93DF93CDB7DEB72C970FB6F6
:1091B000F894DEBF0FBECDBF6C013B015A014901DF
:1091C0000E94792F8F5F9F4F29F46DEF7EEF8FEF15
:1091D0009FEF38C096012F5E3F4F5BE0E52EF12CEC
:1091E00001E040E050E0BE016F5F7F4FC6010E948A
:1091F000962F86E1F601848BD6015596F50186E01F
:1092000001900D928150E1F7A401D60120E030E0F9
:10921000FA018081FD01838FFA018081882341F06A
:109220002F5F3F4F4F5F5F4F11962F30310581F712
:10923000830124E03BE040E050E060E070E0C601E4
:109240000E94EA2F2C960FB6F894DEBF0FBECDBF5A
:10925000DF91CF911F910F91FF90EF90DF90CF9012
:10926000BF90AF909F908F907F906F900895AF9236
:10927000BF92CF92DF92EF92FF920F931F93CF9303
:10928000DF93CDB7DEB72C970FB6F894DEBF0FBED5
:10929000CDBF5C016B01142F9C012F5E3F4F69E035
:1092A000E62EF12C01E040E050E0BE016F5F7F4F01
:1092B0000E94962F87E0F501848BD5015596F60123
:1092C00086E001900D928150E1F7F501138F0FEFC9
:1092D0001FEF24E039E040E050E060E070E0C501BD
:1092E0000E94EA2F2C960FB6F894DEBF0FBECDBFBA
:1092F000DF91CF911F910F91FF90EF90DF90CF9072
:10930000BF90AF9008958F929F92AF92BF92CF92ED
:10931000DF92EF92FF920F931F93CF93DF93CDB71E
:10932000DEB72C970FB6F894DEBF0FBECDBF5C0141
:109330004B016A019C012F5E3F4F78E0E72EF12C34
:1093400001E0A401BE016F5F7F4F0E94962FBC0118
:1093500086E0F501848BD5015596F60101900D92BA
:109360008150E1F70FEF1FEF24E038E0A401C501C1
:109370000E94EA2F2C960FB6F894DEBF0FBECDBF29
:10938000DF91CF911F910F91FF90EF90DF90CF90E1
:10939000BF90AF909F908F9008952F923F924F92E1
:1093A0005F926F927F928F929F92AF92BF92CF9275
:1093B000DF92EF92FF920F931F93CF93DF93CDB77E
:1093C000DEB72D970FB6F894DEBF0FBECDBF5C01A0
:1093D0001B014A0139010D8727011C2DBA010E948A
:1093E000C8506D5F7E4F8F4F9F4F29F069EF7EEF22
:1093F0008FEF9FEFDBC0F4014081D501A358BD4F33
:1094000020E030E08C91841749F5FD019181F40151
:109410008181981719F5FD019281F40182819817D5
:10942000E9F4FD019381F40183819817B9F4FD01FA
:109430009481F4018481981789F4FD019581F401E8
:109440008581981759F4FD018585833009F4A5C0FD
:10945000823009F49DC0843009F49AC02F5F3F4FD9
:1094600057962A30310571F6D501A657BD4F40E019
:1094700050E020E030E0F501E757FD4F8C9185305A
:1094800039F4808182958F70837011F44F5F5F4F44
:109490002F5F3F4F779657962A30310579F747303F
:1094A00051050CF07FC0C5010E94342F6C018F5F05
:1094B0009F4F09F477C095012F5E3F4F05E0E02EE6
:1094C000F12C01E0A101BE016F5F7F4FC5010E9439
:1094D000962FBC018DE0F501848BD5015596F401E2
:1094E00086E001900D928150E1F7F501638E872DA2
:1094F0009927848F2D85258F168E478E852D992748
:1095000080A311A387E190E0C89EF001C99EF00DF1
:10951000D89EF00D1124E358FD4FEA0DFB1DD40138
:1095200086E00D9001928150E1F787E190E0C89EBE
:10953000F001C99EF00DD89EF00D1124EA0DFB1D1F
:10954000E657FD4F83E08083EA58F2408091FC08A3
:109550009091FD08DF01A758BD4F11969C938E9303
:1095600001969093FD088093FC08E757FD4F1295F4
:10957000110F110F107C80818F70812B80830D91D2
:109580001C9124E035E0A101C5010E94EA2F0EC024
:1095900067EF7EEF8FEF9FEF09C068EF7EEF8FEFF1
:1095A0009FEF04C06CEF7EEF8FEF9FEF2D960FB60D
:1095B000F894DEBF0FBECDBFDF91CF911F910F9109
:1095C000FF90EF90DF90CF90BF90AF909F908F90E3
:1095D0007F906F905F904F903F902F9008956F9283
:1095E0007F928F929F92AF92BF92CF92DF92EF9233
:1095F000FF920F931F93CF93DF93CDB7DEB72C97D6
:109600000FB6F894DEBF0FBECDBF4C013B01B42EA8
:10961000A22E68019C012F5E3F4F91E0E92EF12CB4
:1096200001E0AB01BE016F5F7F4FC4010E94962F26
:109630007C01C401885B9D4F0E94BA51F7011482DE
:10964000158216821782D186C08685E0F401848B4C
:1096500083E3858B8BE8868B8EE9878B8B2D81331B
:1096600008F080E3F401808FAA2011F481E0A82E95
:10967000F401A18E0FEF1FEF24E031E0A301B70149
:10968000C4010E94EA2F2C960FB6F894DEBF0FBEDD
:10969000CDBFDF91CF911F910F91FF90EF90DF90A1
:1096A000CF90BF90AF909F908F907F906F900895D4
:1096B0006F927F928F929F92AF92BF92CF92DF92E2
:1096C000EF92FF920F931F93CF93DF93CDB7DEB747
:1096D0002C970FB6F894DEBF0FBECDBF6C013B01D7
:1096E0004A01BA010E94792F5C018FEFA8168FEF13
:1096F000B80629F46DEF7EEF8FEF9FEF1DC0960146
:109700002F5E3F4F46E0E42EF12C02E0A301BE01A4
:109710006F5F7F4FC6010E94962F22E0F601248BD7
:10972000A58A2B2D3327268B840128E036E0A30160
:10973000BC01C6010E94EA2F2C960FB6F894DEBF3A
:109740000FBECDBFDF91CF911F910F91FF90EF9092
:10975000DF90CF90BF90AF909F908F907F906F9051
:1097600008952F923F924F925F926F927F928F92C5
:109770009F92AF92BF92CF92DF92EF92FF920F93A0
:109780001F93CF93DF93CDB7DEB72C970FB6F89426
:10979000DEBF0FBECDBF6C011B012A01490138019C
:1097A000BA010E94792F5C018FEFA8168FEFB806DF
:1097B00029F46DEF7EEF8FEF9FEF25C096012F5EAE
:1097C0003F4FE5E0EE2EF12C02E0A101BE016F5FFC
:1097D0007F4FC6010E94962F26E0F601248BA58AB2
:1097E0002B2D3327268B878A292D3327208F618EB7
:1097F000272D3327228F820128E035E0A101BC010B
:10980000C6010E94EA2F2C960FB6F894DEBF0FBE59
:10981000CDBFDF91CF911F910F91FF90EF90DF901F
:10982000CF90BF90AF909F908F907F906F905F9000
:109830004F903F902F9008956F927F928F929F92BA
:10984000AF92BF92CF92DF92EF92FF920F931F934E
:10985000CF93DF93CDB7DEB72C970FB6F894DEBF6A
:109860000FBECDBF6C013B014A01BA010E94792FA6
:109870005C018FEFA8168FEFB80629F46DEF7EEF2D
:109880008FEF9FEF1DC096012F5E3F4FB4E0EB2E90
:10989000F12C02E0A301BE016F5F7F4FC6010E9461
:1098A000962F22E0F601248BA58A2B2D3327268BB9
:1098B000840128E034E0A301BC01C6010E94EA2F24
:1098C0002C960FB6F894DEBF0FBECDBFDF91CF91BF
:1098D0001F910F91FF90EF90DF90CF90BF90AF90CE
:1098E0009F908F907F906F9008952F923F924F920C
:1098F0005F926F927F928F929F92AF92BF92CF9220
:10990000DF92EF92FF920F931F93CF93DF93CDB728
:10991000DEB760970FB6F894DEBF0FBECDBF5C0117
:109920007E876D87588B4F874901380127011601C3
:10993000BA010E94792F6C018FEFC8168FEFD806FD
:1099400029F46DEF7EEF8FEF9FEF30C095012F5E12
:109950003F4F53E0E52EF12C02E04D855E85BE01C0
:109960006F5F7F4FC5010E94962F2AE0F501248B7F
:10997000C58A2D2D3327268B878A292D3327208FC3
:10998000618E272D3327228F438E252D3327248F59
:10999000258E232D3327268F0F85188928E033E065
:1099A0004D855E85BC01C5010E94EA2F60960FB609
:1099B000F894DEBF0FBECDBFDF91CF911F910F9105
:1099C000FF90EF90DF90CF90BF90AF909F908F90DF
:1099D0007F906F905F904F903F902F9008952F92BF
:1099E0003F924F925F926F927F928F929F92AF922F
:1099F000BF92CF92DF92EF92FF920F931F93CF937C
:109A0000DF93CDB7DEB72C970FB6F894DEBF0FBE4D
:109A1000CDBF6C011B012A0149013801BA010E9426
:109A2000792F5C018FEFA8168FEFB80629F46DEF40
:109A30007EEF8FEF9FEF25C096012F5E3F4FB1E085
:109A4000EB2EF12C02E0A101BE016F5F7F4FC6013A
:109A50000E94962F26E0F601248BA58A2B2D332712
:109A6000268B878A292D3327208F618E272D332738
:109A7000228F820128E031E0A101BC01C6010E94D1
:109A8000EA2F2C960FB6F894DEBF0FBECDBFDF9144
:109A9000CF911F910F91FF90EF90DF90CF90BF90EB
:109AA000AF909F908F907F906F905F904F903F907E
:109AB0002F900895AF92BF92CF92DF92EF92FF92D4
:109AC0000F931F93CF93DF93CDB7DEB72C970FB6CD
:109AD000F894DEBF0FBECDBF6C015B019C012F5E11
:109AE0003F4F1EE0E12EF12C02E0AB01BE016F5FA3
:109AF0007F4F0E94962FF601148A0FEF1FEF28E088
:109B00003EE0A501BC01C6010E94EA2F2C960FB6CB
:109B1000F894DEBF0FBECDBFDF91CF911F910F91A3
:109B2000FF90EF90DF90CF90BF90AF9008954F924D
:109B30005F926F927F928F929F92AF92BF92CF92DD
:109B4000DF92EF92FF920F931F93CF93DF93CDB7E6
:109B5000DEB72C970FB6F894DEBF0FBECDBF6C01F9
:109B60002B013A014901BA010E94792F5C018FEF64
:109B7000A8168FEFB80629F46DEF7EEF8FEF9FEFF9
:109B800021C096012F5E3F4F4DE0E42EF12C02E004
:109B9000A201BE016F5F7F4FC6010E94962F24E095
:109BA000F601248BA58A2B2D3327268B878A292D16
:109BB0003327208F830128E03DE0A201BC01C601CC
:109BC0000E94EA2F2C960FB6F894DEBF0FBECDBFD1
:109BD000DF91CF911F910F91FF90EF90DF90CF9089
:109BE000BF90AF909F908F907F906F905F904F90BD
:109BF00008956F927F928F929F92AF92BF92CF9271
:109C0000DF92EF92FF920F931F93CF93DF93CDB725
:109C1000DEB72C970FB6F894DEBF0FBECDBF6C0138
:109C20003B014A01BA010E94792F5C018FEFA8160F
:109C30008FEFB80629F46DEF7EEF8FEF9FEF1DC019
:109C400096012F5E3F4F6CE0E62EF12C02E0A3015F
:109C5000BE016F5F7F4FC6010E94962F22E0F60182
:109C6000248BA58A2B2D3327268B840128E03CE00A
:109C7000A301BC01C6010E94EA2F2C960FB6F894EE
:109C8000DEBF0FBECDBFDF91CF911F910F91FF902F
:109C9000EF90DF90CF90BF90AF909F908F907F908C
:109CA0006F9008956F927F928F929F92AF92BF9222
:109CB000CF92DF92EF92FF920F931F93CF93DF9398
:109CC000CDB7DEB72C970FB6F894DEBF0FBECDBF71
:109CD0006C013B014A01BA010E94792F5C018FEFB0
:109CE000A8168FEFB80629F46DEF7EEF8FEF9FEF88
:109CF0001DC096012F5E3F4FE9E0EE2EF12C02E0F1
:109D0000A301BE016F5F7F4FC6010E94962F22E024
:109D1000F601248BA58A2B2D3327268B840128E07E
:109D200039E0A301BC01C6010E94EA2F2C960FB6B0
:109D3000F894DEBF0FBECDBFDF91CF911F910F9181
:109D4000FF90EF90DF90CF90BF90AF909F908F905B
:109D50007F906F9008956F927F928F929F92AF92B3
:109D6000BF92CF92DF92EF92FF920F931F93CF9308
:109D7000DF93CDB7DEB72C970FB6F894DEBF0FBEDA
:109D8000CDBF6C013B014A011CE6A12E13E0B12EB0
:109D9000A80EB91E9C012F5E3F4FBFE0EB2EF12CA9
:109DA00002E0AB01BE016F5F7F4F0E94962F7C01E6
:109DB000F50184819581892B39F482E090E00E943D
:109DC0002808F50195838483F501A481B5818D92DE
:109DD0009C9282E0F601848B858A892D9927868B57
:109DE0000FEF1FEF28E03FE0A301B701C6010E947B
:109DF000EA2F2C960FB6F894DEBF0FBECDBFDF91D1
:109E0000CF911F910F91FF90EF90DF90CF90BF9077
:109E1000AF909F908F907F906F9008958F929F92B8
:109E2000AF92BF92CF92DF92EF92FF920F931F9368
:109E3000CF93DF93CDB7DEB72C970FB6F894DEBF84
:109E40000FBECDBF6C014B015A01122FBA010E9407
:109E5000792F8F5F9F4F29F46DEF7EEF8FEF9FEF8C
:109E600023C096012F5E3F4F0BE0E02EF12C02E065
:109E7000A401BE016F5F7F4FC6010E94962F7C0137
:109E800087E0F601848BA6014B5E5F4FB501C601EA
:109E90000E942051F601138F850128E03BE0A401C8
:109EA000B701C6010E94EA2F2C960FB6F894DEBFC8
:109EB0000FBECDBFDF91CF911F910F91FF90EF901B
:109EC000DF90CF90BF90AF909F908F9008956F924A
:109ED0007F928F929F92BF92CF92DF92EF92FF92EA
:109EE0000F931F93CF93DF93CDB7DEB72C970FB6A9
:109EF000F894DEBF0FBECDBF6C01B62E8C010459A5
:109F00001C4FD8018D919C91892B39F481E090E010
:109F10000E942808F80191838083D801ED91FC917B
:109F2000B082B2E0BB16D9F1BB1538F0BB20C1F04E
:109F3000E1E0BE1609F07AC00AC0F4E0BF1609F1EC
:109F4000BF1628F185E0B81609F070C012C0BAE05B
:109F5000BB2E612CA4E87A2EA3E08A2E912C27C078
:109F6000FCE0BF2E612CE8E07E2EE7E08E2E912CE7
:109F70001EC073E0B72E612C6BE4762E812C912CE1
:109F800016C0612C56E9752E812C912C10C046E02C
:109F9000B42E612C31EE732E812C912C08C028E058
:109FA000B22E612C92EC792E91E0892E912C9601A3
:109FB0002F5E3F4F8FE0E82EF12C0FE340E050E0A2
:109FC000BE016F5F7F4FC6010E94962F7C0185E026
:109FD000F601848B83E0858B168A178AB08E118EEA
:109FE0000FEF1FEF2CEF3FE0A701B701C6010E9462
:109FF000EA2F6115710581059105C1F4F601828191
:10A0000093810E941818B401A3010E945C2D892B32
:10A0100069F440E050E060E070E0C7010A960E94F9
:10A02000400A60E070E080E090E004C06FEF7EEFF7
:10A030008FEF9FEF2C960FB6F894DEBF0FBECDBF0B
:10A04000DF91CF911F910F91FF90EF90DF90CF9014
:10A05000BF909F908F907F906F900895FC01E7587C
:10A06000FD4F20E030E0DC01A757BD4F81898530EE
:10A0700071F4808191818617970749F48C918295BC
:10A080008F708370682F77278827992708952F5F0F
:10A090003F4F579677962A30310541F76DEF7EEFA7
:10A0A0008FEF9FEF0895CF93DF93FC01E758FD4FAB
:10A0B00020E030E0EC01C557DD4F81898530B1F4F7
:10A0C000808191818617970789F489819A81AA27CF
:10A0D000BB272227382F492F5A2F88819927AA2753
:10A0E000BB27282B392B4A2B5B2B0BC02F5F3F4FF5
:10A0F000679677962A30310501F72DEF3EEF4FEF47
:10A100005FEFCA01B901DF91CF910895FC01E758D3
:10A11000FD4F20E030E0DC01AB57BD4F8189853039
:10A1200051F4808191818617970729F46D917D9173
:10A130008D919C9108952F5F3F4F579677962A30C7
:10A14000310561F76DEF7EEF8FEF9FEF0895DC0132
:10A15000A758BD4F30E020E0FD018189853079F4BA
:10A160006115710559F0E22FFF27EE0FFF1FE60F73
:10A17000F71F8D919C911197918380832F5F3F5F93
:10A1800057963A3049F7622F7727882799270895FD
:10A19000CF93DF93DB01FC01E358FD4F20E030E07B
:10A1A000AC0147585D4F8585853009F590818C91CC
:10A1B0009817E9F49181ED0189819817C1F4928192
:10A1C0008A819817A1F493818B81981781F49481E7
:10A1D0008C81981761F495818D81981741F4FA016B
:10A1E000808191819C01B901882799270CC02F5F3C
:10A1F0003F4F495E5F4F77962A303105A1F66DEFEC
:10A200007EEF8FEF9FEFDF91CF910895FC01E7582C
:10A21000FD4F20E08189853051F48081918186173E
:10A22000970729F460E070E080E090E008952F5FE8
:10A2300077962A3079F76DEF7EEF8FEF9FEF0895D5
:10A24000FC01E758FD4FA0E0B0E09C0123583D4FD2
:10A250008189853089F4808191818617970761F41F
:10A26000DA01F90186E001900D928150E1F760E09A
:10A2700070E080E090E008951196295E3F4F779658
:10A28000AA30B10529F76DEF7EEF8FEF9FEF0895AC
:10A29000DB01FC01EA59FC4F86E001900D928150F0
:10A2A000E1F760E070E080E090E00895FC018281D9
:10A2B0009381009719F48FEF9FEF0895019793838F
:10A2C000828380E090E008956BE671E58EE595E08D
:10A2D0000E9426720895CF93DF93C0918E07D0918C
:10A2E0008F0719C0E881F981828193819F938F93B1
:10A2F000FF93EF9383E695E09F938F930E94E46F23
:10A300000A80DB81C02D8DB79EB706960FB6F894F4
:10A310009EBF0FBE8DBF209729F7DF91CF91089583
:10A32000FC0182819381680F791F73836283892B7B
:10A3300019F4CF010E94AD0980E090E00895FC017E
:10A340008281938173836283892B19F4CF010E94E8
:10A35000AD0980E090E00895FC018281938101962F
:10A3600093838283019719F4CF010E945E0980E0F4
:10A3700090E00895CF93DF93EC0107C040E050E0F8
:10A3800060E070E0CE010E94400A8A819B810097C4
:10A39000A9F301979B838A8380E090E0DF91CF91BE
:10A3A00008950F931F93CF93DF938C01FC011182CB
:10A3B000108273836283C0918E07D0918F0720979C
:10A3C00059F484E090E00E941409FC0190938F07F7
:10A3D00080938E070CC0EC018A819B810097D9F78E
:10A3E00084E090E00E941409FC019B838A8311831E
:10A3F0000083DF91CF911F910F910895CF93DF9349
:10A40000FC01A081B181109761F0ED018A819B81EF
:10A4100091838083848195810197958384831B82B6
:10A420001A82CD01DF91CF910895FC018081918145
:10A430000895CF93DF93FC0180819181EB019B8391
:10A440008A837183608384819581892B11F473835E
:10A45000628384819581019695838483DF91CF9176
:10A460000895CF93DF93EC018C819D81009721F4B7
:10A47000CE010E9419520CC0EA81FB817383628372
:10A480007B836A83FB011382128201969D838C83F6
:10A49000DF91CF9108950F931F938C01FC01808170
:10A4A00091810E949B08C8010E949B081F910F91F7
:10A4B0000895CF93DF93EC0107C082819381998344
:10A4C0008883CF010E944B52E881F9813097A9F728
:10A4D000CE010E949B08DF91CF9108950F931F93A7
:10A4E000FC0106C002811381CF010E944B52F8018A
:10A4F0003097C1F71F910F91089586E090E00E9478
:10A500001409FC01158214821182108213821282B6
:10A510000895EF92FF920F931F938C0180E190E0DA
:10A520000E9414097C010B5D1D4FF801808191810F
:10A5300007960E941409F70191838083C7011F9138
:10A540000F91FF90EF900895CF92DF92EF92FF92DC
:10A550000F931F93CF93DF936C017B0100E010E01A
:10A56000C0E0D0E009C0C6010E948952FC01D3833B
:10A57000C2830F5F1F4FEC010E151F05A1F7CE011F
:10A58000DF91CF911F910F91FF90EF90DF90CF90CF
:10A590000895089584B7806884BF84BF089584B700
:10A5A0008F7784BF84BF0895EAE9F0E08081877FD8
:10A5B00080838B9893988A9892988C989498159801
:10A5C0001D98A1E6B0E08C918F7B8C93E2E6F0E0E1
:10A5D00080818F7B80838C918F7D8C9380818F7D18
:10A5E00080838C918F7E8C9380818F7E8083089571
:10A5F000EAE9F0E08081886080838B9A939A8A9858
:10A60000929A8C9A15980895882321F084E00E94EC
:10A610008553089584E00E9492530895882321F081
:10A6200085E00E948553089585E00E949253089525
:10A63000882321F087E00E949253089587E00E94CA
:10A6400085530895189A939A8B9A80E00E94A403E8
:10A650000895882321F086E00E94855303C086E098
:10A660000E94925380E795E00E94D45284B780689C
:10A6700084BF84BF08950F931F9300E715E0C801BE
:10A680000E94D45284B7806884BF84BF80E00E9457
:10A69000295381E00E94185368EE73E080E090E057
:10A6A0000E944E0681E00E94295364EF71E080E031
:10A6B00090E00E944E0680E00E94185384B78F7786
:10A6C00084BF84BFC8010E94F85260ED77E080E04B
:10A6D00090E00E944E061F910F9108950FB6F894D6
:10A6E0000F92E82FFF27FE2FEE2790819083C59AC7
:10A6F0000000C5980F900FBE809390070895BD9AF3
:10A70000809190070E946E53089521E030E002C0CE
:10A71000220F331F8A95E2F780919007822B0E94C7
:10A720006E53089521E030E002C0220F331F8A9556
:10A73000E2F720958091900782230E946E5308953E
:10A74000E091830AF091840A309709F00995089501
:10A75000E091850AF091860A309709F009950895ED
:10A76000E091870AF091880A309709F009950895D9
:10A77000E091890AF0918A0A309709F009950895C5
:10A78000E0918B0AF0918C0A309719F480E090E008
:10A79000089509950895E0918D0AF0918E0A3097F9
:10A7A00019F480E090E00895099599270895E091C3
:10A7B000930AF091940A309719F480E090E008959C
:10A7C00009950895E091950AF091960A309709F05D
:10A7D000099508957093900A60938F0A5093920A96
:10A7E0004093910A0895E091970AF091980A30E019
:10A7F00020E0868597858F5F9F4F09F03F5F2F5F31
:10A8000032962A30B1F7832F99270895AC01E09151
:10A81000970AF091980A20E0868597858417950716
:10A8200021F02F5F32962A30B9F780E090E02A308D
:10A8300011F081E090E00895FB0125E030E03596CD
:10A84000DC0115969C91119780813197981710F42F
:10A8500081E009C0891730F0215030408FEF2F3F41
:10A86000380781F780E0992708958F929F92AF92E1
:10A87000BF92CF92DF92EF92FF920F931F93CF93ED
:10A88000DF935C014B0189ECE82E88EFF82E012D57
:10A89000112DC0E0D0E0CC24DD241BC0BE018827F0
:10A8A0009927A80197010E94DD84F50121915F019C
:10A8B000C22FDD27C60FD71FC801B70127EB36EC23
:10A8C00045E050E00E94DD847B018C010894C11CAE
:10A8D000D11CC814D90411F7CE01DF91CF911F917B
:10A8E0000F91FF90EF90DF90CF90BF90AF909F902F
:10A8F0008F900895E091970AF091980AAA27BB27B4
:10A9000083A794A7A5A7B6A70895A091970AB09189
:10A91000980A50E040E0FD0126853785FFEF2F3F84
:10A920003F0749F0E42FFF27EE0FFF1FE80FF91F45
:10A93000318320834F5F5F5F12965A3061F7842F17
:10A940009927089581E795E00895AC01E091970A71
:10A95000F091980A20E030E0DF011E968685978509
:10A960008417950761F48FEF9FEF8D939C93E0918F
:10A97000970AF091980A82A5815082A70BC0822F76
:10A980008F5F2F5F3F4F129632962A30310531F795
:10A990008A3061F0E091970AF091980A82A58823A5
:10A9A00029F442E061E082E30E9474630895CF934A
:10A9B000DF93EC01E091970AF091980A82A5882331
:10A9C00021F440E060E00E947463E091970AF09106
:10A9D000980A20E030E0DF011E96868597858C1767
:10A9E0009D07A1F08F5F9F4F19F4CD93DC9307C0B3
:10A9F0002F5F3F4F129632962A30310571F7E09162
:10AA0000970AF091980A82A58F5F82A7DF91CF9174
:10AA1000089567EC78E586E795E00E942672089530
:10AA2000EF92FF920F931F93CF93DF93E82EFF24B3
:10AA300000E010E0C0E0D0E0A091970AB091980A41
:10AA4000FE01EA0FFB1F668577858FEF6F3F780762
:10AA500079F0FD0182A193A10E942E502E2D332763
:10AA600044275527621773078407950709F4F39461
:10AA70000F5F1F4F22960A301105F1F68F2D99278F
:10AA8000DF91CF911F910F91FF90EF9008958F92DA
:10AA90009F92AF92BF92CF92DF92EF92FF920F936D
:10AAA0001F93CF93DF93CDB7DEB727970FB6F894F8
:10AAB000DEBF0FBECDBF9C01A091970AB091980A4E
:10AAC000FD0182A5F90181937F0188249924AA249C
:10AAD000BB24A091970AB091980AF501EA0FFB1FD9
:10AAE000C684D784FFEFCF16FFEFDF06B1F1AE01CA
:10AAF0004E5F5F4FB601FD0182A193A10E942051DC
:10AB00008A819B81F70191838083E091970AF0917C
:10AB1000980AB60182A193A10E942E5087010D5F71
:10AB20001F4F611571058105910511F482E001C087
:10AB300081E0F7018283E091970AF091980A9E01E3
:10AB40002F5F3F4FA60160E070E082A193A10E94B9
:10AB5000DB7C8981F80181937F010894811C911C21
:10AB600082E090E0A80EB91E9AE08916910409F0DF
:10AB7000B0CFE091970AF091980A82A59927880FA3
:10AB8000991F880F991F019627960FB6F894DEBF7C
:10AB90000FBECDBFDF91CF911F910F91FF90EF902E
:10ABA000DF90CF90BF90AF909F908F900895E091ED
:10ABB000970AF091980AEA54FF4F10828091970A01
:10ABC0009091980A8E549F4F0E945E0908950F93AA
:10ABD0001F93CF93DF9300E010E0C0E0D0E0A0919E
:10ABE000970AB091980AFE01EA0FFB1F4685578528
:10ABF0008FEF4F3F580769F0FD0184859585481711
:10AC0000590739F023E160E070E082A193A10E942E
:10AC1000FF460F5F1F4F22960A30110501F7E091A2
:10AC2000970AF091980A448555854115510509F117
:10AC30008FEF4F3F580739F023E160E070E082A1C9
:10AC400093A10E94FF468091970A9091980AFC0177
:10AC5000DC01169686E00D9001928150E1F7E091BB
:10AC6000970AF091980A8FEF9FEF958784870E944B
:10AC7000D755DF91CF911F910F910895E091970AD9
:10AC8000F091980AEA54FF4F81E080838091970AFF
:10AC90009091980A8C549F4F0E945E090895CF931B
:10ACA000DF93CDB7DEB722970FB6F894DEBF0FBEA5
:10ACB000CDBF1A8219829E012F5F3F4F3F932F9382
:10ACC00029E735E03F932F939F938F930E941A19A2
:10ACD0002DB73EB72A5F3F4F0FB6F8943EBF0FBE69
:10ACE0002DBF019749F489819A81892B19F00E941F
:10ACF000D75502C00E943E5622960FB6F894DEBF8A
:10AD00000FBECDBFDF91CF9108950F931F93CF93C7
:10AD1000DF93CDB7DEB726970FB6F894DEBF0FBE30
:10AD2000CDBF1A8219829E012F5F3F4F3F932F9311
:10AD30008E010D5F1F4F1F930F932CE735E03F935C
:10AD40002F939F938F930E941A192DB73EB7285FB8
:10AD50003F4F0FB6F8943EBF0FBE2DBFE091970A4C
:10AD6000F091980A18161906BCF48B819C81AD816C
:10AD7000BE8187A790ABA1ABB2AB89819A81892BA9
:10AD800009F44AC0980144E050E06DE474E589E4B8
:10AD900091E40E94EA6240C087A590A9A1A9B2A946
:10ADA000BF93AF939F938F9382E895E09F938F9388
:10ADB0000E94E46F980144E050E06DE474E589E49A
:10ADC00091E40E947F622DB73EB72A5F3F4F0FB6D6
:10ADD000F8943EBF0FBE2DBF8823B1F08B819C81BC
:10ADE000AD81BE81BF93AF939F938F9386E995E02A
:10ADF0009F938F930E94E46F8DB79EB706960FB610
:10AE0000F8949EBF0FBE8DBF8DEA95E09F938F9300
:10AE10000E94E46F0F900F9026960FB6F894DEBF55
:10AE20000FBECDBFDF91CF911F910F9108950F936A
:10AE30001F93CF93DF93CDB7DEB724970FB6F89467
:10AE4000DEBF0FBECDBF19821A821B821C828E010B
:10AE50000F5F1F4F1F930F932FEA35E03F932F9300
:10AE60009F938F930E941A192DB73EB72A5F3F4FC9
:10AE70000FB6F8943EBF0FBE2DBF019751F4980155
:10AE800044E050E064E57FE48FE492E50E94EA62EA
:10AE90006CC0E091970AF091980A96818091D30650
:10AEA000981709F597818091D4069817E1F4908559
:10AEB0008091D5069817B9F491858091D606981798
:10AEC00091F492858091D706981769F493858091C3
:10AED000D806981741F481E090E0A0E0B0E08983C3
:10AEE0009A83AB83BC8389819A81AB81BC81BF93F8
:10AEF000AF939F938F9383EB95E09F938F930E94E3
:10AF0000E46F9E012F5F3F4F44E050E064E57FE433
:10AF10008FE492E50E947F622DB73EB72A5F3F4FD4
:10AF20000FB6F8943EBF0FBE2DBF8823B1F08981C4
:10AF30009A81AB81BC81BF93AF939F938F9386E936
:10AF400095E09F938F930E94E46F8DB79EB706960E
:10AF50000FB6F8949EBF0FBE8DBF8DEA95E09F930C
:10AF60008F930E94E46F0F900F9024960FB6F89481
:10AF7000DEBF0FBECDBFDF91CF911F910F9108951E
:10AF80000F931F93CF93DF93CDB7DEB726970FB6FE
:10AF9000F894DEBF0FBECDBF1A8219829E012F5FCB
:10AFA0003F4F3F932F938E010D5F1F4F1F930F93C2
:10AFB0002CE735E03F932F939F938F930E941A19AC
:10AFC0002DB73EB7285F3F4F0FB6F8943EBF0FBE78
:10AFD0002DBFE091970AF091980A18161906BCF453
:10AFE0008B819C81AD81BE8183A794A7A5A7B6A7BD
:10AFF00089819A81892B09F44AC0980144E050E084
:10B0000060E573E589E491E40E94EA6240C083A5AB
:10B0100094A5A5A5B6A5BF93AF939F938F938DEBF2
:10B0200095E09F938F930E94E46F980144E050E075
:10B0300060E573E589E491E40E947F622DB73EB735
:10B040002A5F3F4F0FB6F8943EBF0FBE2DBF882337
:10B05000B1F08B819C81AD81BE81BF93AF939F93F3
:10B060008F9386E995E09F938F930E94E46F8DB74D
:10B070009EB706960FB6F8949EBF0FBE8DBF8DEAA1
:10B0800095E09F938F930E94E46F0F900F90269608
:10B090000FB6F894DEBF0FBECDBFDF91CF911F91E9
:10B0A0000F91089581ED95E09F938F930E94E46F37
:10B0B0000F900F900895E091970AF091980A81817E
:10B0C0009927982F882720813327822B932B9F93B2
:10B0D0008F9383819927982F882722813327822B6A
:10B0E000932B9F938F9385819927982F882724816D
:10B0F0003327822B932B9F938F9381E596E09F9329
:10B100008F930E94E46F8DB79EB708960FB6F894A0
:10B110009EBF0FBE8DBF08950F931F93CF93DF93F4
:10B1200080E796E09F938F930E94E46F00E010E029
:10B130000F900F90C0E0D0E0E091970AF091980A4C
:10B14000EC0FFD1F868597852FEF8F3F920761F0EB
:10B150009F938F9387E896E09F938F930E94E46F6D
:10B160000F900F900F900F900F5F1F4F22960A3095
:10B17000110511F78DEA95E09F938F930E94E46F7C
:10B180000F900F90DF91CF911F910F910895CF9362
:10B19000DF93EC0147E050E06CE876E00E94C08469
:10B1A000892B19F40E948C5872C045E050E064E984
:10B1B00076E0CE010E94C084892BB9F40E94F2632C
:10B1C00024E042E06FE082E00E944F630E94F3536C
:10B1D00022E043E0682F82E00E944F6324E042E0D7
:10B1E0006FE082E00E944F6352C049E050E06AE99C
:10B1F00076E0CE010E94C084892B19F40E94E755A5
:10B2000046C042E050E064EA76E0CE010E94C0848D
:10B21000892B19F40E945B583AC046E050E067EA77
:10B2200076E0CE010E94C084892B29F4CE010696D7
:10B230000E944F562CC048E050E06EEA76E0CE0106
:10B240000E94C084892B29F4CE0108960E94C05721
:10B250001EC046E050E067EB76E0CE010E94C0845D
:10B26000892B29F4CE0106960E94855610C044E031
:10B2700050E06EEB76E0CE010E94C084892B29F469
:10B28000CE0104960E94175702C00E945258DF91C7
:10B29000CF9108950E943C61FDCFAF92BF92CF92B3
:10B2A000DF92EF92FF920F931F93CF93DF935C0196
:10B2B0006B017A0100E010E0C0E0D0E0A091970AB5
:10B2C000B091980AFE01EA0FFB1F468557858FEF64
:10B2D0004F3F580751F04C155D0539F0FD0126A18F
:10B2E00037A1B701C5010E947F290F5F1F4F22962A
:10B2F0000A30110519F7DF91CF911F910F91FF903F
:10B30000EF90DF90CF90BF90AF900895E091970AB3
:10B31000F091980A20EC3BE2AC0160E070E082A181
:10B3200093A10E94E1410895E091970AF091980A53
:10B33000808180FF04C080E00E94936303C080E0AE
:10B340000E947B63E091970AF091980A808181FFC7
:10B3500004C081E00E94936303C081E00E947B638C
:10B36000E091970AF091980A808182FF04C082E000
:10B370000E94936303C082E00E947B63E091970A7E
:10B38000F091980A808183FF04C083E00E94936358
:10B39000089583E00E947B6308950F931F93CF93DA
:10B3A000DF93CDB7DEB724970FB6F894DEBF0FBE9C
:10B3B000CDBF8E010F5F1F4F980144E050E064E560
:10B3C0007FE48FE492E50E947F62892B69F4198201
:10B3D0001A821B821C82980144E050E064E57FE4FD
:10B3E0008FE492E50E94EA6289819A81AB81BC81F7
:10B3F000E091970AF091980A0097A105B105F1F044
:10B400003696A3EDB6E086E00D9001928150E1F70B
:10B41000E091970AF091980AA3EDB6E086E00D90CE
:10B4200001928150E1F7E091970AF091980A158610
:10B430001486EA54FF4F81E080831EC0BF016A5F1B
:10B440007F4F82A193A10E9448518091970A9091C9
:10B45000980AFC01DC01169686E00D90019281505D
:10B46000E1F7E091970AF091980A8FEF9FEF9587A7
:10B470008487EA54FF4F10820E94945924960FB695
:10B48000F894DEBF0FBECDBFDF91CF911F910F911A
:10B4900008954F925F926F927F928F929F92AF9298
:10B4A000BF92CF92DF92EF92FF920F931F93CF93B1
:10B4B000DF93EC013B012A0169014701580187EB49
:10B4C00090E00E941409FC019093980A8093970AD7
:10B4D000D3A3C2A375A264A257A246A2EC54FF4F05
:10B4E0001182108212921292E25BF04084E190E0AD
:10B4F000A0E0B0E083A794A7A5A7B6A783E090E05B
:10B50000A0E0B0E087A790ABA1ABB2AB80E090E049
:10B510002FEF3FEFDF011E962D933D9301968A306A
:10B520009105D1F712A60E94CD59B601CE010E9415
:10B53000B46040E050E061EC7BE5CE010E94296000
:10B5400066E070E08091970A9091980A0E943554C5
:10B550000E94368342E061E082E30E947463E091DE
:10B56000970AF091980AE255FF4F80829182A28259
:10B57000B382EE5AF040A501940160E070E082A130
:10B5800093A10E94903D1F921F921F921F921F92A3
:10B59000E091970AF091980A82A193A19F938F93CB
:10B5A0000E94D6434FEFE42E4FEFF42E4FEF042FBF
:10B5B000112D1F930F93FF92EF92BF92AF929F9224
:10B5C0008F9231E0C32ED12CDF92CF9281E08F9306
:10B5D0001F921F92E091970AF091980A82A193A17D
:10B5E0009F938F930E94D64382E090E09F938F9326
:10B5F0001F930F93FF92EF92BF92AF929F928F9201
:10B60000DF92CF9282E08F931F921F92E091970A70
:10B61000F091980A82A193A19F938F930E94D643A1
:10B62000E091970AF091980A80E090E2A0E0B0E003
:10B6300083AB94ABA5ABB6AB8DB79EB787960FB671
:10B64000F8949EBF0FBE8DBF43A954A960E070E07F
:10B6500082A193A10E94D63E8091970A9091980A68
:10B6600061E070E086559F4F0E94D151E091970AAA
:10B67000F091980A40E050E060E070E082A193A170
:10B680000E94AB4E20E030E046E05DE5B201C30130
:10B690000E9403276B017C0197FD62C00091970A0D
:10B6A0001091980A66E070E0CE010E94A452F80161
:10B6B00091A780A74091970A5091980A485D5F4FE3
:10B6C000B601C3010E946F2787E495E590938C0A29
:10B6D00080938B0A8EE396E59093860A8093850A81
:10B6E00087ED95E59093880A8093870A89E095E530
:10B6F0009093840A8093830A85E894E590938E0A58
:10B7000080938D0A82EA94E59093940A8093930A39
:10B710008AE794E590938A0A8093890A87EE95E5F3
:10B720009093960A8093950A1092900A10928F0A2D
:10B730001092920A1092910A20E038E040E050E026
:10B740006AE479E583EC96E00E94070B20E038E09C
:10B7500040E050E064EB7EE58BEC96E00E94070B46
:10B76000DF91CF911F910F91FF90EF90DF90CF90DD
:10B77000BF90AF909F908F907F906F905F904F9011
:10B780000895FF920F931F93CF93DF93CDB7DEB74A
:10B7900026970FB6F894DEBF0FBECDBFF62E8A01F6
:10B7A000823009F465C0833009F07AC088E06817F8
:10B7B00031F42AE041E061E082E00E944F63E091D1
:10B7C000970AF091980A848595850817190749F515
:10B7D000DF01169686E00D9001928150E1F7E0912D
:10B7E000970AF091980A8FEF9FEF958784870E94C0
:10B7F0009459E091970AF091980ACF01C79617AA39
:10B80000F896A091970AB091980A26E00D900192BF
:10B810002150E1F747E050E0B8010E944D590E94E5
:10B82000D7558091970A9091980A86559F4F0E940C
:10B83000BA51C8010E940654882389F0C8010E94A9
:10B84000A554E0918F0AF091900A309741F0209131
:10B85000910A3091920AA8016F2D83E00995809199
:10B86000970A9091980A86559F4F0E94AC5118C034
:10B87000E091970AF091980A20EC3BE260E070E0DA
:10B8800082A193A10E94E141E091970AF091980A68
:10B89000AE014F5F5F4FB80182A193A10E9420517A
:10B8A00026960FB6F894DEBF0FBECDBFDF91CF91C5
:10B8B0001F910F91FF900895FF920F931F93CF93C5
:10B8C000DF93EC018B01F42EBC018091970A9091DB
:10B8D000980A0E941C546091970A7091980A8823D4
:10B8E00009F44AC0DB01FE0186E001900D9281500F
:10B8F000E1F7E091970AF091980A158704870E9472
:10B900009459E091970AF091980A90818091D3061A
:10B910009817D9F491818091D4069817B1F4928147
:10B920008091D506981789F493818091D60698174F
:10B9300061F494818091D706981739F495818091AC
:10B94000D806981711F40E943E56E091970AF0919C
:10B95000980ACF01C79617AAF896A091970AB091B6
:10B96000980A26E00D9001922150E1F747E050E05F
:10B97000B8010E944D5942C0CE010E941C54882338
:10B9800059F1E091970AF091980A848595850817F6
:10B990001907A1F5DF01FE0186E001900D928150AB
:10B9A000E1F70E949459E091970AF091980ACF012B
:10B9B000C79617AAF896A091970AB091980A26E020
:10B9C0000D9001922150E1F747E050E0B8010E944C
:10B9D0004D590E94D75512C082E0F81679F0E091D7
:10B9E000970AF091980A23E1A80160E070E082A133
:10B9F00093A10E94FF4681E090E002C080E090E0C9
:10BA0000DF91CF911F910F91FF900895CF92DF9218
:10BA1000EF92FF920F931F93CF93DF93CDB7DEB7D3
:10BA200026970FB6F894DEBF0FBECDBF6C018B0119
:10BA3000FC01808191810E94F0237C01F8018081CA
:10BA40008130B1F0813020F0823009F0C0C07FC079
:10BA5000DE011196F801319686E001900D92815039
:10BA6000E1F740E0B701CE0101960E945C5CAFC0F7
:10BA70008091970A9091980A86559F4F0E94BA51DB
:10BA800080E00E941055DE011196F801319686E0A3
:10BA900001900D928150E1F7E091970AF091980A98
:10BAA000B70182A193A10E9406516115710581051C
:10BAB000910509F084C041E0B701CE0101960E94D2
:10BAC0005C5C882309F07BC0C7010E94D754E091D9
:10BAD0008F0AF091900A309741F02091910A3091AD
:10BAE000920AA70161E082E00995E091970AF0913E
:10BAF000980A8F01095C1F4F82E087ABF896A091EE
:10BB0000970AB091980A86E00D9001928150E1F772
:10BB1000E091970AF091980A26A137A1A70167E062
:10BB200070E0C8010E947F296115710581059105AA
:10BB300009F445C0E091970AF091980A23E1A70122
:10BB400060E070E082A193A10E94FF4638C080911E
:10BB5000970A9091980A86559F4F0E94BA51DE012C
:10BB60001196F801319686E001900D928150E1F72F
:10BB7000E091970AF091980AB70182A193A10E94DF
:10BB800006516115710581059105C9F442E0B701BF
:10BB9000CE0101960E945C5C882389F4C7010E9453
:10BBA000D754E0918F0AF091900A309741F020919C
:10BBB000910A3091920AA70160E082E00995809194
:10BBC000970A9091980A86559F4F0E94AC51C601E2
:10BBD00026960FB6F894DEBF0FBECDBFDF91CF9192
:10BBE0001F910F91FF90EF90DF90CF900895CF922B
:10BBF000EF92FF920F931F93CF93DF93CDB7DEB7F2
:10BC00002C970FB6F894DEBF0FBECDBFCE2C7801B7
:10BC1000022F9A01AB01BE016F5F7F4F0E94CD4999
:10BC20007B018C0197FD3BC0E091970AF091980A47
:10BC300023A934A945A956A9CA01B901E6E0660FAE
:10BC4000771F881F991FEA95D1F7621B730B840B2E
:10BC5000950B24E630E040E050E00E941B85205F19
:10BC6000384D4F4F5F4FBA01A901CE010B960E948C
:10BC7000400A892B81F02AE041E06CE082E00E94DA
:10BC80004F6388E190E02FE00FB6F894A89581BD4E
:10BC90000FBE21BD04C0ED80FE800F811885C80154
:10BCA000B7012C960FB6F894DEBF0FBECDBFDF9163
:10BCB000CF911F910F91FF90EF90CF900895EF9249
:10BCC000FF920F931F93CF93DF93CDB7DEB72C97DF
:10BCD0000FB6F894DEBF0FBECDBF8901242F462FCB
:10BCE000BE016F5F7F4F0E94EF4A7B018C01E091A4
:10BCF000970AF091980A67A570A981A992A920E0F6
:10BD000035E040E050E00E94DD84AB01BC01405FC3
:10BD1000584D6F4F7F4FCE010B960E94400A892BE2
:10BD200081F02AE041E06FE082E00E944F6388E109
:10BD300090E02FE00FB6F894A89581BD0FBE21BD0D
:10BD400004C0ED80FE800F811885C801B7012C96D4
:10BD50000FB6F894DEBF0FBECDBFDF91CF911F911C
:10BD60000F91FF90EF900895CF93DF93CDB7DEB79B
:10BD7000CA5AD0400FB6F894DEBF0FBECDBF68E8F8
:10BD800073E180E090E00E944E06E091970AF09106
:10BD9000980AEA54FF4F8081E65BF040882309F05F
:10BDA0009AC0E3A4F4A405A516A50E9431835C0102
:10BDB000CC24B7FCC094DC2CC801B70128EE33E0DA
:10BDC00040E050E00E94DD849B01AC01C601B5015A
:10BDD0000E94DD842FEF3FE740E050E00E941B858A
:10BDE00028573C4E4F4F5F4F8091970A9091980A89
:10BDF000BA01A9018C549F4F0E94A90AE091970AA9
:10BE0000F091980AEA54FF4F8081882309F063C0BB
:10BE10002FEF41E060E087E00E944F63E091970AD6
:10BE2000F091980A9E012B5E3F4F4AE067A582A1E0
:10BE300093A10E945F5EC62E0E94F263DD249924C6
:10BE400046C02D2D33270091970A1091980A8FE054
:10BE500090E0289FB001299F700D389F700D11242C
:10BE60005E010894A11CB11CFB01EA0DFB1D0255EB
:10BE70001F4F238D348D458D568DF8018081918122
:10BE8000A281B3810E5A1040281739074A075B0771
:10BE9000E9F455E1E52EF12CEC0EFD1E6E0D7F1D33
:10BEA000F80182A193A10E94C85097FF0FC0E92D0D
:10BEB000FF27EE0FFF1FEA0DFB1D8FE0D89EC0018C
:10BEC0001124E80EF91EF182E0829394D394DC14DD
:10BED00009F0B7CF01C09924BB249FC0062F1127BA
:10BEE000F801EE0FFF1FE80FF91FA081B181109735
:10BEF000A9F0FFEF4F3F5F0781F0FA01EE0FFF1F40
:10BF0000E80FF91F80819181FD0125853685FC01AF
:10BF100085859685821793070CF4A8016F5FCE0183
:10BF200001966915D9F6FA01EE0FFF1FE80FF91F08
:10BF3000C080D180118210828091970A9091980AD6
:10BF400048E853E160E070E08C549F4F0E94A90ADA
:10BF5000E091970AF091980AEA54FF4F8081E65BDE
:10BF6000F040882309F06BC021E041E060E088E008
:10BF70000E944F63F6010385148526812F70E0919E
:10BF8000970AF091980AA1E0EA2E48E154E0B60140
:10BF900082A193A10E94F75D7B018C010E94F26354
:10BFA00017FD3AC0E091970AF091980A8F01095C59
:10BFB0001F4F81E087ABF896A091970AB091980A3D
:10BFC00086E00D9001928150E1F70E941055F80132
:10BFD000878368EC70E080E090E00E944E06E0917C
:10BFE000970AF091980A26A137A1A70167E070E0AF
:10BFF000C8010E947F29611571058105910561F0D5
:10C00000E091970AF091980A23E1A70160E070E0BF
:10C0100082A193A10E94FF46B394B91421F060E07D
:10C020004FEF5FEF7CCFE091970AF091980AEA54C6
:10C03000FF4F8081E65BF040882309F4A6CE40E004
:10C0400050E060E070E0CF018E549F4F0E94400AA4
:10C050009CCEE091990AF0919A0A76A765A750AB19
:10C0600047A70895CF93DF93982FA091990AB09195
:10C070009A0A1296ED018AA5882349F5E9A5FF27BA
:10C08000EE0FFF1FEE0FFF1FEA0FFB1F53834283CC
:10C09000E9A5FF27EE0FFF1FEE0FFF1FEA0FFB1FA3
:10C0A0009083E9A5FF27EE0FFF1FEE0FFF1FEA0F9A
:10C0B000FB1F618389A58F5F89A78A3009F419A6C0
:10C0C000FD0191A580A5981711F481E082A7DF9169
:10C0D000CF9108950F931F93CF93DF938C019B0112
:10C0E000A091990AB0919A0A1296ED01E8A589A546
:10C0F000E81731F48AA5882319F480E090E02EC077
:10C10000FF27EE0FFF1FEE0FFF1FEA0FFB1F8081BF
:10C11000F8018083ED01E8A5FF27EE0FFF1FEE0F6A
:10C12000FF1FEA0FFB1F8181F9018083E8A5FF272C
:10C13000EE0FFF1FEE0FFF1FEA0FFB1F828193819F
:10C14000EA0199838883FD0180A58F5F80A78A30EB
:10C1500009F410A6ED011AA681E090E0DF91CF91DD
:10C160001F910F9108950895EF92FF920F931F93DF
:10C170008C017B0184E390E00E941409FC01909300
:10C180009A0A8093990A83EB90E696A785A740E0E8
:10C1900050E063E371E6C801F701099569ED70E6C7
:10C1A00089ED96E00E9426721F910F91FF90EF900B
:10C1B00008950F931F93CF93DF93C091990AD09165
:10C1C0009A0A22968AA5882311F00AE00BC089A555
:10C1D000992728A5821B91090A966AE070E00E94BF
:10C1E0000885082F802F99279F938F9381EE96E0E3
:10C1F0009F938F930E94E46F10E00F900F900F9029
:10C200000F902AC088A5810F912D911D6AE070E0E2
:10C210000E940885FC01EE0FFF1FEE0FFF1FEC0FC1
:10C22000FD1F828193819F938F93818199279F9393
:10C230008F93808199279F938F9384E097E09F93BA
:10C240008F930E94E46F1F5F8DB79EB708960FB65D
:10C25000F8949EBF0FBE8DBF1017A1F6DF91CF914E
:10C260001F910F9108950E9432608091990A9091D8
:10C270009A0A0E945E090895CF93DF93CDB7DEB787
:10C2800024970FB6F894DEBF0FBECDBF40E050E05C
:10C2900060E070E08091990A90919A0A0E94400AA9
:10C2A0000EC0E091990AF0919A0A27A530A94B8116
:10C2B0005C8105A4F6A5E02D6A8189810995AE010E
:10C2C0004D5F5F4FBE016E5F7F4FCE0101960E94B2
:10C2D0006A60882331F7DACF6D3321F4413128F0D9
:10C2E00040E103C0453008F044E0842F99270895C9
:10C2F000FC01DC0113960E947085602D772788274A
:10C300009927982F872F762F6627DF0112960E9494
:10C310007085202D332744275527622B732B842BC0
:10C32000952B982F872F762F6627DF0111960E9475
:10C330007085202D332744275527622B732B842BA0
:10C34000952B982F872F762F6627DF010E94708507
:10C35000202D332744275527622B732B842B952BB5
:10C360000895DC010196042E0E9478859C012F5FC0
:10C370003F4FDC01052E0E947885D901062E0E94D0
:10C380007885472F5527662777272F5F3F4FD9019D
:10C39000042E0E94788508950F931F93CF93DF9307
:10C3A0008C01C8E1D0E0CE010E9478616F3F2FEF91
:10C3B00072072FEF82072FEF9207E9F061157105E1
:10C3C0008105910509F16D33710581059105C1F074
:10C3D00001151105E9F0015010409E012C5F3F4FFF
:10C3E0006D3319F4E901609602C0E901249680E1F9
:10C3F000C030D807C0F260E070E080E090E008C094
:10C400009E012C5F3F4FEECF9E012C5F3F4FEDCF43
:10C41000DF91CF911F910F910895EF92FF920F93AB
:10C420001F93CF93DF937B018C01C8E1D0E0CE0155
:10C430000E9478616E157F058007910711F4CE0187
:10C4400017C06F3F2FEF72072FEF82072FEF920772
:10C4500069F09E012C5F3F4F6D3311F4649602C06A
:10C46000E901249680E1C030D8070CF38FEF9FEFED
:10C47000DF91CF911F910F91FF90EF900895EF9270
:10C48000FF920F931F93CF93DF937B018C010E9448
:10C490000D62EC0197FF03C080E090E029C08DE3BE
:10C4A000E81639F44DE350E060E070E000E110E0A0
:10C4B00006C040E050E060E070E004E010E0CE0133
:10C4C0000E94B1619E012C5F3F4F40E050E060E070
:10C4D00006C0D9012F5F3F4F062E0E947885842F1A
:10C4E00099274F5F5F4F8017910798F381E090E0A5
:10C4F000DF91CF911F910F91FF90EF900895AF9230
:10C50000BF92CF92DF92EF92FF920F931F93CF9340
:10C51000DF93CDB7DEB761970FB6F894DEBF0FBEDD
:10C52000CDBF6B017C018A015901452B09F43FC045
:10C530000E940D6297FD3BC09C012C5F3F4F8DE335
:10C54000C81639F56E010894C11CD11CC801D90167
:10C55000F601019724F00E9470850192FACF198AA2
:10C560000C0D1D1D01501040D8011C92F6010190C8
:10C570000020E9F73197FE2EFC180F2D1127A80196
:10C58000B601C5010E94CE840A0D1B1DF801108260
:10C590000BC0C9010E947861D5016D937D938D9385
:10C5A0009C931397F1E0FF2E8F2D992702C080E016
:10C5B00090E061960FB6F894DEBF0FBECDBFDF915D
:10C5C000CF911F910F91FF90EF90DF90CF90BF9090
:10C5D000AF900895AF92BF92CF92DF92EF92FF9209
:10C5E0000F931F93CF93DF937B018C016A01590155
:10C5F0000E940D62EC0197FF1DC08DE3E81629F43F
:10C600006DE370E080E090E004C060E070E080E006
:10C6100090E00E940D62EC0197FF0CC06FEF7FEF7E
:10C620008FEF9FEF0E940D62EC0197FF03C080E047
:10C6300090E02AC04C2DC801B7010E946C616C01CA
:10C64000B801A701CE010E94B1619E012C5F3F4F4E
:10C65000EDE3EE1681F4F50107C08191D9012F5F5A
:10C660003F4F082E0E9478858E2F8A1999278C15A6
:10C670009D0598F308C0F501408151816281738165
:10C68000C9010E94B161C601DF91CF911F910F9145
:10C69000FF90EF90DF90CF90BF90AF900895A09162
:10C6A000B30ABB27FD01EE0FFF1FEE0FFF1FE3567E
:10C6B000F54F8083618342832383CD01019665E03A
:10C6C00070E00E940885282F8093B30A80919C0A0D
:10C6D000281749F4822F9927019665E070E00E949F
:10C6E000088580939C0A089580932707609391079B
:10C6F0004093280708951F93182F8091B10A88232B
:10C7000019F4812F0E940D7E81E090E002C0880F15
:10C71000991F1A95E2F7809520919B0A2823209370
:10C720009B0A1F9108951F93182F8091B10A8823A7
:10C7300019F4812F0E941B7E81E090E002C0880FD7
:10C74000991F1A95E2F720919B0A282B20939B0AA8
:10C750001F910895CF93DF93C82FDD27C0FF04C03A
:10C7600080E00E941B7E03C080E00E940D7EC1FF1E
:10C7700004C081E00E941B7E03C081E00E940D7E08
:10C78000C2FF04C082E00E941B7E03C082E00E94C0
:10C790000D7EC3FF04C083E00E941B7E03C083E0C4
:10C7A0000E940D7EDF91CF910895CF93DF93C0E07B
:10C7B000D0E080919B0A99270C2E02C09595879511
:10C7C0000A94E2F780FF04C08C2F0E941B7E03C0F6
:10C7D0008C2F0E940D7E2196C430D10551F7DF9138
:10C7E000CF9108958091B30A80939C0A0E94D563EB
:10C7F0001092B10A08951F93182F0E94297E10925B
:10C80000B30A10929C0A112351F020E034E040E07A
:10C8100050E061E174E683E297E00E94070B1F910C
:10C82000089586E90E948C07E0919C0A8091B30AE2
:10C83000E81719F41092B10A45C0FF27EE0FFF1F49
:10C84000EE0FFF1FE356F54F80818093B10A00E0A1
:10C8500010E0802F0E940D7E0F5F1F4F04301105E6
:10C86000C1F780919C0AA82FBB27FD01EE0FFF1F87
:10C87000EE0FFF1FE356F54F83818F3F11F081507C
:10C88000838312818091B10A843009F469C08530B4
:10C8900060F4813009F449C08130A0F0823009F49D
:10C8A00052C0833009F062C187C0863009F4CEC01F
:10C8B000863008F4A3C0873009F4F9C0883009F045
:10C8C00055C127C180912807882329F10E94D67578
:10C8D00020912707EFE32E9F90011124442755272D
:10C8E0000E941B856F33710581059105A0F460914D
:10C8F0009107662321F021E04091280707C080912D
:10C900009B0A882331F421E041E061E084E00E9449
:10C910004F631092B20A8091B20A8F5F8093B20A7D
:10C920006FE370E080E090E00BC081810E94AA6319
:10C930006FE3169FB0011124882777FD8095982F0B
:10C940000E944E061BC181810E94AA638FE3189F3B
:10C95000C00111247C010027F7FC0095102F21C095
:10C9600080E00E94AA638FE3189FC00111247C011C
:10C970000027F7FC0095102FC801B7010E944E0652
:10C980008091B10A882309F44FCFE0919C0AFF27D8
:10C99000EE0FFF1FEE0FFF1FE356F54F81810E9440
:10C9A000AA63C801B7010E944E068091B10A88238C
:10C9B00009F43ACF80E01FC080E00E94AA638FE3B1
:10C9C000189FC00111247C010027F7FC0095102F4F
:10C9D000C801B7010E944E068091B10A882309F46C
:10C9E00023CFE0919C0AFF27EE0FFF1FEE0FFF1FE2
:10C9F000E356F54F81810E94AA63B5C080E00E9492
:10CA00001B7EC12FDD278FE390E09C01C29FC001F8
:10CA1000C39F900DD29F900D11247C010027F7FC3D
:10CA20000095102FDD24C801B7010E944E068091A9
:10CA3000B10A882391F18D2D0E940D7ED3948D2D06
:10CA40000E941B7E33E0D31671F727C083E00E945B
:10CA50001B7EC12FDD278FE390E0FC01CE9FC0013C
:10CA6000CF9F900DDE9F900D11247C010027F7FCD5
:10CA70000095102F63E0D62EC801B7010E944E0624
:10CA80008091B10A882349F08D2D0E940D7EDA94A1
:10CA90008D2D0E941B7EDD2079F78FE390E0C89FEB
:10CAA000B001C99F700DD89F700D112445CF80E053
:10CAB0000E941B7E8FE3189FC00111246C01EE249D
:10CAC000D7FCE094FE2C10E0C701B6010E944E0690
:10CAD0008091B10A882349F0812F0E940D7E1F5F4B
:10CAE000812F0E941B7E133079F713E0C701B60136
:10CAF0000E944E068091B10A882309F495CE812FB9
:10CB00000E940D7E1150812F0E941B7E1123B1F1D6
:10CB1000EDCF80E00E941B7E81E00E941B7E82E0C0
:10CB20000E940D7E83E00E940D7E8FE3189FC0015E
:10CB300011247C010027F7FC0095102FC801B701D4
:10CB40000E944E068091B10A882309F46DCE80E0E0
:10CB50000E940D7E81E00E940D7E82E00E941B7E7D
:10CB600083E00E941B7EC801B701EACEAA0FBB1F5B
:10CB7000AA0FBB1FA356B54FFD0113828091B10AC6
:10CB8000882309F451CE80919C0A282F3327F9017C
:10CB9000EE0FFF1FEE0FFF1FE356F54F8381882333
:10CBA00009F042CEC901019665E070E00E94088557
:10CBB0002091B30A33278217930711F40E94D5639B
:10CBC00080919C0A9927019665E070E00E94088593
:10CBD00080939C0A29CEE82F81508F3118F08FEF77
:10CBE0009FEF0895FF27EE56F84F82819927089509
:10CBF000E82F81508F3120F4FF27EE56F84F6283E3
:10CC000008959C018091BC089091BD08892B19F072
:10CC10008FEF9FEF08953093BD082093BC08709369
:10CC2000BF086093BE085093BB084093BA0880E0E9
:10CC300090E008951092BD081092BC081092BF08B1
:10CC40001092BE081092BB081092BA08089581E0B5
:10CC50008093C00808951092B7081092B6081092F9
:10CC6000B5081092B4081092B9081092B808109242
:10CC7000C0081092C2081092C10840E058EC60E071
:10CC800074E082E090E00E94606990939307809343
:10CC90009207E4E9F7E08FEF819397E0E43BF9072F
:10CCA000D9F71092BD081092BC081092BF081092DC
:10CCB000BE081092BB081092BA0820E034E040E0B1
:10CCC00050E065E776E689E297E00E94070B089559
:10CCD0001092C0088091C1089091C208892B21F060
:10CCE00081EC98E00E94ED090895CF93DF93CDB7D2
:10CCF000DEB7CB50D1400FB6F894DEBF0FBECDBF2C
:10CD000088EC0E948C0740E050E060E070E088EB27
:10CD100098E00E94400AAA24BB2401C057018091D8
:10CD20009207909193070E94EC688C01E090B608FE
:10CD3000F090B7080894E108F1088091C0088823B2
:10CD400011F140E050E060E070E081EC98E00E947A
:10CD5000400AC8010E945669882389F4A090B60849
:10CD6000B090B7080894A108B108C8010E942869CA
:10CD700080919207909193070E94EC688C0188EB58
:10CD800098E00E945E094E010894811C911C4BE0C2
:10CD900050E0B401C8010E948869892B09F03FC0A6
:10CDA00089819A818A159B05D1F18091BC08909167
:10CDB000BD08892B61F18B81E091BA08F091BB0825
:10CDC000E80FF11D208133278C819927019702C03C
:10CDD000359527958A95E2F720FF19C049855A8530
:10CDE0008CE0C82ED12CCC0EDD1EB601C8010E94ED
:10CDF0008869892BA1F44091BE085091BF08E09149
:10CE0000BC08F091BD08B401C601099505C069854B
:10CE10007A85C8010E94BC680E9410088ECFC801A4
:10CE20000E9428698091B6089091B7080197E8168A
:10CE3000F90609F073CF40E050E060E070E088EB65
:10CE400098E00E94400A6ACF7F928F929F92AF92A1
:10CE5000BF92CF92DF92EF92FF920F931F93CF93E7
:10CE6000DF93CDB7DEB72B970FB6F894DEBF0FBEBA
:10CE7000CDBF6C018B014A015901809192079091BD
:10CE800093070E94EC687C01892BE9F101151105DB
:10CE900019F00C0D1D1D06C00091B6081091B708C1
:10CEA0000150104077244BE050E0BE016F5F7F4F90
:10CEB000C7010E948869892B19F589819A818C158F
:10CEC0009D05F1F049855A8564EB77E0C7010E9422
:10CED0008869892BA9F489819A818017910719F4AF
:10CEE00091E0792E02C0772041F0A501BE016F5F6D
:10CEF0007F4F84EB97E0F40109950E941008D3CF8F
:10CF0000C7010E9428692B960FB6F894DEBF0FBEAA
:10CF1000CDBFDF91CF911F910F91FF90EF90DF90E8
:10CF2000CF90BF90AF909F908F907F9008954F9239
:10CF30005F926F927F928F929F92AF92BF92CF92A9
:10CF4000DF92EF92FF920F931F93CF93DF93CDB7B2
:10CF5000DEB72B970FB6F894DEBF0FBECDBF6C01C6
:10CF6000562E442E390148018091920790919307E3
:10CF70000E94EC688C01892BE9F1EE24FF245E010C
:10CF80000894A11CB11C4BE050E0B501C8010E94FF
:10CF90008869892B61F549855A8564EB77E0C8017A
:10CFA0000E948869892B19F5552019F08B81851508
:10CFB00091F4242D33278C819927019702C0359550
:10CFC00027958A95E2F720FF06C0A401B50184EBFE
:10CFD00097E0F30109950894E11CF11CC114D104F8
:10CFE00019F0CE14DF0419F00E941008C8CFC80150
:10CFF0000E9428692B960FB6F894DEBF0FBECDBFF6
:10D00000DF91CF911F910F91FF90EF90DF90CF9024
:10D01000BF90AF909F908F907F906F905F904F9058
:10D02000089580919207909193070E944169089515
:10D03000CF93DF932EEF30E08091B4089091B50844
:10D04000281B390BEA012417350708F4E901809100
:10D050009207909193070E94DF698091B4089091A4
:10D06000B5088C0F9D1F9093B5088093B408CE012E
:10D07000DF91CF910895EF92FF920F931F93CF937B
:10D08000DF93CDB7DEB72D970FB6F894DEBF0FBE96
:10D09000CDBFFE88EF88EF2DFF27EE56F84F228197
:10D0A00033278E2D9927019702C0359527958A95AC
:10D0B000E2F720FF54C00E94D6756F837887898776
:10D0C0009A871092B5081092B4089E01265E3F4FD1
:10D0D0003A832983488D598D60E070E088E198E6B5
:10D0E0000E942D1A0091B4081091B5080E3F110549
:10D0F00061F441E050E060E377E080919207909125
:10D1000093070E94DF690FEF10E041E050E062E317
:10D1100077E080919207909193070E94DF69809158
:10D12000B6089091B7089C838B8301969093B708BB
:10D130008093B608FD82EE820F5F1F4F1C870B871E
:10D140004BE050E0BE016D5F7F4F80919207909160
:10D1500093070E94DF6988EB98E00E94AD092D9645
:10D160000FB6F894DEBF0FBECDBFDF91CF911F91F8
:10D170000F91FF90EF900895CF93DF93FC01A08172
:10D18000B1818681823019F48DEF9FEF22C08481B6
:10D1900095818617970728F482E086838EEF9FEFAC
:10D1A00018C0861B970B9583848382819381861791
:10D1B000970738F4681B790BED018885998593836F
:10D1C000828382819381861B970B9383828380E085
:10D1D00090E0DF91CF910895CF93DF93DC01EC01D4
:10D1E0008889882321F480E090E020E012C0FD01CE
:10D1F0008789882321F481E090E021E00AC0ED01D5
:10D200008E8D882319F080E090E01FC082E090E0CE
:10D2100022E0FC0133E0EE0FFF1F3A95E1F7E81B37
:10D22000F90BEA0FFB1FED018C819D8195878487A7
:10D230008E819F819787868781E0808B87E0289FFA
:10D24000C00111240A968A0F9B1FDF91CF91089588
:10D25000FC01892BA9F020813181C9010A968E1722
:10D260009F0709F41682C90141968E179F0709F49A
:10D270001682D9015896AE17BF0711F4FD01168228
:10D280000895FC018089813011F482E0808B8789C8
:10D29000813011F482E0878B868D813011F482E039
:10D2A000868F1582148217821682089520E030E05E
:10D2B000FC018681813011F421E030E0C90108953C
:10D2C000CF92DF92EF92FF920F931F937B018C011D
:10D2D0006A018FE190E00E941409FC01E082F18272
:10D2E00002831383D186C086158214821782168228
:10D2F00093878287108A928B818B178A918F808F78
:10D30000168E1F910F91FF90EF90DF90CF900895B0
:10D31000CF92DF92EF92FF920F931F93CF93DF9301
:10D32000EC016B018A01E880F9808E81823019F46A
:10D330008DEF9FEF3BC08C819D818417950728F46A
:10D3400082E08E838EEF9FEF31C0841B950B9D830F
:10D350008C832A813B812417350788F4021B130B29
:10D36000F7014081518162817381C601800F911F55
:10D370000E940E7FF701808591859B838A834A8175
:10D380005B81401B510B5B834A8366277727F7013C
:10D3900080819181A281B381480F591F6A1F7B1F31
:10D3A0009801C6010E940E7F80E090E0DF91CF914E
:10D3B0001F910F91FF90EF90DF90CF900895CF9243
:10D3C000DF92EF92FF920F931F93CF93DF93EC01C5
:10D3D0006B017A01488559854E155F0518F48EEF6B
:10D3E0009FEF62C02E813F81CA018E199F0982176B
:10D3F000930718F45F834E8304C02E0D3F1D3F83B7
:10D400002E83FE0140E052E080898130A1F42E811C
:10D410003F81888599852817390769F4868597851E
:10D420008E159F0520F4508B1786168604C08E1922
:10D430009F09978786874F5F3796433029F74C813E
:10D440005D8108851985041B150B0E151F05A0F4B9
:10D450006627772788819981AA81BB81480F591F48
:10D460006A1F7B1F9801C6010E946D7E1D821C826F
:10D47000E01AF10AC00ED11E4C815D816627772724
:10D4800088819981AA81BB81480F591F6A1F7B1F20
:10D490009701C6010E946D7E8C819D818E0D9F1D1E
:10D4A0009D838C8380E090E0DF91CF911F910F915D
:10D4B000FF90EF90DF90CF900895CF93DF93DC0142
:10D4C000E4EBFAE020E030E0AF01445F5F4F828997
:10D4D00093898F5F9F4FD9F094858C919817B9F4F9
:10D4E0009585ED018981981791F496858A81981721
:10D4F00071F497858B81981751F490898C819817D6
:10D5000031F491898D81981711F4CA010AC02F5FF7
:10D510003F4F465F5F4F3A962A303105C1F680E0B3
:10D5200090E0DF91CF9108959093400B80933F0B53
:10D530007093420B6093410B0895CF93DF93FC01EE
:10D54000C0ECDAE08E819F818617970771F598818C
:10D550008081981751F599818181981731F59A81C9
:10D560008281981711F59B8183819817F1F49C8132
:10D5700084819817D1F49D8185819817B1F4E09149
:10D580003F0BF091400B309739F04091410B509197
:10D59000420B61E0CE0109958FEF9FEF9F838E8351
:10D5A0001886198680E090E007C02A968BE0C43286
:10D5B000D80741F68FEF9FEFDF91CF91089584EB6D
:10D5C0009AE0089590933C0B80933B0B70933E0B35
:10D5D00060933D0B0895AF92BF92CF92DF92EF928E
:10D5E000FF920F931F93CF93DF937C01EB016A01AE
:10D5F00059019093BB0A8093BA0A7093BD0A609355
:10D60000BC0A5093BF0A4093BE0A64EB7AE00E94C2
:10D61000485181E08093260B10923C0B10923B0BFB
:10D6200010923E0B10923D0B1092400B10923F0B4C
:10D630001092420B1092410BE6ECFAE08FEF9FEF55
:10D640009183808312823A962BE0EA32F207C1F787
:10D6500033978FEF9FEF819391932BE0EB33F2079A
:10D66000D1F720E030E04EEE5BE6B601CE010E943D
:10D67000032740E050E0CE010E946F27A50168E03B
:10D6800070E0C7010E9481279093250B8093240BA3
:10D6900020E030E04EEB5EE6B6010E94032740E05A
:10D6A00050E063E67DE6C701F8010995DF91CF916F
:10D6B0001F910F91FF90EF90DF90CF90BF90AF90B0
:10D6C00008950E949728429708950E94072904967A
:10D6D00008950E9407290A960895EF92FF920F93EA
:10D6E0001F93CF93DF937C018B01642F722F40E057
:10D6F00050E0C0E0D0E0A0ECBAE020E030E0FD0176
:10D70000868197818F5F9F4F39F19C91F7018081CE
:10D71000981729F5FD019181F70181819817F9F496
:10D72000FD019281F70182819817C9F4FD0193816F
:10D73000F7018381981799F4FD019481F7018481A1
:10D74000981769F4FD019581F7018581981739F4DF
:10D75000E901C054D54F0BC0209709F4ED014F5F8C
:10D760005F4F265F3F4F1A964A30510541F620978A
:10D7700019F48FEF9FEF2BC08E819F818F5F9F4F9A
:10D78000C9F4DE01F70186E001900D928150E1F7C6
:10D7900068871F830E837987E0913F0BF091400BE0
:10D7A000309799F04091410B5091420B60E0CE01CF
:10D7B00009950BC08885861B813418F48EEF9FEF86
:10D7C00006C01F830E836887798780E090E0DF9131
:10D7D000CF911F910F91FF90EF9008958F929F929C
:10D7E000AF92BF92CF92DF92EF92FF920F931F936F
:10D7F000CF93DF93CDB7DEB722970FB6F894DEBF95
:10D800000FBECDBF5C016B014A01FC01808191819B
:10D810000E94F023BC01F6010089F188892B09F4EC
:10D8200052C08081823039F4C60142960E949D6ABE
:10D83000892B99F068C0813081F4F6012381418100
:10D84000C60104960E946D6BFFEF8F3F9F0709F49E
:10D850005AC08E5F9F4F09F456C0F60192858091A1
:10D86000B40A9817C9F493858091B50A9817A1F462
:10D8700094858091B60A981779F495858091B70AB6
:10D88000981751F496858091B80A981729F49785CE
:10D890008091B90A9817B9F0F6019281992319F08D
:10D8A0008381981780F10091BE0A1091BF0A7E0112
:10D8B0000894E11CF11C9401A601B5018091240B90
:10D8C0009091250B1AC011278F2D9927982F882703
:10D8D000082B192B8EEE9FEF880E991EE2E1F0E0E7
:10D8E000CE0EDF1E7E010894E11CF11C9401A601FE
:10D8F000B5018091BC0A9091BD0A0E94C327892B73
:10D9000011F4A980BA80C50122960FB6F894DEBF43
:10D910000FBECDBFDF91CF911F910F91FF90EF9080
:10D92000DF90CF90BF90AF909F908F900895AF926F
:10D93000BF92CF92DF92EF92FF920F931F93CF93FC
:10D94000DF936C015B01EA01C9014E5E5F4F60919C
:10D95000BE0A7091BF0A0E942E297B018C016115BD
:10D96000710581059105A1F462E170E0C6010E9494
:10D970000B297B018C01611571058105910531F43D
:10D98000209721F0BE01C5010E940B290E94142995
:10D99000C801B701DF91CF911F910F91FF90EF90D8
:10D9A000DF90CF90BF90AF900895AF92BF92CF928B
:10D9B000DF92EF92FF920F931F93CF93DF93EC01CF
:10D9C0005B017A0169018B818F5F8B83888188235A
:10D9D000A1F4CE010A960E945D6AFC01892B29F40C
:10D9E0006EEF7FEF8FEF9FEF23C026813781A70176
:10D9F000B501CE010E94976C1BC007E21BE0F80145
:10DA000020813181FFEF2F3F3F0741F02C153D056D
:10DA100029F0A701B501CE010E94976C0E5F1F4F40
:10DA20008BE00B33180759F760E070E080E090E07E
:10DA3000DF91CF911F910F91FF90EF90DF90CF90EA
:10DA4000BF90AF9008950F931F93CF93DF93CDB7FF
:10DA5000DEB762970FB6F894DEBF0FBECDBF8C0164
:10DA600082E089831A826B831C82DE011596E4EBC7
:10DA7000FAE086E001900D928150E1F7DE011B96FD
:10DA8000E7E8F7E086E001900D928150E1F78091A0
:10DA9000BE0A9091BF0A898B892F99278A8B20E033
:10DAA00030E046E050E0B801CE0101960E94D56C0E
:10DAB00062960FB6F894DEBF0FBECDBFDF91CF9157
:10DAC0001F910F9108958F929F92AF92BF92CF9224
:10DAD000DF92EF92FF920F931F93CF93DF93982ED5
:10DAE000862E6A0122E08217A9F4E7E2FBE080813A
:10DAF00091818C159D0509F458C08F5F9F4F39F0B7
:10DB000032968BE0EB33F80709F44FC0F0CFD182A7
:10DB1000C0824BC093E0891709F047C0E7E2FBE001
:10DB20002FEF3FEF808191818C159D0511F431839A
:10DB3000208332968BE0EB33F807A1F700EC1AE074
:10DB40005801A00EB11EE501C45BDA404AEFE42E95
:10DB50004FEFF42EEC0EFD1EF701808191818C15A4
:10DB60009D05C9F4E0913F0BF091400B309739F0DF
:10DB70004091410B5091420B61E0C80109958FEF34
:10DB80009FEFF7019183808324971992188260E0B8
:10DB9000C8010E94236D065F1F4F8AE090E0A80E27
:10DBA000B91E9BE00432190771F6E0913B0BF0912E
:10DBB0003C0B309741F020913D0B30913E0BA6017C
:10DBC000682D892D0995DF91CF911F910F91FF90BD
:10DBD000EF90DF90CF90BF90AF909F908F9008957F
:10DBE0006F927F928F929F92AF92BF92CF92DF926D
:10DBF000EF920F93CF93DF93CDB7DEB762970FB657
:10DC0000F894DEBF0FBECDBF3C015B016A01490144
:10DC10000E94972842978A159B0528F42FEF3FEF23
:10DC20004FEF5FEF96C00023F9F0F60190818091ED
:10DC30008707981719F59181809188079817F1F453
:10DC40009281809189079817C9F4938180918A07FE
:10DC50009817A1F4948180918B07981779F4958196
:10DC600080918C07981751F481E089838091260B6D
:10DC70008A838F5F8093260BEB8203C019821A82FE
:10DC80001B82EB821C82DE011596E4EBFAE086E053
:10DC900001900D928150E1F7DE011B96F60186E0BE
:10DCA00001900D928150E1F7898A892D99278A8BFD
:10DCB00020E030E0A501B301CE0101960E94D56CB1
:10DCC0009B01AC01F6016081809187076817C9F458
:10DCD0009181809188079817A1F49281809189079A
:10DCE000981779F4938180918A07981751F4948159
:10DCF00080918B07981729F4958180918C0798174C
:10DD0000F1F08091B40A681721F5F60191818091B4
:10DD1000B50A9817F1F492818091B60A9817C9F460
:10DD200093818091B70A9817A1F494818091B80AE1
:10DD3000981779F495818091B90A981751F420E0E9
:10DD400030E0A501B301CE0101960E94976C9B01C2
:10DD5000AC01CA01B90162960FB6F894DEBF0FBEDE
:10DD6000CDBFDF91CF910F91EF90DF90CF90BF901B
:10DD7000AF909F908F907F906F9008958F929F9219
:10DD8000AF92BF92CF92DF92EF92FF920F931F93C9
:10DD9000CF93DF93CDB7DEB722970FB6F894DEBFEF
:10DDA0000FBECDBF5C017B016A0172E1872E912C11
:10DDB0008E0C9F1C8EEE9FEFC80ED91EF501808140
:10DDC00091810E94F0239C01A601B401C7010E9429
:10DDD000D56CF7019285809187079817A9F59385EF
:10DDE00080918807981781F5948580918907981705
:10DDF00059F5958580918A07981731F59685809118
:10DE00008B07981709F5978580918C079817E1F48F
:10DE100080818230C9F00089112781899927982F44
:10DE20008827082B192B7E010894E11CF11C960110
:10DE3000A401B5018091BC0A9091BD0A0E94C3273C
:10DE4000892B11F4A980BA80C50122960FB6F894E7
:10DE5000DEBF0FBECDBFDF91CF911F910F91FF901D
:10DE6000EF90DF90CF90BF90AF909F908F900895EC
:10DE70009C01E091430BF091440BE657FD4F8081EC
:10DE80009181EA58F2408217930719F420E030E0BC
:10DE90000EC0E157F94F80819181EF58F64082170B
:10DEA000930719F080E090E0089521E030E085E0EC
:10DEB00094E0AC01249FC001259F900D349F900DEC
:10DEC000112486579D4F8E0F9F1F089580E090E08C
:10DED0000E94386FFC01892B19F481E090E00895CD
:10DEE0008091E3089091E40891838083ED5FFB4F7C
:10DEF0001182108280E090E008958091E308909173
:10DF0000E4080E94386FFC01892B19F481E090E04D
:10DF1000089581E08283ED5FFB4F1182108280E0E3
:10DF200090E008958091E3089091E4080E94386F92
:10DF3000DC01892B19F480E090E00895AD5FBB4FC0
:10DF4000ED91FC911197A350B440EA0FFB1F13828F
:10DF5000FD011282CD01039608950F931F93DC01FA
:10DF6000FC0101900020E9F731970E2F081B0431C6
:10DF700008F003E111278091430B9091440BA80115
:10DF8000BD01805E924F0E94CE848091430B9091A0
:10DF9000440B080F191F005E124FF80110821F91E9
:10DFA0000F9108958091430B9091440B8C5C924F9C
:10DFB0000E941D7608958091430B9091440B8C5CD8
:10DFC000924F0E943A7608950F931F93CF93DF9359
:10DFD000CDB7DEB722970FB6F894DEBF0FBECDBF28
:10DFE00009851A858091E3089091E4080E94386FB2
:10DFF000FC01892B71F08281882359F09E01255FF5
:10E000003F4F3A832983A801BF018AE290E70E942B
:10E010002D1ACE010B969A8389830E94DB6FAE0185
:10E02000455F5F4F5A834983B8018091450B9091BA
:10E03000460B0E9438198C010E94D26FC8012296AB
:10E040000FB6F894DEBF0FBECDBFDF91CF911F9109
:10E050000F9108950F931F93CF93DF938C010D5F62
:10E060001B4FF80120813181CEEFD3E0C21BD30BCF
:10E070004C175D0708F4EA010396AE01820F931F67
:10E080000E949884F801808191818C0F9D1F91835B
:10E090008083CE01DF91CF911F910F910895EF9270
:10E0A000FF920F931F937C01062F8091430B909159
:10E0B000440B8C5C924F0E943A768091450B909174
:10E0C000460B0E9418181127A801B7010E94E219F7
:10E0D0008091430B9091440B8C5C924F0E941D7673
:10E0E0001F910F91FF90EF900895EF92FF920F9381
:10E0F0001F93CF93DF93CDB7DEB722970FB6F89477
:10E10000DEBF0FBECDBF8E01055F1F4FF801E1904E
:10E11000F1908F018091430B9091440B8C5C924F56
:10E120000E943A761A830983A801B7018091450BB2
:10E130009091460B0E94377C8C018091430B90910B
:10E14000440B8C5C924F0E941D76C80122960FB63C
:10E15000F894DEBF0FBECDBFDF91CF911F910F911D
:10E16000FF90EF9008950F931F938C018091430BC4
:10E170009091440B8C5C924F0E943A766091450BD3
:10E180007091460BC8010E94CB1F8091430B909168
:10E19000440B8C5C924F0E941D761F910F91089545
:10E1A000E091430BF091440BE256F24F24E641E03C
:10E1B000608182E00E944F638091430B9091440BF9
:10E1C000865C924F0E94B37008950F931F93982F0F
:10E1D000DB01E091430BF091440BE65CF24F808150
:10E1E000EA53FD40882321F5E256F24F9083FB016C
:10E1F00001900020E9F731970E2F061B043608F036
:10E2000003E611278091430B9091440BA801BD01B7
:10E21000865C924F0E94CE848091430B9091440B78
:10E22000080F191F065C124FF80110820E94D0706F
:10E230001F910F9108958091430B9091440B805E44
:10E24000924F0E94B37008950E941B71E091430B9E
:10E25000F091440BDF01A15EB24FE25EF24F80818C
:10E26000EE51FD4022E8829FC00111248C56954F4B
:10E270006C918E0F9F1F0E944F700895CF93DF9374
:10E28000EB019093460B8093450B8FE99DE00E9434
:10E2900014099093440B8093430B009749F48BED42
:10E2A00090E09F938F930E9475700F900F902BC0FA
:10E2B000FE0101900020E9F731974E2F4C1B4531AC
:10E2C00008F044E15527BE01805E924F0E94CE8443
:10E2D00020E030E08091430B9091440BFC013B9691
:10E2E000118210823D962F5F3F4F22333105C1F7D7
:10E2F0008C5C924F0E940176E091430BF091440BAD
:10E30000E65CF24F1082DF91CF9108956F927F9279
:10E310009F92AF92BF92CF92DF92EF92FF920F93B4
:10E320001F93CF93DF937C01A090430BB090440BDD
:10E330006501662477248501962CF60183859485F2
:10E34000892BF9F0E80109900020E9F72197C01B1B
:10E35000D10BAE01B701C8010E94C084892B89F49A
:10E36000F701EC0FFD1F8081803209F44AC0F701EC
:10E3700001900020E9F73197EE19FF09CE17DF076A
:10E38000A1F093940894611C711C035F1F4F8DE0F2
:10E3900090E0C80ED91E92E36916710469F6E2E3B3
:10E3A0009E1619F481E090E043C0292D33278DE0BB
:10E3B00090E0289FF001299FF00D389FF00D112467
:10E3C000EA0DFB1DDF010D900020E9F71197AE1B50
:10E3D000BF0BAE0DBF1D8C91811111968DE090E0A9
:10E3E000289FF001299FF00D389FF00D1124EA0DB0
:10E3F000FB1D0384F485E02DCD01099580E090E0BC
:10E4000017C0262D33278DE090E0289FF001299F2B
:10E41000F00D389FF00D1124EA0DFB1DDF010D906A
:10E420000020E9F71197AE1BBF0BAE0DBF1DD5CF76
:10E43000DF91CF911F910F91FF90EF90DF90CF90E0
:10E44000BF90AF909F907F906F900895CF93DF9390
:10E45000EC01FC0101900020E9F73197E81BF90B72
:10E460003B97C0F09F938F9385EC91E09F938F93A0
:10E470000E9475708DEA91E09F938F930E94757052
:10E480004DB75EB74A5F5F4F0FB6F8945EBF0FBEE1
:10E490004DBF3EC0A091430BB091440BFD0120E065
:10E4A00083859485892BD9F02F5F3D962233C1F760
:10E4B000DF93CF9389E991E09F938F930E947570CA
:10E4C0008EE791E09F938F930E9475708DB79EB7F2
:10E4D00006960FB6F8949EBF0FBE8DBF19C03327A6
:10E4E0008DE090E0FC012E9FC0012F9F900D3E9F7C
:10E4F000900D1124A80FB91FFD0174876387209127
:10E50000430B3091440BBE01820F931F0E94B984CC
:10E51000DF91CF9108952F923F924F925F926F9229
:10E520007F928F929F92AF92BF92CF92DF92EF92A3
:10E53000FF920F931F93CF93DF93CDB7DEB723974F
:10E540000FB6F894DEBF0FBECDBF7C01062F498306
:10E5500022241FEF3324442455246624772488245E
:10E560009924AA24BB24C090430BD090440BC5012E
:10E570008C0D9D1D9B838A83FC0183859485892B4B
:10E5800009F45DC0402F5527B701CF010E94C08418
:10E59000892B09F054C0F981FF2349F11F3F19F07D
:10E5A00091E0392E08C08FED91E09F938F930E94E8
:10E5B00075700F900F908091430B9091440B880DD4
:10E5C000991D0E94B3702394822D65E00E94FC8403
:10E5D000992319F48DED91E002C08BED91E09F93AA
:10E5E0008F930E947570102F0F900F9028C01F3FBF
:10E5F00011F0202F20C0EA81FB8101900020E9F773
:10E6000031971E2F8A81181B6A817B81C7010E9466
:10E61000B98415C0122F11C0822F9927D701A80FD6
:10E62000B91FF301EC0DFD1DE80FF91F9C918081CE
:10E63000981781F72F5F211778F381E0382E08941F
:10E64000411C511CEDE0F0E0AE0EBF1E8E0E9F1E71
:10E650006E0E7F1EF2E34F16510409F084CF1F3F68
:10E6600019F4802F992723C0332031F4F701E10FEB
:10E67000F11D80E280831F5F8981882379F089ED15
:10E6800091E09F938F930E9475700E941B71612F80
:10E69000C7010E944F700F900F9007C0612F601B41
:10E6A000C701800F911D0E944F70812F99272396DB
:10E6B0000FB6F894DEBF0FBECDBFDF91CF911F9193
:10E6C0000F91FF90EF90DF90CF90BF90AF909F9011
:10E6D0008F907F906F905F904F903F902F90089514
:10E6E000DF92EF92FF920F931F93CF93DF93CDB7FB
:10E6F000DEB723970FB6F894DEBF0FBECDBF86E915
:10E700000E948C070E942471EE24DD24FF24809156
:10E71000450B9091460B0E94181841E050E0BE0155
:10E720006F5F7F4F0E94047C8F3F39F480E591E05A
:10E730009F938F930E947570E2C1813041F7809161
:10E74000450B9091460B0E9418180E94D680882392
:10E7500069F099279F938F938BE391E09F938F9319
:10E760000E9475700F900F900F900F9099819B31C0
:10E7700009F0BCC010E08091450B9091460B0E94BF
:10E780001818212F332727FD309542E050E0421B17
:10E79000530BBE016F5F7F4F620F731F0E94047C9B
:10E7A000180F123044F389818B3509F04BC08A81F0
:10E7B0008134D1F42E2D3327E091430BF091440B9B
:10E7C000E25EF24F80819927821B930B059665E0EC
:10E7D00070E00E9408850497A9F1DD2011F4EE2075
:10E7E00089F1C90104960EC0E091430BF091440BEE
:10E7F000823471F4E25EF24F8081E81619F18E2DB9
:10E800009927019665E070E00E940885E82E1AC0FD
:10E81000E25EF24FE08016C081508C9388E090E079
:10E820009F938F939F938F9385E391E09F938F9313
:10E830000E9475708DB79EB706960FB6F8949EBF6E
:10E840000FBE8DBFE091430BF091440BDF01A15E41
:10E85000B24F8C91882301F7E25EF24F4081EE5176
:10E86000FD40E41609F452CF2E2D332782E890E0C4
:10E87000289F8001299F100D389F100D11240C56E0
:10E88000154FBF01600F711F32E8F32E4F9DC0017D
:10E8900011248C56954F42E850E08E0F9F1F0E9426
:10E8A000CE848091430B9091440B800F911F0E9466
:10E8B000B3708091430B9091440B825E924FDC01C8
:10E8C000EC918E519D40EF9DF0011124EC56F54FD7
:10E8D000E80FF91FDF010D900020E9F71197AE1B3B
:10E8E000BF0B815E924FFC01A08310CF9A3019F0CC
:10E8F0009D3009F08FC0A091430BB091440BA15EF5
:10E90000B24F4C918E91AE51BD40992722E830E034
:10E91000829FF001839FF00D929FF00D1124EA0F6A
:10E92000FB1FE40FF11DEC56F54F108283E391E0DD
:10E930009F938F930E947570E091430BF091440B6D
:10E94000E15EF24F0F900F908081EF51FD408823E0
:10E9500009F45DC0E25EF24F80818F010E511D40CF
:10E9600022E8829FC00111248C56954F080F191F71
:10E97000C8010E948671882361F01F930F938CE178
:10E9800091E09F938F930E9475700F900F900F905E
:10E990000F90E091430BF091440BE25EF24F8081C7
:10E9A0008F5F8083E091430BF091440BE25EF24F66
:10E9B0008081853019F4108221E0D22EE091430B42
:10E9C000F091440BE25EF24FE190108220E030E0E3
:10E9D00042E850E0A091430BB091440BA25EB24FCD
:10E9E0008C91AE51BD409927849FF001859FF00D19
:10E9F000949FF00D1124EA0FFB1FE20FF31FEC565A
:10EA0000F54F10822F5F3F4F2238310519F70E94D2
:10EA10001B717CCE983019F09F3709F044C0E0910B
:10EA2000430BF091440BE15EF24F8081882309F49F
:10EA30006DCE88E090E09F938F939F938F9386E1B4
:10EA400091E09F938F930E947570E091430BF0913A
:10EA5000440BE15EF24F808181508083A091430B93
:10EA6000B091440BA15EB24F4C918E91AE51BD401E
:10EA7000992722E830E0829FF001839FF00D929F5A
:10EA8000F00D1124EA0FFB1FE40FF11DEC56F54FBA
:10EA90001082FF248DB79EB706960FB6F8949EBFDE
:10EAA0000FBE8DBF34CEE091430BF091440B9930F3
:10EAB000C9F48F01015E124FE25EF24F8081EE5188
:10EAC000FD4022E8829FC00111248C56954F4F2DA6
:10EAD000D8016C918E0F9F1F0E948B72F80180836A
:10EAE000F39415CEE15EF24F80818F3759F483E0C5
:10EAF00091E09F938F930E9475700E9424710F90F4
:10EB00000F9005CE892F99279F938F9380E091E0F6
:10EB10009F938F930E947570A091430BB091440B0B
:10EB2000A15EB24F4C918E91AE51BD40992722E823
:10EB300030E0829FF001839FF00D929FF00D112431
:10EB4000EA0FFB1FE40FF11DEC56F54F898180831E
:10EB5000E091430BF091440BE15EF24F80818F5FB7
:10EB60008083FF240F900F900F900F90D0CD9B01CA
:10EB7000882359F420503C4F40E050E068EC75E7A2
:10EB800084E397E00E94070B08950E947073089534
:10EB90000E947073FFCF6093C3087093C408809382
:10EBA000C5089093C6084093470B08958091470B82
:10EBB000813089F40E9441059B01AC018091C3081A
:10EBC0009091C408A091C508B091C608280F391FBC
:10EBD0004A1F5B1F10C00E9441059B01AC01809140
:10EBE000C3089091C408A091C508B091C608281B1D
:10EBF000390B4A0B5B0BCA01B90108950E9441050C
:10EC00000895FC01138212821582148211821082EF
:10EC10000895FC0184819581892B61F022813381E3
:10EC20008091E3089091E4082817390719F08FEFD5
:10EC30009FEF089580E090E00895FC0122813381E8
:10EC40008091E3089091E4082817390719F08FEFB5
:10EC50009FEF089584819581019795838483892B03
:10EC600019F080E090E00895CF010E94ED0980E066
:10EC700090E00895CF93DF93EC012A813B8180914E
:10EC8000E3089091E4082817390741F40BC040E0ED
:10EC900050E060E070E0CE010E94A90A8C819D8165
:10ECA000892BA9F78091E3089091E4089B838A83DC
:10ECB0008C819D8101969D838C83DF91CF910895F6
:10ECC000FC0184819581892B61F0228133818091BF
:10ECD000E3089091E4082817390719F08FEF9FEFA8
:10ECE0000895CF010E943A7680E090E008950F9356
:10ECF0001F93CF93DF93FC01C189D289EDA9FEA9AF
:10ED000009958C01892B49F4CF5BDF4FE881F981AC
:10ED100060E072EC81E090E00995C801DF91CF914D
:10ED20001F910F910895CF93DF93EC01EA81FB814E
:10ED30000188F289E02D0FB6F8940F9264A575A5AD
:10ED40000F900FBE88279927DF91CF910895CF921A
:10ED5000DF92EF92FF920F931F93CF93DF93EC011B
:10ED60008B017A0169018C819D81288539850FB6D7
:10ED7000F8940F92198618860F900FBE2617370742
:10ED800089F0232B21F0009711F00E94F51901154D
:10ED9000110509F1C8010E94F819009729F48FEFB5
:10EDA0009FEF1BC0672BB9F09D838C839983888369
:10EDB0009B838A83800F911F9F838E83FD86EC86C1
:10EDC000DF86CE861B861A860FB6F8940F921987B7
:10EDD00008870F900FBE80E090E0DF91CF911F91E8
:10EDE0000F91FF90EF90DF90CF900895CF92DF9238
:10EDF000EF92FF920F931F93CF93DF938A01DA0173
:10EE0000CD90DD90ED90FC902C2DFC01C189D28934
:10EE1000F1E067307F0709F464C081E0683078076B
:10EE2000ECF491E06330790709F44AC0A1E0643062
:10EE30007A0754F4B1E061307B0799F1E1E0623088
:10EE40007E0709F0CCC030C0F1E065307F0709F4DF
:10EE500042C0665071400CF041C03AC091E06B3046
:10EE6000790709F4A8C0A1E06C307A0754F4B1E046
:10EE700069307B0709F441C06A5071400CF076C0DC
:10EE800033C0F1E06D307F0709F49FC081E06D3041
:10EE900078070CF495C091E06E30790709F09FC0B7
:10EEA00099C0CF5BDF4F5FC0CD5BDF4FE881F98159
:10EEB0000995D8016D937D938D939C93139736C1DB
:10EEC000CB5BDF4FE881F9818C2D09958C0130C136
:10EED000C95BDF4F0BC0C75BDF4FF4CFC55BDF4FB4
:10EEE00005C0C35BDF4FEECFC15BDF4FE881F98127
:10EEF00009959927AA27BB2714C1C6FC03C000E0C7
:10EF000010E011C0FE01B2962685378544855585EF
:10EF100060857185CF010E94A7768C01892B19F439
:10EF2000EBADFCAD0995C7FE10C00115110509F048
:10EF3000FFC0FE017096268537854485558560851E
:10EF40007185CF010E94A7768C010115110509F08A
:10EF5000EFC0CF5ADF4F8FE39FEFAFEFBFEFC82275
:10EF6000D922EA22FB22E881F9815DC0CD5ADF4F28
:10EF7000E881F981C355D04009959B01AC01D801C6
:10EF80006D937D938D939C9313978CA59DA5892B51
:10EF900031F42064F80120833183428353838A8DC6
:10EFA0009B8D892B09F0C2C0F80180819181A281DB
:10EFB000B3818068B7C0C886D986EA86FB86B6C0AA
:10EFC00088859985AA85BB85ACC0CC86DD86EE8612
:10EFD000FF86ACC08C859D85AE85BF85A2C0FB0138
:10EFE000EF50F140E931F10540F4EA5BFF4FEE0FDD
:10EFF000FF1F0590F491E02D09940FEF1FEF98C0CB
:10F0000088819981AA81BB81222311F0806422C06A
:10F010008F7B20C088819981AA81BB8186FF27C010
:10F0200021C0EDADFEADC701B60109954FCFEF96FA
:10F03000E881F9810995F801608371838283938364
:10F0400075C088819981AA81BB81222311F08068D3
:10F0500001C08F7788839983AA83BB8367C0888127
:10F0600087FF05C081E090E0A0E0B0E05AC0D80181
:10F070001D921D921D921C92139758C0CB5ADF4FC0
:10F08000E881F981822F21CFC95ADF4F2FCFFE01AE
:10F0900070962685378544855585B601CF010E9437
:10F0A000A7768C01892B09F043C0EBADFCAD099527
:10F0B0003FC0888D998D33C0FE01B2962685378575
:10F0C00044855585B601CF010E94A776FFCE8AA55B
:10F0D0009BA525C00FB6F8940F92DD8ECC8E1AC07A
:10F0E0008C8D9D8D1CC00FB6F8940F92DF8ECE8E46
:10F0F00011C08E8D9F8D13C00FB6F8940F92DFA6AE
:10F10000CEA608C08EA59FA50AC00FB6F8940F9290
:10F11000D9AAC8AA0F900FBE09C088A999A9AA2781
:10F12000BB27F80180839183A283B38300E010E0C2
:10F13000C801DF91CF911F910F91FF90EF90DF9069
:10F14000CF900895CF92DF92EF92FF920F931F938B
:10F15000CF93DF936C018A01FC01C189D28983E0DE
:10F16000E82EF12CE422F522E114F10481F028E3E9
:10F1700030E048E250E060E470E0CE0140960E944A
:10F18000A776892BA1F4F1E0EF16F10499F020EFB6
:10F1900030E040ED50E060E071E0CE0182960E94E8
:10F1A000A776892B39F08C899D890E94F5190FEF7C
:10F1B0001FEF2CC086E090E00E94F819009739F408
:10F1C0008C899D890E94F5198EA19FA1EECF0070B8
:10F1D000107C288139814A815B810050104811F4EC
:10F1E0002F7701C02068288339834A835B838C0191
:10F1F000FC0111821082D382C28215821482F1E056
:10F20000EF16F10419F0EBADFCAD0995C801DF91E3
:10F21000CF911F910F91FF90EF90DF90CF900895C5
:10F22000CF93DF93DC01EC01EA81FB81C189D289B4
:10F2300001978E5F9F4F18F08FEF9FEF19C0CD01A0
:10F240000E94F51920E030E040E050E060E070E01E
:10F25000CE0140960E94A77620E030E040E050E0EA
:10F2600060E070E0CE0182960E94A77680E090E098
:10F27000DF91CF910895CF92DF92EF92FF920F939B
:10F280001F93CF93DF937C016A01EC0160960FB668
:10F29000F8940F928A859B85860F971F9B878A8794
:10F2A00013C0F70181AD92ADFC010995F7014485CA
:10F2B000558566857785CE0140960E94400A892B48
:10F2C00051F40FB6F8940F920A851B850F900FBE6C
:10F2D000C016D10630F3C801DF91CF911F910F9175
:10F2E000FF90EF90DF90CF9008956F927F928F9272
:10F2F0009F92AF92BF92CF92DF92EF92FF920F93C5
:10F300001F93CF93DF93CDB7DEB722970FB6F89454
:10F31000DEBF0FBECDBF4A015901FC01E188F28872
:10F32000A0E16A2E712C6E0C7F1CF3018085918503
:10F33000892B21F4FFEFCF2EDF2E9BC061157105C5
:10F3400049F440E050E060E070E0C7010E943B7982
:10F350006C018FC0F70180819181A281B3819C01F2
:10F36000AD01E9E05695479537952795EA95D1F790
:10F3700021702A8327E0B695A795979587952A95BA
:10F38000D1F7817089830FB6F8940F92F30142850B
:10F3900053850F900FBE8B0160E070E0CC24DD241C
:10F3A00050C09A01260F371FF301868597852817CD
:10F3B000390778F044855585C7010E943B79AC0137
:10F3C000F301848595858417950708F452C060E0A1
:10F3D00070E0A114B10419F0F801849102C0D801C1
:10F3E0008C91B981B13069F48A3081F4EA81E130DD
:10F3F00019F0F2E0F98303C082E08A8389838DE00B
:10F400000AC09981923011F4A1E0A9830F5F1F4FC8
:10F410000894C11CD11CD301ED91FC9111978193EB
:10F420001196FC93EE932D913C91F3018681978187
:10F430002817390721F484819581918380836F5F38
:10F440007F4FC814D9040CF4ACCF6115710589F055
:10F450000FB6F8940F92F30182859385860F971F5C
:10F46000938782870F900FBEF70181AD92ADFC01AB
:10F470000995C60122960FB6F894DEBF0FBECDBF28
:10F48000DF91CF911F910F91FF90EF90DF90CF9080
:10F49000BF90AF909F908F907F906F90089521E0E4
:10F4A00030E0FC01828193810E947579089520E00B
:10F4B00030E0FC01828193810E9475790895AF92BA
:10F4C000BF92CF92DF92EF92FF920F931F93CF9351
:10F4D000DF937B015A01EC01EA81FB8101891289EA
:10F4E000E801A296688579856115710519F48FEF99
:10F4F0009FEFA1C0E114F10461F42E853F854C8596
:10F500005D85CE010E94A776E801EBADFCAD0995C3
:10F510001AC00FB6F8940F926A857B850F900FBEC4
:10F520006115710599F4F80183AD94ADFC0109955D
:10F53000F8014085518562857385CE0140960E9411
:10F54000400A892B31F380E090E075C0D701F801C3
:10F55000808187FF35C0CC24DD24EE24FF245AE0CF
:10F560002BC0E616F70609F44FC0EA81FB814191F2
:10F57000FB83EA832A813B818E819F81281739078B
:10F5800021F48C819D819B838A834D3011F04A3018
:10F5900051F4F80184A9882311F0841751F4F8017B
:10F5A00044AB5D9303C0F80114AA4D930894C11CA9
:10F5B000D11C0894E11CF11CCA14DB0490F221C098
:10F5C0006B01A616B70608F4650140E050E0D701CC
:10F5D00014C0EA81FB8181918C93FB83EA832A81A9
:10F5E0003B818E819F812817390721F48C819D8171
:10F5F0009B838A834F5F5F4F11964C155D0549F7DA
:10F600007601E114F104B1F00FB6F8940F928A85F7
:10F610009B858E199F099B878A870F900FBE2A852D
:10F620003B858C859D852817390720F4E801EBADD3
:10F63000FCAD0995C601DF91CF911F910F91FF900D
:10F64000EF90DF90CF90BF90AF900895CF93DF936E
:10F65000DC01EC01EA81FB81309719F08D919C91DE
:10F660000995DF91CF910895EF92FF920F931F9329
:10F67000CF93DF93EC017B018A01EC81FD81309710
:10F6800019F480E090E005C060E070E080E090E078
:10F69000099519830883FB82EA82DF91CF911F913C
:10F6A0000F91FF90EF900895CF93DF93EC01EC81E1
:10F6B000FD81309719F48FEF9FEF05C060E070E097
:10F6C00081E190E00995DF91CF910895CF93DF9389
:10F6D000EC01EC81FD81309719F48FEF9FEF05C0AD
:10F6E00060E070E082E190E00995DF91CF910895AC
:10F6F0000F931F93CF93DF93CDB7DEB724970FB649
:10F70000F894DEBF0FBECDBF8C017C836B83FC0100
:10F71000248135812115310519F48FEF9FEF17C032
:10F72000BE016F5F7F4F80E290E0F901099500977D
:10F7300071F4F80124813581BE016D5F7F4F81E254
:10F7400090E0F9010995009711F489819A81249636
:10F750000FB6F894DEBF0FBECDBFDF91CF911F91E2
:10F760000F9108950F931F93CF93DF93CDB7DEB71B
:10F7700024970FB6F894DEBF0FBECDBF8C017C83FB
:10F780006B83FC01248135812115310519F48FEF3C
:10F790009FEF17C0BE016F5F7F4F88E190E0F901D6
:10F7A0000995009771F4F80124813581BE016D5FE0
:10F7B0007F4F89E190E0F9010995009711F4898163
:10F7C0009A8124960FB6F894DEBF0FBECDBFDF91AD
:10F7D000CF911F910F910895FC0140E050E060E04F
:10F7E00070E0808191810E94E219892B19F08FEFDE
:10F7F0009FEF089580E090E0089560917304709108
:10F8000074040E94A31F0895CF93DF93DC01EC01E1
:10F81000EA81FB81309719F4ED81FE8103C00788EE
:10F82000F08DE02DCD010995DF91CF910895CF9313
:10F83000DF93CDB7DEB722970FB6F894DEBF0FBEC9
:10F84000CDBFFE01379661917191FA83E983AF01D3
:10F8500080917304909174040E94377C22960FB6B5
:10F86000F894DEBF0FBECDBFDF91CF910895AF9268
:10F87000BF92CF92DF92EF92FF920F931F93CF939D
:10F88000DF935C017B016A01CB010E9482848C01C1
:10F890000F5F1F4FC8010E942808EC01009719F460
:10F8A0000FEF1FEF11C0A801B7010E946E84F50190
:10F8B000608171819601AE0182EE99E10E942D1A5C
:10F8C0008C01CE010E949B08C801DF91CF911F914E
:10F8D0000F91FF90EF90DF90CF90BF90AF90089581
:10F8E0005F926F927F928F929F92AF92BF92CF92D0
:10F8F000DF92EF92FF920F931F93CF93DF93CDB7D9
:10F90000DEB72C970FB6F894DEBF0FBECDBF6C01EB
:10F910003B01542E480181E0481719F0AA24BB246A
:10F920000DC0B901C6010E94792F5C018F5F9F4F06
:10F9300029F46DEF7EEF8FEF9FEF27C096012F5ECA
:10F940003F4F97E0E92EF12C05E0A301BE016F5F68
:10F950007F4FC6010E94962FDC01FC0114821582A4
:10F96000168217829186808683E0F601848BA58AB1
:10F970008B2D9927868B578A0FEF1FEF24E137E0F5
:10F98000A301BD01C6010E94EA2F2C960FB6F89480
:10F99000DEBF0FBECDBFDF91CF911F910F91FF90C2
:10F9A000EF90DF90CF90BF90AF909F908F907F901F
:10F9B0006F905F9008954F925F926F927F928F92B7
:10F9C0009F92AF92BF92CF92DF92EF92FF920F93EE
:10F9D0001F93CF93DF93CDB7DEB72C970FB6F89474
:10F9E000DEBF0FBECDBF6C012B014A013901BA0148
:10F9F0000E94792F5C018FEFA8168FEFB80629F4CB
:10FA00006DEF7EEF8FEF9FEF25C096012F5E3F4F8A
:10FA100042E1E42EF12C0FE3A201BE016F5F7F4FA4
:10FA2000C6010E94962FDC01FC0114821582168209
:10FA300017827186608682E0F601848BA58A8B2D01
:10FA40009927868B84012CEF32E1A201BD01C6010A
:10FA50000E94EA2F2C960FB6F894DEBF0FBECDBFE2
:10FA6000DF91CF911F910F91FF90EF90DF90CF909A
:10FA7000BF90AF909F908F907F906F905F904F90CE
:10FA800008954F925F926F927F928F929F92AF9262
:10FA9000BF92CF92DF92EF92FF920F931F93CF937B
:10FAA000DF93CDB7DEB72C970FB6F894DEBF0FBE4D
:10FAB000CDBF6C012B014A013901BA010E94792F97
:10FAC0005C018FEFA8168FEFB80629F46DEF7EEF7B
:10FAD0008FEF9FEF25C096012F5E3F4F65E0E62E2A
:10FAE000F12C05E0A201BE016F5F7F4FC6010E94AD
:10FAF000962FDC01FC011482158216821782718612
:10FB0000608682E0F601848BA58A8B2D9927868BEF
:10FB1000840124E135E0A201BD01C6010E94EA2F63
:10FB20002C960FB6F894DEBF0FBECDBFDF91CF91FC
:10FB30001F910F91FF90EF90DF90CF90BF90AF900B
:10FB40009F908F907F906F905F904F9008954F920D
:10FB50005F926F927F928F929F92AF92BF92CF925D
:10FB6000DF92EF92FF920F931F93CF93DF93CDB766
:10FB7000DEB72C970FB6F894DEBF0FBECDBF6C0179
:10FB80002B014A013901BA010E94792F5C018FEFE4
:10FB9000A8168FEFB80629F46DEF7EEF8FEF9FEF79
:10FBA00025C096012F5E3F4FE3E0EE2EF12C05E0DD
:10FBB000A201BE016F5F7F4FC6010E94962FDC013C
:10FBC000FC0114821582168217827186608682E09B
:10FBD000F601848BA58A8B2D9927868B840124E1DD
:10FBE00033E0A201BD01C6010E94EA2F2C960FB698
:10FBF000F894DEBF0FBECDBFDF91CF911F910F9163
:10FC0000FF90EF90DF90CF90BF90AF909F908F903C
:10FC10007F906F905F904F900895882321F08130FE
:10FC200011F0823019F40E9492530895833011F438
:10FC30000E9492530895882321F0813011F0823080
:10FC400019F40E9485530895833011F40E9485535E
:10FC500008950E947F5380E00E940D7E81E00E9403
:10FC60000D7E82E00E940D7E83E00E940D7E08954D
:10FC7000DC01CB0120E030E066277727480F591FD1
:10FC80006A1F7B1F40505D4C6240704010F021E0C5
:10FC900030E0C901089520E03FEE40E050E00E94CE
:10FCA0001B852F5F822F9927089520E03FEE40E0CB
:10FCB00050E00E941B85DC01CB0180509F4E0895CF
:10FCC00020E03FEE40E050E00E941B859B01AC012C
:10FCD00080E09FEE821B930B08957F928F929F92FC
:10FCE000AF92BF92CF92DF92EF92FF920F931F934A
:10FCF000CF93DF93EC015A016B0149017901002791
:10FD00001127E40EF51E061F171F20E0E2162DEC4A
:10FD1000F20622E0020720E0120708F05FC061C08F
:10FD2000272D33278F2D992701972817390709F099
:10FD300055C0C601B5010E94607E8C01C601B501A7
:10FD40000E94557E22E0721661F023E0721671F077
:10FD500021E0721609F042C0A801BE010E94728023
:10FD600009C0A801BE010E94828004C0A801BE0192
:10FD70000E949280272D33278F2D992701972817CE
:10FD8000390749F582E0F81689F023E0F216C9F048
:10FD900081E0F81619F5801A910AC00FD11FA4014D
:10FDA000BE0180E091E10E94728015C0801A910A24
:10FDB000C00FD11FA401BE0180E091E10E948280AA
:10FDC0000AC0801A910AC00FD11FA401BE0180E0B1
:10FDD00091E10E94928080E090E012C081E090E08A
:10FDE0000FC0CB01BA010E944B7E782EC801B7012B
:10FDF0000E944B7EF82E781609F092CF84019ECF98
:10FE0000DF91CF911F910F91FF90EF90DF90CF90F6
:10FE1000BF90AF909F908F907F9008957F928F9228
:10FE20009F92AF92BF92CF92DF92EF92FF920F9389
:10FE30001F93CF93DF934C015A016B01E9017901C4
:10FE400000271127E40EF51E061F171F80E0E81695
:10FE50008DECF80682E0080780E0180708F060C023
:10FE600062C0272D33278F2D99270197281739072F
:10FE700009F056C0C601B5010E94607E8C01C60122
:10FE8000B5010E94557EBC0182E0781661F083E0E6
:10FE9000781671F081E0781609F042C0A801C4011B
:10FEA0000E94A48009C0A801C4010E94B48004C0BB
:10FEB000A801C4010E94C480272D33278F2D9927C4
:10FEC00001972817390749F582E0F81689F083E091
:10FED000F816C9F081E0F81619F5C01BD10BAE0178
:10FEE00060E071E1C401800F911F0E94A48015C0E1
:10FEF000C01BD10BAE0160E071E1C401800F911F06
:10FF00000E94B4800AC0C01BD10BAE0160E071E159
:10FF1000C401800F911F0E94C48080E090E012C055
:10FF200081E090E00FC0CB01BA010E944B7E782E99
:10FF3000C801B7010E944B7EF82E781609F091CFC8
:10FF40008E019DCFDF91CF911F910F91FF90EF9088
:10FF5000DF90CF90BF90AF909F908F907F9008954B
:10FF60002F923F924F925F926F927F928F929F92C9
:10FF7000AF92BF92CF92DF92EF92FF920F931F93B7
:10FF8000CF93DF93CDB7DEB7E2970FB6F894DEBF1D
:10FF90000FBECDBF49015A01AB01BC01222433245D
:10FFA0004BC082E3C82ED12CE12CF12CC40ED51EFF
:10FFB000E61EF71ED701C6018C149D04AE04BF04D3
:10FFC00010F4D501C4012C013D01441A550A660AFA
:10FFD000770A92018E010F5F1F4FC8010E940E7FAA
:10FFE00040E050E060E070E0D8011FC0FD01E40F88
:10FFF000F51F80812826222D22952225022E269566
:020000021000EC
:1000000026952025022E269520252770022C232CAC
:10001000269507942795302C222606942795302480
:1000200022264F5F5F4F6F4F7F4F44155505660582
:100030007705E1F6B701A601481559056A057B0564
:1000400008F4AFCFC101E2960FB6F894DEBF0FBE41
:10005000CDBFDF91CF911F910F91FF90EF90DF9077
:10006000CF90BF90AF909F908F907F906F905F9058
:100070004F903F902F900895EF92FF920F931F9310
:10008000CF93DF93CDB7DEB722970FB6F894DEBFDC
:100090000FBECDBF79018A010E94B07F8983892F6D
:1000A00099278A8322E030E0B801A701CE010196AA
:1000B0000E946D7E22960FB6F894DEBF0FBECDBFB4
:1000C000DF91CF911F910F91FF90EF9008952E5FD8
:1000D0003F4F4F4F5F4F0E94B07F009711F081E07C
:1000E00090E00895FB01DC01E89447F4689406C0B1
:1000F000F8940190C79A0D92C79878944150504057
:10010000B8F70895FB01DC01E89447F4689406C051
:10011000F8940190C69A0D92C69878944150504038
:10012000B8F70895FB01DC01E89457F4689408C01F
:10013000F8940190C79AC69A0D92C798C698789479
:1001400041505040A8F70895FB01DC01E89447F4C2
:10015000689406C0F894C79A0190C7980D92789455
:1001600041505040B8F70895FB01DC01E89447F492
:10017000689406C0F894C69A0190C6980D92789437
:1001800041505040B8F70895FB01DC01E89457F462
:10019000689408C0F894C79AC69A0190C798C69800
:1001A0000D92789441505040A8F70895DF92EF9255
:1001B000FF920F931F93CF93DF93CDB7DEB72497B2
:1001C0000FB6F894DEBF0FBECDBF8C017E01089440
:1001D000E11CF11CA7016AE071E00E9478192981F5
:1001E0003A814B815C81DA01C90187709070A070FF
:1001F000B0700097A105B10511F4DD2411C087E0AE
:10020000D82ED22287E090E0A0E0B0E089839A83E4
:10021000AB83BC83A70169E071E0C8010E94781933
:100220008D2D992724960FB6F894DEBF0FBECDBF53
:10023000DF91CF911F910F91FF90EF90DF90089584
:10024000CF92DF92EF92FF920F931F93CF93DF93A2
:100250006C01EB01E42EFF243BC08E01020F131F43
:10026000C6010E94181841E050E0B8010E94047CC9
:10027000F8010081083011F00F3761F4FF2041F1DF
:100280008FE397E09F938F930E94E46FFA940F900F
:100290000F901EC00A3011F00D3049F483E497E04E
:1002A0009F938F930E94E46F0F900F901AC0802F3E
:1002B000992787FD90959F938F9385E497E09F936F
:1002C0008F930E94E46FF3940F900F900F900F9014
:1002D0002F2D33278E2D99270197281739070CF4D6
:1002E000BCCFCF0DD11D1882F3948F2D9927DF91AC
:1002F000CF911F910F91FF90EF90DF90CF900895D5
:10030000FC01808199279F938F93818199279F93E7
:100310008F93828199279F938F93838199279F93AE
:100320008F93848199279F938F93858199279F939A
:100330008F9388E497E09F938F930E94E46F8DB72B
:100340009EB70E960FB6F8949EBF0FBE8DBF089550
:100350005F926F927F928F929F92AF92BF92CF9255
:10036000DF92EF92FF920F931F93CF93DF934C0195
:100370003B01EC0101C0219688818032E1F35301F9
:1003800095E0592E1881E12EFF24E7FCF094C70177
:100390000E945185892B89F10981C02EDD24C7FC7B
:1003A000D094C6010E945185892B39F11A3314F477
:1003B000105305C0C7010E946A85182F17550A33CC
:1003C0001CF4802F805304C0C6010E946A858755A3
:1003D0001295107F182BF5011583CE01029655203A
:1003E000A9F08A818A3349F423965A940894A10883
:1003F000B108FFEF5F1659F0C5CFF301A7E8B7E0EA
:1004000086E00D900192815019F0FBCFEC014E0176
:10041000C401DF91CF911F910F91FF90EF90DF907A
:10042000CF90BF90AF909F908F907F906F905F9094
:1004300008950F931F93FC01808199279F938F93B9
:10044000818199279F938F93828199279F938F937F
:10045000838199279F938F93848199279F938F936B
:10046000858199279F938F9388E497E09F938F933B
:1004700007EC18E01F930F930E9486828DB79EB7FA
:1004800040960FB6F8949EBF0FBE8DBFC8011F9156
:100490000F910895AF92BF92CF92DF92EF92FF92A9
:1004A0000F931F93CF93DF937C015B016A01EC01F3
:1004B00000E010E018C0EA0DFB1D808199279F9392
:1004C0008F9386E697E09F938F93DF93CF930E945D
:1004D0008682C80FD91F8DB79EB706960FB6F894BF
:1004E0009EBF0FBE8DBFE02FFF270F5F1F4FEC1584
:1004F000FD0508F3C701DF91CF911F910F91FF9088
:10050000EF90DF90CF90BF90AF900895CF93DF939F
:10051000CDB7DEB722970FB6F894DEBF0FBECDBFC2
:10052000AE01455F5F4F5A83498369857A858F8124
:1005300098850E94A48222960FB6F894DEBF0FBE63
:10054000CDBFDF91CF910895CF93DF93CDB7DEB7C5
:1005500022970FB6F894DEBF0FBECDBF9A83898372
:100560009A01AB01BE016F5F7F4F85EC92E80E945C
:100570002D1AE981FA81108222960FB6F894DEBF17
:100580000FBECDBFDF91CF910895EF92FF920F93F1
:100590001F937C018A01FC01808191810E949884D3
:1005A000F70180819181800F911F91838083C80121
:1005B0001F910F91FF90EF900895AF92BF92CF924D
:1005C000DF92EF92FF920F931F93CF93DF93EC0193
:1005D000E880F9800A811B81C801B7012DE133EF62
:1005E00041E050E00E941B8527EA31E440E050E002
:1005F0000E94DD845B016C01C801B7012DE133EF7E
:1006000041E050E00E941B85CA01B90124E13BE0B2
:1006100040E050E00E94DD84A61AB70AC80AD90A51
:100620001A141B041C041D0444F08FEF9FEFAFEF5E
:10063000BFE7A80EB91ECA1EDB1EA882B982CA82F5
:10064000DB82C5019F77DF91CF911F910F91FF90C2
:10065000EF90DF90CF90BF90AF9008950E94DD8221
:1006600008958CE697E00E94DD820895AA27BB27B3
:1006700080936C0790936D07A0936E07B0936F07FC
:1006800008953F924F925F926F927F928F929F92C6
:10069000AF92BF92CF92DF92EF92FF920F931F9390
:1006A000CF93DF938C012B01EA016115710519F0DD
:1006B000FB0191838083209749F0CE0102978397B5
:1006C00028F060E070E080E090E0F6C0F801E19092
:1006D0008F018E2D99270E945B85892BB9F7FDE24A
:1006E000EF1631F4F801E1908F0181E0382E07C058
:1006F000FBE2EF1619F4F801E1908F013324209703
:1007000019F0C031D105C1F4F0E3EF1679F4F80126
:100710008081883711F0883549F4F801E1800E5F57
:100720001F4FF2E03F2AC0E1D0E006C0209721F43D
:1007300080E3E816E9F427C0C830D10531F1C930AB
:10074000D10524F4C230D10531F50CC0CA30D10531
:1007500089F0C031D105F9F4A12CB12CC12CB8E03D
:10076000DB2E26C0A12CB12CC12CA0E4DA2E20C097
:10077000CAE0D0E0FCECAF2EFCECBF2EFCECCF2EA0
:10078000FCE0DF2E15C0C8E0D0E0A12CB12CC12CBC
:10079000E0E1DE2E0DC09E01442737FD4095542F29
:1007A00060E070E080E090E80E941B8559016A01DA
:1007B00020E030E040E050E060E03E01882477FC3B
:1007C0008094982C70EDF72EFE0CE9E0EF1570F494
:1007D0008E2D81548A3118F499ECF92E06C08E2D95
:1007E00081568A3150F589EAF82EFE0C8F2D992713
:1007F0008C179D0714F567FD1CC0A216B306C4062E
:10080000D506B0F0CA01B901A40193010E94DD84AC
:100810009B01AC012F0D311D411D511D2130F0E018
:100820003F07F0E04F07F0E85F0710F461E001C018
:100830006FEFF801E1908F01C5CF4114510481F0B1
:10084000662331F001501040F2011183008308C08B
:1008500031FE1AC002501040F2011183008314C00F
:1008600067FF12C030FE05C020E030E040E050E8F5
:1008700004C02FEF3FEF4FEF5FE782E290E09093ED
:10088000490B8093480B16C030FE08C05095409528
:10089000309521953F4F4F4F5F4F0CC057FF0AC017
:1008A00082E290E09093490B8093480B2FEF3FEF4B
:1008B0004FEF5FE7CA01B901DF91CF911F910F910F
:1008C000FF90EF90DF90CF90BF90AF909F908F9070
:1008D0007F906F905F904F903F900895FB01DC01F7
:1008E00040FF05C002C005900D9205900D92425048
:1008F0005040C8F70895FB01DC0105900D920020DF
:10090000E1F70895FC0105900020E9F780959095A6
:100910008E0F9F1F0895FC014150504030F0019010
:100920000616D1F73197CF010895882799270895A2
:10093000FB01DC0140FF05C002C001900D92019057
:100940000D9242505040C8F70895DC0140FF03C0AB
:1009500001C06D936D9342505040D8F70895FB014C
:10096000DC018D910190801911F40020D1F7990BD1
:100970000895FB01DC0101900D920020E1F708953C
:10098000FB01DC014150504030F08D910190801905
:1009900019F40020B9F7881B990B0895FB01DC01BD
:1009A0004150504048F001900D920020C9F701C01D
:1009B0001D9241505040E0F70895629FD001739F0F
:1009C000F001829FE00DF11D649FE00DF11D929FEB
:1009D000F00D839FF00D749FF00D659FF00D99272A
:1009E000729FB00DE11DF91F639FB00DE11DF91F4E
:1009F000BD01CF0111240895991B79E004C0991F0E
:100A0000961708F0961B881F7A95C9F78095089568
:100A100097FB092E07260AD077FD04D02ED006D0EA
:100A200000201AF4709561957F4F0895F6F7909520
:100A300081959F4F0895A1E21A2EAA1BBB1BFD01B1
:100A40000DC0AA1FBB1FEE1FFF1FA217B307E407AD
:100A5000F50720F0A21BB30BE40BF50B661F771F05
:100A6000881F991F1A9469F76095709580959095E5
:100A70009B01AC01BD01CF010895AA1BBB1B51E135
:100A800007C0AA1FBB1FA617B70710F0A61BB70BFE
:100A9000881F991F5A95A9F780959095BC01CD01A3
:100AA0000895082E8062813624F087360CF408956C
:100AB0002BC0802D36C0911127C0803251F08A3072
:100AC00041F08C3031F08D3021F0893011F08B30D5
:100AD00099F708958F931DD08F9109F08062089542
:100AE000E199FECFBFBBAEBBE09A11960DB208955F
:100AF000E199FECFBFBBAEBB0DBA11960FB6F8940D
:100B0000E29AE19A0FBE089599278827089585FDF6
:100B1000FBCF80629111F8CF8136ECF38B37DCF795
:0E0B200008959111F1CF80538A50E0F70895A7
:100B2E006572726F72207265676973746572696E31
:100B3E006720626C696E6B207365727669636521DE
:100B4E0000722B000A23202D2D2D2D2D2D2D2D2D18
:100B5E002D2D2D2D2D2D2D2D2D2D2D2D2D2D2D2DB7
:100B6E002D2D2D2D2D2D2D2D2D2D2D2D2D2D2D2DA7
:100B7E002D2D2D000A232057656C636F6D65207433
:100B8E006F2042546E75742028632920323030361F
:100B9E0020455448205A75726963680032303036E9
:100BAE00313231382D3135313800232070726F6774
:100BBE0072616D2076657273696F6E3A2025730AC5
:100BCE000023202D2D2D2D2D2D2D2D2D2D2D2D2D8B
:100BDE002D2D2D2D2D2D2D2D2D2D2D2D2D2D2D2D37
:100BEE002D2D2D2D2D2D2D2D2D2D2D2D2D2D2D0054
:100BFE000A626F6F74696E6720626C7565746F6FD1
:100C0E007468206D6F64756C652E2E2E20006F6BD0
:100C1E002E0A0D00696E69742062742D73746163FF
:100C2E006B2E2E2E2000646F6E652E00736574740D
:100C3E00696E672061636C20706B742074797065C7
:100C4E00732E2E2E2000696E69742070726F74637D
:100C5E006F6C2F73657276696365206D75782E2EB5
:100C6E002E2000696E697420636F6E6E6563746901
:100C7E006F6E6C657373206C326361702E2E2E2036
:100C8E0000696E697420636F6E6E656374696F6E52
:100C9E00206D616E616765722E2E2E2000696E6961
:100CAE007420636F6E6E656374696F6E6C657373BB
:100CBE00206D756C74692D686F702070726F746F13
:100CCE00636F6C2E2E2E20005B6D626C696E6B4016
:100CDE0062746E6F64655D2400686974207461626D
:100CEE0020747769636520666F722061206C69736A
:100CFE0074206F6620636F6D6D616E64730A0D00F4
:100D0E00626C696E6B007265706C79002532783A90
:100D1E002532783A2532783A2532783A2532783AA1
:100D2E0025327800626C696E6B207265706C79206A
:100D3E0073656E743A2025640A006572726F7220B4
:100D4E0075736167653A20626C696E6B203C6164F5
:100D5E0064723E0A00626C696E6B2072717374204D
:100D6E0073656E742E0A0065746865726E75740014
:100D7E0069646C65006D61696E00FF000000001F04
:100D8E000C00007561727430000000000500000058
:100D9E00000084037776F6765F7A577A4F7AA278D8
:100DAE0010799376000000000000000000000000A3
:100DBE000000000000000000000000000000000025
:100DCE000000000000000000000000000000000015
:100DDE00000000000000000000A60F7D0FC60EC828
:100DEE000ECB0FA60E2610300FF40E880DA210A5F6
:100DFE000DD610B60D2A0EC00D66108F0E000075A2
:100E0E006172743100000000050100000000000452
:100E1E007776F6765F7A577A4F7AA278107993764C
:100E2E0000000000000000000000000000000000B4
:100E3E0000000000000000000000000000000000A4
:100E4E000000000000000000000000000000000094
:100E5E000000000000981350147113771369145199
:100E6E0013C4140014BB13231253154212881553C6
:100E7E0012C9125D120815381300000000E31500A8
:100E8E00000000941600000000001700000000642F
:100E9E001701000200030000000000000000000027
:100EAE0000286E756C6C290030313233343536378C
:100EBE0038396162636465660030313233343536F9
:100ECE003738394142434445460020202020202017
:100EDE0020202020202020202020303030303030A4
:100EEE003030303030303030303031323334004208
:100EFE0054537461636B0070736D7578005F554168
:100F0E0052547772697465206572726F72210A008D
:100F1E005F5541525472656164206572726F722121
:100F2E000A006672616D696E67206572726F720A71
:100F3E0000627566666572206F76657272756E20D8
:100F4E006572726F720A00706172697479206572CF
:100F5E00726F720A007061636B6574206F75742016
:100F6E006F662073796E6320746F20425420756112
:100F7E007274210A00722B00307825580A007365AE
:100F8E006D610073656D612025703A2025640A003D
:100F9E00005472656500636D00257500256C75251E
:100FAE007500417574696E71206C656E6774683A70
:100FBE0020256C752E002053746F72656420696E47
:100FCE0020454550524F4D3A20256C75000A00259C
:100FDE006C7500526F6F743A2025752E0041757432
:100FEE00696E7120706572696F643A20256C752E7A
:100FFE0000636D3A206572723A2075736167653AC7
:10100E000A69640A72656C636F6E730A617574693E
:10101E006E71205B20307C31205B307C315D205D39
:10102E000A6169706572696F64205B205345434F96
:10103E004E4453205B307C315D205D0A61697469DA
:10104E006D65205B205345434F4E4453205B307CEF
:10105E00315D205D0A626C696E6B0A726F6F74206F
:10106E005B307C315D0A646973636F6E616C6C0A10
:10107E00004C6F63616C20747265652049443A20A0
:10108E00252E34783A252E34783A252E34780A00D7
:10109E0072656C6961626C6520636F6E6E656374F8
:1010AE00696F6E733A0A0025752C200072656C63A9
:1010BE006F6E7300626C696E6B00646973636F6E42
:1010CE00616C6C00696400617574696E71006169B0
:1010DE00706572696F6400616974696D6500726F25
:1010EE006F7400434F4E5F42554600436F6E6D67FF
:1010FE00724900F8FFFFFFFFFF636F6E5F62756658
:10110E0000636F6E206576656E7420627566666527
:10111E0072207769746820256420656E7472696523
:10112E00733A0A00747970652025642C2064657406
:10113E0061696C2025642C2068616E646C652025C5
:10114E00640A004C4544000F014C6F6745767400ED
:10115E000A000000545F5445524D494E414C000860
:10116E002008000A00256300252E32783A252E32FB
:10117E00783A252E32783A252E32783A252E327844
:10118E003A252E327800252E3278200001000000FC
:00000001FF
